:020000040800F2
:1020000070890020452100084D2100084F2100085B
:10201000512100085321000855210008000000004C
:102020000000000000000000000000005721000830
:1020300059210008000000005B2100085D21000814
:102040005F2100085F2100085F2100085F21000870
:102050005F2100085F2100085F2100085F21000860
:102060005F2100085F2100085F2100085F21000850
:102070005F2100085F2100085F2100085F21000840
:102080005F2100085F2100085F2100085F21000830
:102090005F2100085F2100085F2100085F21000820
:1020A0005F2100085F2100085F2100085F21000810
:1020B0005F21000889E60108D1E601085F210008D8
:1020C0005F2100085F2100085F2100085F210008F0
:1020D0005F2100085DF501085F21000835F6010861
:1020E0005F2100085F2100085F2100085F210008D0
:1020F0005F2100085F2100085F2100085F210008C0
:102100005F2100085F2100085F2100085F210008AF
:102110005F2100085F2100085F2100085F2100089F
:102120005F2100085F2100085F2100085F2100088F
:10213000DFF80CD000F042FC004800473577020879
:10214000708900200648804706480047FEE7FEE702
:10215000FEE7FEE7FEE7FEE7FEE7FEE7FEE7FEE757
:1021600081C10108312100082DE9F05F05460020FA
:1021700092469B4688460646814640241BE02846F8
:1021800041464746224600F0BAF953465A46C01A1D
:10219000914110D311461846224600F0A1F92D1A9C
:1021A00067EB01084F4622460120002100F098F914
:1021B00017EB00094E41201EA4F10104DFDC484664
:1021C00031462A464346BDE8F09F000038B5D0E9C5
:1021D0000221491E01EB410102EBC1014268C1EB42
:1021E000011102EB81010268C1EB011102EB8103D5
:1021F000D0E9042101EB410102EB8101A1F552710B
:10220000302491FBF4F2154D04FB1211554303EBFE
:10221000C51300931A2902DB114A1A4400920C23B9
:1022200091FBF3F20F4C009D544303FB121105EB9D
:10223000C4140D4B009408E0491E40F2A3245A5CDC
:102240006243009C04EBC21200920029F4DC0146B8
:10225000684600F06FF9009838BD00003F0C0F0091
:102260008051010067C2030013AE020840EA010377
:102270009B0703D009E008C9121F08C0042AFAD23C
:1022800003E011F8013B00F8013B521EF9D2704700
:10229000D2B201E000F8012B491EFBD270470022A8
:1022A000F6E710B513460A4604461946FFF7F0FF55
:1022B000204610BD421E12F8013F002BFBD111F841
:1022C000013B02F8013B002BF9D1704730B50546C0
:1022D0002A460B4612F8010B13F8014B08B1A04235
:1022E000F8D01CB1002802D06D1CF1E7284630BDA3
:1022F00010B5044604E00B7800F8013B03B1491C1B
:10230000521EF8D2204610BDCAB2401E10F8011F5E
:102310008A4202D00029F9D100207047421C10F8EF
:10232000011B0029FBD1801A704710B5002200E084
:10233000521C835C8C5CA34201D1002BF8D1D8B233
:10234000E1B2401A10BD30B504460020034600E05B
:102350005B1C934203D2E05CCD5C401BF8D030BDE7
:10236000034611F8012B00F8012B002AF9D1184679
:1023700070472DE9F04791460F46804604460026F7
:1023800014F8015B2DB100F0CBF80068405DC00788
:10239000F6D12B2D02D02D2D18D0641E4A46394679
:1023A000204600F007F927B13968A14201D1C7F8EA
:1023B000008071054FF002040BD54042002803DD78
:1023C00024F0EEF80460A007BDE8F08746F48066CC
:1023D000E4E70028F8DA24F0E3F804606FF0004046
:1023E000F2E770B5064624F0DBF8046805460A22D9
:1023F00000213046FFF7BDFF2C6070BD70B506466A
:1024000024F0CEF8046805460A2200213046FFF782
:10241000B0FF2C6070BD80EA010210B502F00043ED
:10242000400026D04A0023D04FEA106101EB126130
:10243000C0F35600C2F3560240F4000042F400021A
:10244000A0FB0220A1F17F014FEA0040140401D05B
:1024500000F1010050EA124001D44000491EC2B20E
:102460000C0604EBD010401C4008802A02D003E088
:10247000002010BD20F00100002900DA00201843E0
:1024800010BD00F0004220F00040C10DC0F3160066
:1024900040F400007F2901DA00207047962903DC10
:1024A000C1F19601C84001E096398840002AF4D075
:1024B0004042704730B50B460146002020220124DF
:1024C00009E021FA02F59D4205D303FA02F5491B02
:1024D00004FA02F52844151EA2F10102F1DC30BD18
:1024E000202A04DB203A00FA02F1002070479140D4
:1024F000C2F1200320FA03F3194390407047202AC9
:1025000004DB203A21FA02F00021704721FA02F39D
:10251000D040C2F1200291400843194670470000A4
:1025200000487047A0AE0208014900F003B800005F
:102530004461002030B503683C22B3FBF2F002FB9B
:1025400010330B60B0FBF2F302FB13001824486059
:10255000B3FBF4F004FB10328A60021D0723B2FBC8
:10256000F3F403FB14228A61820002F66C3240F21B
:10257000B555B2FBF5F404F144000346486105FB90
:1025800014208008C8613B2802D39A0700D0401C61
:102590000022074C13460A61E25C824203D8801A8B
:1025A0005B1C0B61F8E7401CC860084630BD0000AA
:1025B000A4AE02082DE9F05F824600780027154698
:1025C0008B460AF10104B946302801D09DB113E0D1
:1025D00014F8010B0127782803D0582801D045B101
:1025E0000AE00DB1102D07D10027102514F8010BBA
:1025F00002E0082500E00A250026B0460EE005FBB3
:10260000080005FB06F1012701EB10461FFA80F8D0
:10261000B6F5803F00D3B94614F8010B294600F007
:10262000F1F90028EBDABBF1000F05D00FB1641E01
:1026300000E05446CBF80040B9F1000F06D023F07B
:10264000AFFF02210160C81EBDE8F09F48EA0640C6
:10265000FAE72DE9FE4F804681EA0300C00F0C46E1
:10266000009021F0004123F00045B8EB0200A941A1
:1026700005D24046214690461C460B46024623F0B2
:102680000040104304D14046214603B0BDE8F08F1E
:10269000270DC7F30A00C3F30A510290401A0190B4
:1026A000402866DAC3F3130040F4801B009892467A
:1026B00020B10023D2EB030A63EB0B0B01985946C0
:1026C000C0F140025046FFF70BFF06460D4650464C
:1026D0005946019A00F084F910EB0800614100248A
:1026E00087EA115284EAE7731A433BD0009A3AB35F
:1026F000019A012A4FEA075210DC001B61EB02012C
:102700004FF0004202EA0752CDE90042001C41F5B9
:10271000801132462B4600F090F9B6E7001B61EBC2
:102720000201001C41F5801300185B412018A2F53E
:10273000001747EB030140EAD570B6196D4111E06F
:102740006D084FEA360645EAC0754FEA0752001B8E
:1027500061EB0201001C41F5801149084FEA30008D
:102760000019514132462B4603B0BDE8F04F00F04E
:1027700057B90098012240000023D0EB020263EB1E
:10278000E073009821464FEAE074B8EB000061EB7B
:102790000401E9E783F000435BE781F0004158E77B
:1027A0002DE9FE4F81EA030404F0004421F00041CA
:1027B00000944FF0000B23F0004350EA010402D0D4
:1027C00052EA030404D10020014603B0BDE8F08FB3
:1027D000C3F30A54C1F30A552C44A4F2F334019410
:1027E000A0FB0254C1F3130141F48011C3F313039E
:1027F00043F4801301FB024400FB034E840A970A52
:1028000044EA815447EA8357A4FB076802958D0A7E
:1028100005FB07854FEA932C04FB0C542705029D0A
:102820004FEA065847EA1637B5EB08056EEB070C7A
:10283000870E920E47EA811742EA8312A7FB020134
:10284000B6EB0B0164EB00042B0D43EA0C335E186E
:1028500044EB1C50DA465146E7FB0201C5F3130472
:102860004FEA0B3343EA14534FEA0432019C43EA24
:102870000603A4F10C040294009CCDE900B400F01E
:10288000DCF8A2E72DE9F04D81EA030404F0004BE7
:1028900021F0004514464FF0000A23F0004150EAB1
:1028A000050220D054EA01021DD0C5F30A570246A2
:1028B000C5F31303C1F31300C1F30A5640F48015A6
:1028C00043F48013A7EB0608101BD64608F2FD3828
:1028D00073EB050002D308F1010801E092185B4197
:1028E000B8F1000F03DA00200146BDE8F08D0020AA
:1028F0004FF48011064684460EE0171B73EB050764
:1029000005D3121B63EB050306434CEA010C49088F
:102910004FEA300092185B4150EA0107EDD152EACC
:10292000030012D082EA040083EA0501084303D1C0
:1029300000224FF0004308E0101BAB4102D20122FD
:10294000002302E06FF0010253101AEB06004CEB7B
:10295000085110EB0A0041EB0B01BDE8F04D00F00F
:102960005FB8C1F30A52C1F3130140F2FF3341F4DF
:1029700080119A4202DA00200146704740F2334348
:102980009A42A2F2334202DC5242FFF7B8BDFFF78F
:10299000A7BD000030B5002904DB4FF000444042E1
:1029A00064EB0101002B04DB4FF00044524264EB66
:1029B0000303994208BF904230BD0000064C074D0A
:1029C00006E0E06840F0010394E8070098471034FF
:1029D000AC42F6D3FFF7B0FB0CC702082CC70208C5
:1029E000202A06DBCB17203A41FA02F043EAE073D3
:1029F00006E041FA02F3D040C2F1200291400843C0
:102A0000194670473A2800D2303820F02002412A77
:102A100001D3A2F13700884201D34FF0FF30704755
:102A200010B5002B08DA401C41F1000192185B41FF
:102A30001A4301D120F0010010BD2DE9F04D92465E
:102A40009B4611B1B1FA81F202E0B0FA80F2203275
:102A50009046FFF745FD04460F4640EA0A0041EA6A
:102A60000B0153465A46084303D120463946BDE878
:102A7000F08D114653EA010015D0C8F140025046CE
:102A8000FFF73DFD05460E46504659464246FFF7C4
:102A900027FD084301D0012000E00020054346EA5D
:102AA000E0762C4337430A984FEA4453A0EB0800E2
:102AB0004FEAD4240A304FF0000244EA47544FEA68
:102AC000D72502D500200146D1E70105101969413B
:102AD000DDE9084500196941BDE8F04DA0E770B592
:102AE00001EB020410F8015B15F0070301D110F8A7
:102AF000013B2A1106D110F8012B03E010F8016BFD
:102B000001F8016B5B1EF9D12B0705D40023521E7F
:102B10000FD401F8013BFAE710F8013B02F1020281
:102B2000A1EB030303E013F8015B01F8015B521E04
:102B3000F9D5A142D6D3002070BDC94301607047CA
:102B40000029816802D041F0010101E021F001017A
:102B500081607047014600208968490700D501203F
:102B60007047C06C80B270470246002012680A426B
:102B700000D001207047014600208968090700D570
:102B80000120704710B542680E4B0C791A400B6853
:102B900042EA04221343436082680B4B1A40D1E996
:102BA000024323434C7942EA440213438360C26ADE
:102BB000097C22F47002491EC9B242EA0151C16285
:102BC00010BD0000FFFEF0FFFDF7F1FF816841F04E
:102BD0000801816070470029816802D041F4A0019A
:102BE00001E021F4A00181607047816841F0040197
:102BF000816070477047704741617047002070479F
:102C00004209231978041712720000002DE9F041DF
:102C10001CF00CF9384C4FF4FA7300226168411A29
:102C2000591A72EB020059D21CF000F96060DFF80B
:102C3000CC80334E002408EB040595F85832D806B2
:102C400048D0304A0021084602EB041232F81070D6
:102C5000401CC0B239440828F8D3C808A0F2F94093
:102C600040F22E61884225D306EB040797F8360020
:102C7000C0062FD404F12100C0B223F0BDF995F8AD
:102C8000580200F01F00072897F8360008D0000708
:102C900020D404F12000C0B2022118F00DFC19E08C
:102CA000010617D440F0800087F83600512019F053
:102CB0003BF80FE003F01F00072806EB04000FD0DD
:102CC00090F83600C00605D504F12000C0B20221FC
:102CD00002F03CF9641CE4B2082CACD3BDE8F081EE
:102CE00090F836100A06F5D521F0800180F83610EC
:102CF000512019F0FDF8EDE708000020E415002050
:102D0000801C00203203002070B5072609290AD94B
:102D1000C568A1F10A0404EB4404A640B543A340EE
:102D20001D43C56007E0056901EB4104A640B543BA
:102D3000A3401D4305611F23072A09D2446B521E7D
:102D400002EB820293409C4391400C43446370BD6C
:102D50000D2A09D2046BD21F02EB820293409C43DE
:102D600091400C43046370BDC46A0D3A02EB8202C9
:102D700093409C4391400C43C46270BD70B52D4D8F
:102D800002212846FFF7F0FE2B4C01280AD02078BC
:102D900001284DD1002020702846BDE87040012157
:102DA000FFF719BF02212846FFF7C7FE2846FFF7A5
:102DB000D8FE0146214890F8902000EB0212903096
:102DC000437822F813100178491CC9B20922B1FBDB
:102DD000F2F302FB131100F8901929B910F8912FA2
:102DE000521C02F00702027001202070082913D241
:102DF0001348C26822F4E052C260C26801F00703BF
:102E000042EA8322C260002912D14FF007034FF03B
:102E100001024FF00A0106E00AD14FF007034FF01C
:102E200001024FF00B012846BDE87040FFF76CBF70
:102E300070BD000000240140080000203203002083
:102E4000001001400548FF21017141718171C1717C
:102E5000017241724FF0FF3101607047FA22002089
:102E60000C4A00681268824209D00B4BD3F808C0A4
:102E700062450CD11A6850405A68104207D0074882
:102E8000D0F80E200A60408A888001207047002018
:102E900070470000FA220020555C0020F02200203C
:102EA00030B587B02E4D2F4C2878002802D001284D
:102EB0004FD13DE01C21684612F002FE12F010FDD9
:102EC000684618F04FFDBDF80000012807D19DF8B5
:102ED0000400062803D19DF80500042802D007B09D
:102EE000012030BDBDF80600022802D001280DD017
:102EF0001EE00298C4F80E00BDF80C006082DDF8F8
:102F00000E00C4F80A0007B0012030BD164906982B
:102F10000968884202D007B0012030BDDDF80E00FC
:102F2000206002986060BDF80C00208101202870AC
:102F30000220ADF806006068CDF812002089ADF8D7
:102F4000160020680690684600F010F820B10020B6
:102F5000287007B0012030BD07B0002030BD000050
:102F600018010020F0220020555C002010B5044616
:102F700012F07CFF0028FBD040F6CF2013F024F99C
:102F800001202080C0026080062020710420607132
:102F90000D48D0F82D10A160B0F83110A181006863
:102FA000C4F80E00204618F0DDFC1C22062104F1B6
:102FB000120013F09DF81C21204613F06BF812F05C
:102FC000B3FC012010BD0000555C002000B587B0A7
:102FD0000121ADF80610FF218DF812108DF81310A5
:102FE0008DF814108DF815108DF816108DF8171037
:102FF000074900680A684B6842401A4202D0886854
:10300000069000E006906846FFF7B0FF07B000BDED
:10301000555C0020094991F8560000280DD0401E4B
:1030200010F0FF0081F8560007D1086840F4806076
:1030300008600D21002013F0F9BA7047801C0020B1
:1030400030B5012185B0480215F062F800244FF434
:103050006020CDE902040120174D8DF804408DF861
:10306000100000948DF8054069462846FFF78AFD58
:103070001249072301220C704C700A212846FFF7E1
:1030800043FE01212846FFF75BFD2846FFF79EFD22
:103090002846FFF770FD0028FAD12846FFF7A5FD66
:1030A0002846FFF757FD0028FAD101212846FFF7EF
:1030B00092FD05B030BD000000240140C203002095
:1030C0002DE9F0471BF0B2FEF84C00252168401AAC
:1030D000401E75F1000007D31BF0A8FE2060606859
:1030E000012801D9401E6060606801287ED16560BA
:1030F000207EEF4F40F30001491C61F30000207671
:10310000388840F22A320A26EA4DDFF8AC83A0F272
:103110002A314FF416794FF4FA7A904267D073DC73
:1031200040F2CD12A0F2CD119042F7D036DC40F241
:103130003712A0F2371190427ED01ADCE7280CD06B
:103140000CDC792829D004DC5A2876D06F2875D178
:10315000E7E0D328F3D0DD2870D14FE1F128FCD08F
:10316000FB286CD0A0F58070053801D00A2865D105
:10317000A8E16429E0D008DC0A29DDD0142971D047
:103180001E290AD0282959D138E16E29D4D07829AE
:10319000D2D08229D0D08C2950D113E1FA2926D05F
:1031A00014DC5A2908D008DC322973D03C2972D0AB
:1031B000462970D0502941D104E1642917D06E29E5
:1031C00015D0782913D0F92938D1FBE040F20F123D
:1031D000A1F20F1091420DD00DDC10F10C0109D0BD
:1031E000012904D00A2902D00B2902E063E20AE097
:1031F0000AE023D1E6E001284DD0022803D00828B8
:1032000076D009287DD1C9E041F22252881A914234
:103210006ED041DC41F20B42A1EB0200914220D082
:1032200021DC1E291DD010DC012978D00229FCD018
:10323000DFF88882192503E059E0D7E261E03FE139
:103240000A296DD014295CD1ACE2A1F580719139C5
:1032500063D0A1F590515C3903D00A291BD0142901
:103260004FD19BE032E1B3287ED008DC0A287BD026
:10327000142810D0A92877D0AA2842D111E1B42867
:1032800073D0BD2870D0A0F580700D3830D00128E3
:1032900037D106E195E0B1E0B0F5C37F16D016DC7A
:1032A000642825D008DC01285FD00A2820D05A28BD
:1032B0001ED05B2825D1E7E0BE2819D0BF2805D055
:1032C000C8287FD0A0F5807023381AD1E9E040F6F5
:1032D000BC62A0F6BC61904209D00ADC11F1520038
:1032E0006FD00A286ED00B2817D0512809D1EBE0F7
:1032F00068E001296FD002296DD0032962D004292A
:103300004CD012F005F93888B0FBF6F106FB11013C
:10331000BDE8F0474C2002F0D5BC042702E0CCE128
:1033200012E2062712F0F4F898F81D00411CCDB205
:10333000BD4200D9054610B9207EC0070AD00B2136
:103340004C2002F0BFFC98F81D00012802D1207E1D
:10335000C0070DD00B21542002F0B4FC98F81D00DA
:10336000022805D1207E01E018E09DE0C0070AD0C8
:103370000B215C2002F0A6FC98F81D00032802D364
:10338000207EC00701D00B21EAE0B5FBF6F10F4625
:103390006C2002F097FC06FB1751D3E112F0B8F84D
:1033A000207EC00704D098F800104C2002F08AFC60
:1033B00000216C2002F086FC0121C3E102F082FCB6
:1033C00077E1D1E012F0A4F898F81D00454618B155
:1033D000012809D048E077E0207EC0070BD029788B
:1033E0004C2002F06FFC06E029784C2002F06AFCC9
:1033F000207EC00738D06978542033E012F088F876
:1034000098F81D100327B1FBF7F007FB1011454694
:1034100011B9217EC90705D000EB4000295C4C2082
:1034200002F050FC697FB1FBF7F007FB1011012996
:1034300002D1217EC90706D000EB40002844417824
:10344000542002F03FFC697FB1FBF7F007FB10113D
:10345000022902D1217EC90706D000EB4000284492
:1034600081785C2002F02EFC687F401CB0FBF6F0F7
:10347000C1B26C2002F026FC687F00F10100B0FBB5
:10348000F6F106FB11015DE1F879400707D512F06E
:103490003FF8207EC00775D00B214C208EE70A270D
:1034A00015E0F8798007F2D1092710E0E41D00202B
:1034B0007000002014870208C0150020888C0208C4
:1034C000052704E0082702E0122700E0042712F095
:1034D0001FF898F81D00411CCDB2BD4200D9054629
:1034E000052D28D205F00707012F02D1207EC00745
:1034F00004D098F800104C2002F0E4FB022F02D117
:10350000207EC00704D098F80110542002F0DAFBA6
:10351000032F02D1207EC00704D098F802105C204F
:1035200002F0D0FB042F03D1207EC0073FF42DAF63
:1035300098F8031014E008EB05074C2017F8041D59
:1035400002F0C0FB7978542002F0BCFBB9783F1D33
:103550005C2002F0B7FB207EC007E7D017F8011C03
:10356000642002F0AFFB10E711F0D2FF98F81D00C5
:10357000464610B9207EC00705D03078285C40F060
:10358000100101E095E0102118201DF0D5F9707FA1
:10359000012802D1207EC00704D07078285C40F05A
:1035A000100100E0102120201DF0C6F9707F0228D4
:1035B00002D003280ED10AE0207EC00704D0F078A4
:1035C000285C40F010010DE0F078295C0AE0207ED4
:1035D000C00703D0B0780128F6D1F0E7B078012811
:1035E00009D1102100201DF0A7F9707F042802D115
:1035F000207EC00704D03079285C40F0100100E044
:10360000102108201DF098F9707F052802D1207E36
:10361000C00704D07079285C40F0100100E0102150
:1036200010201DF089F9707F062802D1207EC00786
:103630000AD0B079295C4C201DF07EF9707F0728F4
:1036400002D1207EC0070AD0F079295C54201DF0F9
:1036500073F9707F082802D1207EC00704D0307A29
:10366000285C40F0100100E010215C201DF064F99E
:10367000707F092802D1207EC0070AD0707A295CA9
:1036800064201DF059F9707F0A2802D1207EC007FE
:103690000AD0B07A295C6C201DF04EF9707F0B289F
:1036A00002D1207EC00704D0F07A295C74201DF07E
:1036B00043F9C4F80490BDE8F08711F029FF98F8A9
:1036C0001D00C246411CCFB2042F00D9074607F0A7
:1036D0000708B8F1010F02D1207EC00704D09AF884
:1036E00000104C2002F0EEFAB8F1020F02D1207E59
:1036F000C00704D09AF80110542002F0E3FAB8F1A0
:10370000030F02D1207EC00705D09AF80200285C82
:1037100040F0100100E010215C201DF00DF9B8F11F
:10372000040F02D1207EC00704D09AF80310642051
:1037300002F0C8FAB7FBF6F10D466C2002F0C2FAAF
:1037400006FB1571742039E6B87958B101282DD8D7
:1037500019D14FF0000148481CF004F9012002F093
:10376000FDFF2CE005F020F968B94448BD710088E0
:1037700010F4C04F04D14248017841F001010170BA
:10378000012140482FE0B8794008B0FBF6F14C2009
:1037900002F098FAB8794008B0FBF6F106FB110187
:1037A000542058E0B87990B1012803D9A0F1010064
:1037B000B871E8E703D005F0F7F80028E3D1B8784E
:1037C00000EB800108EB8100C0883880DBE705F062
:1037D000EBF80028D7D1BD7102F0E0FF042002F021
:1037E000DDFF002128481CF0BDF8CCE711F090FE69
:1037F00098F81D00454610B9207EC00709D02978E9
:103800004C2002F05FFA687F012802D1207EC007B9
:1038100003D06978542002F055FA0B215C2002F0A5
:1038200051FA7879E0B1207EC00704D0687F295C26
:10383000642002F047FA687F401E90FBF6F0C1B2A8
:103840006C2002F03FFA687F401E90FBF6F106FB09
:103850001100C1B2742002F035FAC4F804A02AE7BE
:1038600000216C2002F02EFA0021742002F02AFAC6
:10387000A9786420EFE7000040810208801C002046
:103880006E000020E2870208E6870208174B10B599
:103890009878174900EB80001A8831F8200082429E
:1038A00023D0002000EB800431F82440A24218D13C
:1038B000987000EB800001EB80000E4C01692162E2
:1038C000C06801211CF04EF80B4801214160017EC7
:1038D00041F00101017600206077BDE8104000F062
:1038E0000DB8401CC0B2C828DCD310BD7000002049
:1038F000888C0208C0150020E41D00202DE9FC5F23
:10390000DFF8049440F2DD2C4B46B9F80000DF7874
:1039100093F804A0791CFE4BFC4C0A25A0F2DD2292
:103920004FF0640B01F0FF0E03EB8706604575D086
:1039300075DC40F2B912A0F2B911904270D073DC7C
:10394000FB286FD027DC6F286DD00FDC502804D007
:1039500004DC0C28FBD046284CD1C1E15A2871D098
:10396000632847D1BDE8FC5F02F078BDDD286AD04E
:1039700006DC792868D0D3283CD1D3F8461005E07E
:10398000E72874D0F12835D1D3F87110BDE8FC5F79
:10399000DE480FF08BBF40F25512A0F25511904255
:1039A00076D032DC40F23712A0F23711904270D05C
:1039B00022DC11F132006DD00A281BD193F9B1003D
:1039C000002868D030382070B233187830386070F2
:1039D00058783038A07098783038E070D87830381F
:1039E000207118793038607158793038A071987921
:1039F0003038E071BDE8FC9F0A297DD01429F9D147
:103A0000C348D0F8E1002060F4E70A2975D04629C0
:103A100074D0502973D05A29ECD1BAE14DE256E066
:103A2000BEE101E080E153E1A92930D020DC642926
:103A300066D011DC462979D007DC0A2977D0142911
:103A4000D8D13FE16BE269E16FE0502970D05A298B
:103A5000D0D193F8330132E26E296AD0782969D047
:103A6000822968D08C29C5D193F8380155E258E1F4
:103A700040F21713A74AA1F21710994255D015DC4E
:103A8000C72904D008DCB32901D0BD29B2D127E170
:103A9000A4E173E16BE19CE1A1F580710D3944D0A3
:103AA0000129A7D1B85C00F01F0036E201286ED0D2
:103AB0000A287ED00B286CD00C289BD196F85D028A
:103AC000B0FBF5F105FB11002170607092E7DFF8A3
:103AD000388241F2655CA2EB0C0098F80710019166
:103AE00021F00301491C009198F80310DFF82082AF
:103AF00001EB4101414404E043E172E1D6E002E11F
:103B000078E1624511D060DC41F23A4CA2EB0C0046
:103B1000624571D02EDC4F2A6FD01CDC082A6DD094
:103B20000ADC012A6BD0072AD0D1E0E084E038E13A
:103B30005DE162E164E166E14D2A3AD04E2AC5D1E9
:103B400096F87C02B0FBF5F105FB11002170607066
:103B500096F87D02D1E16B2A7ED004DC572A7CD016
:103B6000612AB3D1D3E1A2F58072033A76D0DB2A81
:103B7000ACD1B2E0C7281CD013DC1E286FD009DC02
:103B80000A286DD01428A1D193F83B01C5E18DE13D
:103B90000FE08FE128287DD0322897D193F83E019D
:103BA0008DE1C82877D0D12803D0D22874D0DB2863
:103BB0008CD14946704689F803E05246D64502D971
:103BC000104681F803A0C0B2A7E140F22D1CA0F27C
:103BD0002D12604579D01CDC652877D010DC0B28CD
:103BE00075D004DC012856D00A289DD17FE0142826
:103BF0007DD0642898D17AE008E174E170E16CE14D
:103C00006E2874D0C82872D0C92844D0D2288BD14D
:103C10006DE040F65D51A2F65D508A4273D049DCFA
:103C200040F65151A2F651508A4260D03ADC632AE4
:103C300031D010F10A0294D137480178B1FBF5F286
:103C400005FB1211227061704178B1FBF5F205FBA2
:103C50001211A270E17004E05DE155E140E0DBE0AB
:103C6000D7E08178B1FBF5F205FB12112271617189
:103C7000C178B1FBF5F205FB1211A271E171017976
:103C8000B1FBF5F205FB1211227261724079B0FBB3
:103C9000F5F102E0C3E0C5E0C8E005FB1100A17248
:103CA000E072A7E6012818D00B28FAD11849122291
:103CB000E83171E001286CD0022873D03F2870D021
:103CC0004028EED193F8310127E1DBE0D4E0BBE0FE
:103CD000186820609888A0808CE6D6F8020092E6EA
:103CE000002189F80310FF2189F8041082E6494673
:103CF000704689F803E05246D64502D9104681F84D
:103D000003A0C0B2DCE640E070000020C015002037
:103D1000E41500201B18002068000020D3F84E1086
:103D200034E6D3F84A1031E6B3F8A60042F2107236
:103D3000B0FBF2F102FB110221704FF47A71B2FB79
:103D4000F1F26270B0FBF1F201FB12025946B2FBD4
:103D5000F1F2A270B0FBFBF20BFB1201B1FBF5F12B
:103D6000E170B0FBF5F105FB1100207142E693F91B
:103D7000A80070B330382070A93326E612226B49B0
:103D800013E06A49122212310FE0684912223D31D4
:103D90000BE0664912224F316548FEF767FA07E0EB
:103DA00000E021E06149122261316148FEF75EFACC
:103DB000002002460E23012A0CD0215C50290BD092
:103DC000092901D925540122401CC0B21228F2D37E
:103DD00010E64BE02554F7E72354F5E793F8E500A8
:103DE0006EE6B3F8E6006AE093F8300168E693F80F
:103DF000320164E093F8340162E693F835015FE63E
:103E000093F8360189E093F8370186E093F8390199
:103E100083E093F83A0152E093F83C017DE093F897
:103E20003D017AE0009889F80700E3E57F1E03EB87
:103E3000E70007F0070390F8402101209840024274
:103E400014D001F245110CE0FF1D03EBD70007F081
:103E5000070390F8402101209840024206D001F269
:103E60005D11BDE8FC5F32481CF074BCBDE8FC5F2E
:103E700009212F48FEF713BA019941F0040189F88E
:103E80000710B7E593F847010B2220F0010083F8F3
:103E9000470109212648FEF7FBF9009989F8071028
:103EA000BDE8FC5F2349E1201BF0B2BEB85CC0F363
:103EB000411032E096F85C0202E696F85E02B0FB32
:103EC000FBF121700BFB1101B1FBF5F16170B0FB4F
:103ED000F5F105FB1100A0708CE596F85F021CE07F
:103EE0001548385C19E096F87E02B0FBF5F105FB49
:103EF00011002170607096F87F02B0FBF5F105FBB0
:103F00001100A170E07075E5012002F047FC00206F
:103F100089F806006EE593F8D20220706AE5002069
:103F200089F8050025706570A57063E5A11600206D
:103F3000C01500209D650108B618002070B5114C11
:103F400005462168480701D4480608D521F04000FD
:103F500020600C4900202071486481F8480000204E
:103F600000F084FB284600F053FF208810F4C04F77
:103F700006D10549087840F0040040F004000870BC
:103F800070BD0000801C00206E0000202DE9F0476D
:103F900007465348DFF85091DFF85081C278514806
:103FA000BCB000EB4105012AA9782BD0002002907B
:103FB000069003900490059007904AF65520ADF8BE
:103FC000080049F21000ADF80E001020ADF80A000C
:103FD0008DF81A10E97809EB8100C3788278CDE971
:103FE0000023437819F8212041A10DF1120022F09D
:103FF000A9FAFF208DF81B00002318F837001822BB
:1040000002A967E0DFF8F8A03C4C9AF815030028F5
:1040100014BF3C4E3C4E481EC0B237A922F0F1F905
:104020002EA937A802F03EFFE8780EA906EB800023
:1040300050F8040C02F036FF0AF15A00FEF76EF950
:1040400006460EA8FEF76AF90146A8782EABCDE920
:104050000A032E4A2E48CDE90C6282780DF1180E23
:1040600090F805C00679C378AEE84C104278007825
:104070000EABCDE90213CDE90402E97809EB81002A
:10408000C3788278CDE90023437819F821202149AB
:1040900004F1100022F056FA0546014604F1100022
:1040A0001CF032FF1CA0211D00682060284612F081
:1040B000FBFA4FF03031A1606019E1601030C4F8B4
:1040C0003002462122F064FA18F83700002305F187
:1040D0001402214623F036FC3CB0BDE8F087000016
:1040E00010020020DC1C0020289C0208F05E00204A
:1040F000256425642564256400000000D85C002048
:10410000E4150020D8AA020838AA02083E160020AA
:1041100068000020B0AC020840616C410000000063
:104120002DE9F14F7948ADF58A6DDFF8E891067811
:1041300081208DF80C0000208DF8240074484C4636
:104140000DF10E01807800EBC00009EB4000E83073
:1041500013F0A4FE704894F8152309A900F1080B88
:1041600000F1180ACDF84C148AB143686B48C17845
:1041700002798DE80E008378427869A1DDF84C045D
:1041800022F0E0F900208DF80D00A0258BE00268F8
:1041900068A1DDF84C0422F0D5F908208DF80D0057
:1041A000462580E0701C00F01F08584800EB4804CA
:1041B000E078292876D2DFE800F075151515151579
:1041C0001515158383838383838315151583838353
:1041D00015838315831515838383151515151515FB
:1041E00015151500A078411E272905D8C8B20DF273
:1041F0000C4122F006F905E010B3292829D000204F
:104200008DF80C0499F815030028DDF84C042DD026
:10421000FEF784F807460DF20C40FEF77FF8E178D0
:1042200007440AEBC1004068FEF778F83844A8421A
:104230003ED20DF20C41DDF84C04FEF73BF851E0A4
:1042400099F8150310B1DBF8041007E0DBF8001053
:1042500004E099F8150330B1DBF80C100DF20C40B6
:10426000FEF77EF8CEE7DBF80810F7E7FEF756F822
:1042700007460DF20C40FEF751F8E17807445AF872
:104280003100FEF74BF83844A84211D20DF20C4130
:10429000DDF84C04FEF70EF834E003E0DDF84C04E2
:1042A000FEF708F84646DDF8500486427FF47AAF00
:1042B00003A805F02BFD0DF2544D3046BDE8F08FFC
:1042C00099F815030028DDF84C0410D0FEF726F805
:1042D000E17807460AEBC1004068FEF71FF8384452
:1042E000A842E5D2E1780AEBC1004168D6E7FEF7C3
:1042F00015F8E17807465AF83100FEF70FF8384410
:10430000A842D5D2E1785AF83110C7E7A21D0020A3
:1043100048000020E4150020C8830208680000203F
:10432000253032642D2530326420253032643A2520
:10433000303264202573000010B5437804785B1C8C
:1043400003F01F039C4203D1641C04F01F0404709B
:1043500000EB4304A170E2704370012010BD000027
:1043600070B51D4D05F11406E879401CE8713079EF
:10437000A979884202D0A8710021E971174909780A
:10438000C943890726D0EA79042A23D2F17809B9EA
:1043900000281FD0124C04EB820292F880328B422C
:1043A00006D192F88112814202D1502017F0BCFC54
:1043B000E879F27804EB800090F88212914209D1FA
:1043C00090F883023179884204D1BDE870405020D2
:1043D00017F08EBD70BD000054000020801C00202E
:1043E000E415002070B50D46064A0824146040F01C
:1043F000A00016F05BFB284616F058FB024804604C
:1044000070BD0000140801401008014070B50D4651
:10441000064A0824146040F0800016F047FB284646
:1044200016F044FB0248046070BD0000140801400F
:104430001008014030B5154890F81703C0F10B0083
:10444000C0B2062801D0072800D1052010494A79BA
:10445000104D02241AB90A8812F4C04F04D04879CA
:10446000002800D02C6030BD0B4B1A7852B1194691
:104470000978491EC9B2824202D10648001D046073
:10448000197030BD2C60187030BD0000E41500209C
:10449000801C002010080140B400002001B5032159
:1044A0001F20FFF79FFF9DF80110BDE808401F2067
:1044B000FFF7ACBF70B405464FF0000C00204C1E57
:1044C000A4B2002935D015F8011BA1F14106192E1F
:1044D00001D8F1B219E0A1F16106192E02D84739CD
:1044E000C9B212E0A1F13006092E02D8091DC9B2E5
:1044F0000BE02B2906D02D2904D02F2904D05F29C9
:1045000002D011E03E2100E03F21BCF1000F12D0AB
:10451000BCF1010F18D0BCF1020F23D04FF0000CFA
:104520001678314302F8011B2100A4F10104A4B262
:10453000C9D170BC70474FF0010C9842F9D2401CB1
:1045400080B289001170EFE74FF0020C167846EA4E
:10455000111602F8016B9842EBD2401C80B209019F
:104560001170E1E74FF0030C167846EA910602F865
:10457000016B9842DDD2401C80B289011170D3E7F3
:10458000F8B40025042B68D3FF276E468DF8007021
:104590008DF801708DF802708DF8037000295CD0E1
:1045A00010F801CB491E89B24FEA9C048DF80040F7
:1045B0004FEA8C7C4FEA9C648DF80140D1B110F831
:1045C00001CB491E89B244EA1C148DF801404FEA20
:1045D0000C7C4FEA9C648DF8024059B110F801CB75
:1045E000491E89B244EA9C148DF802400CF03F0C3D
:1045F0008DF803C0002416F804C0BCF1190F04D8CC
:104600000CF1410C0CF0FF0C17E0BCF1330F04D897
:104610000CF1470C0CF0FF0C0FE0BCF13D0F04D87F
:10462000ACF1040C0CF0FF0C07E0BCF13E0F17D00E
:10463000BCF13F0F17D04FF03D0C02F801CB04F155
:10464000010C0CF0FF04042CD5D31B1F9BB205F109
:10465000040C1FFA8CF5042B98D22846F8BC70473E
:104660004FF02B0CE9E74FF02F0CE6E72DE9F05F58
:10467000724EDFF8D0C1744D96F83411DFF8C09156
:10468000C1EB01114FEA810BDCF800206A4F296869
:104690004FF0080E4FF4004409F1040A42F4802858
:1046A00007287DD2DFE800F0042E62C67D9AA000C4
:1046B00022F48020654ACCF80000C2F800E010F433
:1046C000F01F02D1002002F049F8286820F40060B1
:1046D0006FF30A00286000215D481AF01EF8387850
:1046E00020F00800387096F8D202012806D153480D
:1046F00090F87106AA2875D050460460BDE8F05FB6
:104700001BF056BA6BF30A012960480548D012F431
:10471000F01F03D14D49091FC1F800E00020CCF87B
:10472000008002F03BF82868010504D420F4F03042
:1047300000F500502860444940F6AC500C394880E0
:104740000121434819F0E9FF96F8D202012806D169
:104750003A4890F87106AA2806D04846046038788E
:1047600040F0080038705FE05046F7E76BF30A014D
:10477000296048055ED012F4F01F03D13349091FA8
:10478000C1F800E00020CCF8008002F007F82868AB
:1047900020F4F03040F4006000F5A0302860DEE73F
:1047A00048E042F40020CCF8000041F4C02028602A
:1047B0000021274819F0B1FF96F8D202012806D14E
:1047C0001E4890F87106AA2805D050460460BDE83E
:1047D000F05F1BF00DBA4846F8E703E0084661F3C6
:1047E000DD4075E7484688E71A48014222D0C1F308
:1047F000CA4060F30A012960134940F6AC500C39F5
:1048000048800121124819F088FF387840F00800EC
:10481000387096F8D202012806D1084890F871063F
:10482000AA2805D048460460BDE8F05F1BF0D0B967
:104830005046F8E7BDE8F09F6E000020E415002028
:1048400010080140801C0020B0000020140C014022
:10485000002C01400000F83F00200022DFF818C0C3
:10486000FF2300EB40010CEBC1010A714B75401CAA
:104870000828F6D3704700000423002070B51AF012
:10488000D5FA3D4C32220023A168401A101A73EB6E
:1048900003014DD21AF0CAFA384BA060384A587852
:1048A0004FF04004010705D0A0F1010161F30300BE
:1048B00058702DE019784D090BD0072505EB5115DF
:1048C00065F3471119704FEA101161F30300587036
:1048D0000DE0CD0610D520F00F0000F10A0020F009
:1048E000F00000F1A000587021F0E0001870D068CE
:1048F00080F04000D0600BE0080708D51E480C305F
:104900000088C0F30A00012801D9146100E0546155
:104910001878C1070DD020F001001870587820F0E9
:104920000F0000F101005870D06880F04000D060A6
:1049300070BD81070ED5597820F0020021F00F01DB
:1049400001F1040121F0F00101F11001597040F072
:10495000E0000EE04107EBD520F00401587820F08C
:104960000F00001D20F0F0001030587021F0E00022
:1049700060301870546170BDA40000206E000020EB
:1049800000100140F0B5404D0020404E2978404CC9
:10499000491C01F01F0302460146B71804EB010C45
:1049A000521C491C97F8E170D2B28CF82F70C9B232
:1049B000042AF2D36218491CC9B20126671882F88A
:1049C0002F60082287F82F2005EB4303491C314F45
:1049D000DD78C9B2002207EB850504EB010CAF5C62
:1049E000491C521CD2B28CF82F70C9B2042AF4D3DD
:1049F00062180025491C82F82F50C9B26218491C60
:104A000082F82F609A786426B2FBF6F3C9B2671871
:104A100006FB132687F82F300A23491CB6FBF3F652
:104A2000C9B26718491C87F82F60B2FBF3F603FB85
:104A30001622C9B26318491C83F82F20CBB200217B
:104A400007E0621892F82F2092B11044491CC0B2BE
:104A5000C9B29942F5D30F21B0FBF1F201FB12006C
:104A6000C0F10F00E1180A2881F82F0002D003E0FE
:104A70000A30EBE781F82F5012205B1CD9B2214499
:104A800081F82F00F0BD0000DC1C0020E4150020A0
:104A900038150020289C020830B40F4B0F4C002022
:104AA0001A1892F82F10122910D0401C615CC0B265
:104AB00082F82F101828F3D30948074B09A190F862
:104AC000192330BC2F330E4821F03CBD184400217F
:104AD00080F82F10F0E70000381500204881020808
:104AE000E415002041542B515744544D463D256454
:104AF0002C302C2225732C38302C3530220D000020
:104B00006005002070B5044600200246064D07E00F
:104B1000A65CC3B27340521C35F8133083EA1020F0
:104B20008A42F5DB70BD0000CC9C020810B5002263
:104B3000044B03E050F822401C60521C8A42F9D317
:104B4000186810BD0030024001490120886070479C
:104B5000003002402DE9F04389B004460026079654
:104B6000002013F06BFF00909DF800808DF82080EE
:104B7000012013F063FF00909DF800908DF82190C4
:104B800034B301AF142C01D9142500E02546069555
:104B9000294601A810F094FF601B84B29DF818000C
:104BA00010F0010F02D07E55681C069001A9BDF8D7
:104BB000180058B131F8020B079A10440790BDF85D
:104BC0001800801E82B20692002AF3D1002CD9D19F
:104BD000414600201BF066FE494601201BF062FEA4
:104BE000BDF81C00BDF81E1008440790BDF81C005D
:104BF000BDF81E100844C04309B080B2BDE8F08380
:104C000081B04B08002200925A1E92B2002B0AD0AB
:104C100030F8023BDDF800C0634400931300A2F1BA
:104C2000010292B2F4D111F0010F03D00078009983
:104C300008440090BDF80000BDF802100844009040
:104C4000BDF80000BDF802100844C04380B201B0B6
:104C50007047000070B51AF0E9F81F4D4FF47A72F2
:104C600000242968401A101A74EB040133D21AF098
:104C7000DDF81A494FF47A7200238969401A2146F7
:104C8000FDF772FA84B21AF0D1F82860287E40F35A
:104C90004001491C61F34100287610F039FC64267C
:104CA000B4FBF6F5E9B24C2001F00CF806FB154018
:104CB0000A25B0FBF5F1542001F004F8B4FBF5F03F
:104CC00005FB10415C2000F0FDFF102140201BF08F
:104CD00033FE0348457170BDE41D0020C01500205F
:104CE000801C002070B4184C237F0F2B04D00B2B9A
:104CF00002D070BC0FF0EEB8144D0020E87008E050
:104D0000EB78265C03EB830306EB4303401CEB705C
:104D1000C0B29042F4D3E878884208D8A8780C4A08
:104D200000EB800002EB8000C088288009E0094881
:104D3000008810F4C04F04D10748027842F0020204
:104D40000270297170BC7047C015002070000020EF
:104D5000888C0208801C00206E00002010B516F020
:104D60007FFF2A48284C0078A4F5257200EB40010B
:104D700001EBC00102EB8100638AA0F8273052F8F2
:104D80002110C160016142684261826190F8252072
:104D900012F0080F01D0042300E00D2380F8243026
:104DA00022F0070222F0100222F0200222F040023C
:104DB00022F0800280F8252090F8262022F00102BF
:104DC00022F0020222F0040222F0080242F0100255
:104DD00080F8262094F8260020F0010020F0020040
:104DE00020F0080020F0100084F82600E16010F0A8
:104DF000F3FBA08010F0F0FBE0804FF0FF30A084C8
:104E00000120A08210BD000078540020A2010020E3
:104E1000104A10B511684B0708D521F0040141F084
:104E2000080111600F2111F001FC0FE008070DD5FA
:104E300000201118401C8B7DC0B223F003038B753A
:104E40002928F6D3106820F0180010600248417835
:104E5000017010BD801C00201E1D00202DE9F041B6
:104E6000144E154F002406EB0405A87D010715D547
:104E700020F00800A875601CC0B2192111F0D6FB03
:104E8000A87DC10603D4810601D4400606D57878F2
:104E9000401C7870306840F480703060641CE4B26C
:104EA000292CE0D3306820F4007030600020387086
:104EB000BDE8F081801C002099000020094B0020F3
:104EC0001918401C8A7DC0B222F070028A75292808
:104ED000F6D31868044920F48070186000204870E8
:104EE00070470000801C002099000020154B10B571
:104EF0001844154A817D0C0707D521F008018175FA
:104F0000117811B1A1F101011170817D4C0603D41A
:104F1000CC0601D48C0606D521F07001817550783D
:104F200018B1401E5070507818B9186820F480707D
:104F300018601078002803D1186820F400701860F9
:104F400010BD0000801C002099000020FEB5494DD6
:104F5000494E421C6F78341807297CD2DFE801F0F3
:104F60007B041D4655607700A07D010773D520F0B6
:104F70000800A075297811B1A1F101012970C106BD
:104F800003D4810601D4400665D507F101076F708F
:104F9000306840F4807030605DE0A17DCB065AD56A
:104FA00021F01001A175890710D034A1D1E9003793
:104FB00089680093CDE901713349084490F83802BB
:104FC00000F01F001DF80010D0B201E0D0B21C218B
:104FD00011F02CFBA07D81063DD44FEA40602FE00C
:104FE000687880B3A0F10100687034E0A07D81068C
:104FF00031D520F02000A075C1062CD440062AD45B
:105000000FB3A7F101076F7025E0A07D410722D5FE
:1050100020F00400A075D0B2272111F007FB1AE0A0
:10502000A17D4B0617D521F04001A17528280BD092
:10503000D0B2282111F0FAFAA07DC1060BD4800667
:105040000028CDDA07E008E01E212920F2E7A07D44
:1050500020F08000A075687818B9306820F480705E
:1050600030602878002803D1306820F40070306068
:10507000FEBD000099000020801C0020002021229D
:105080002324252608000000E41500200E49B1F86D
:105090004A00002817D0401E0004000CA1F84A0066
:1050A00011D1A1F29C60B0F8E60000280BD0C0EB53
:1050B00000104FF6FF7202EA8000A1F84A001521A5
:1050C000002011F0B3BA7047801C00202DE9F04396
:1050D00089B00121402012F0F7FFFFF735FDE948C4
:1050E000032100680590E748001D00680690E54828
:1050F00008300068079005A8FFF718FD81460021D9
:10510000402012F0E1FFE04EE0A0FF220168316094
:105110008088B0804021B01DFDF7BAF8DDA00024E2
:10512000006846F8060FDD48C6F8669086F86440C9
:1051300086F8654030646FF07F407064D848B06492
:10514000D848F0644FF008303065CF48D6A15A30C7
:10515000FDF706F9D7A1D948FDF702F9D748D8A13C
:105160001030FDF7FDF8D548D7A12038FDF7F8F845
:10517000D248D7A11038FDF7F3F8022586F86A5017
:10518000C6F86B4041F62670BF49A6F8A00001F1B1
:10519000B10081F8A840047086F86F40012786F8B6
:1051A000B570B42186F8B41086F8B670122186F86E
:1051B000B71086F8C91004634FF0050886F8DF8041
:1051C000A6F8E04086F8E21086F8F41086F806119A
:1051D00086F8181186F82A8186F82B5186F83751FF
:1051E00086F8317186F830510A2186F838111E226E
:1051F00086F8342186F8355186F83671032286F810
:10520000322186F8335186F82C11404686F82D114C
:1052100086F82E019C4886F82F41B61FC0F8404101
:10522000C0F84441A0F8F64100203118401C91F824
:105230003822C0B222F06002203222F0800281F8CF
:1052400038222828F1D306F50E76307820F01F009A
:10525000401C3070707820F01F00801C7070B07897
:1052600020F01F00801CB070F07820F01F00C01CE0
:10527000F070A6F50E7604203118401C91F8382203
:10528000C0B222F01F02921C81F838222028F3D3EA
:1052900020203118401C91F83822C0B222F01F02A1
:1052A00081F838222828F4D3002006EB800101F58C
:1052B0001871401C0C704C708C70C0B2CD700828F6
:1052C000F3D37E4884A1BB38046044608460C4602A
:1052D0001130FDF745F80E2086F8D102774886F8A0
:1052E000907286F8D27210216838FCF7D8FF7348A4
:1052F0004FF4A0712030FCF7D2FF6349624A01F5F8
:10530000906081F89C441921A2F8CC1480F84E409A
:1053100080F87E40104680F8164580F8464580F8B3
:10532000C64580F8F64580F8264600200721321849
:10533000401CC0B282F8E3120828F8D30820414686
:105340003218401CC0B282F8E3120F28F8D30F20A5
:1053500009223318401CC0B283F8E3221628F8D380
:10536000162008223318401CC0B283F8E3221A2802
:10537000F8D31A203218401CC0B282F8E342282821
:10538000F8D306F201360420317037757476B5759E
:10539000777530763C20F075A6F2013622F006FCD7
:1053A0003949A1F856065020A1F858064E48C1F8D0
:1053B0005A0644F27260A1F85E064CA14E48FCF712
:1053C000CFFF3148552180F8711600203218401C5B
:1053D000C0B282F872462828F8D32B4880F89A1673
:1053E0002949632081F89B0615F0B8FB002015F0D1
:1053F00083FB40F29C61244815F074FC4A463FA1AF
:10540000684621F09FF84FF4D83015F075FB6846D8
:10541000FCF784FF401C81B2684615F063FC0EF077
:105420009DFA4FF4A04015F06DFB3648016821F05D
:105430000301016016F068FC3348048044804FF497
:10544000005015F05FFB04222F49022001F09AFC66
:105450002E490122087820F0020040F00100087077
:10546000002001F08FFC0EF079FA13F05FF820F0C5
:10547000AFFF0EF073FA4FF4004015F043FB09B094
:10548000BDE8F083E8F7FF1FE415002000010203E8
:10549000040500000102030400000000C0A801513F
:1054A000C0A80101CA60805654435049505F504122
:1054B0004E454C0061646D696E0000001F190020AC
:1054C00030313233343500007573657200000000EE
:1054D000313233340000000074696D652E6E6973DB
:1054E000742E676F760000002F5B4A6631323334CA
:1054F0003536373800000000441C0020303125309C
:1055000038580000801C00209E00002078000020F9
:105510002DE9F0410122284E0546002406EB8400C7
:1055200090F8631201293FD190F86012A94203D08C
:1055300090F86112A94237D1204F002207EB840175
:105540008B78D3B14878A8422BD117F824000021DA
:10555000401EC0B215F0B0FF354495F8370200F098
:105560001F0117F8240011F061F895F83702C0F315
:105570004110FFF77BF801221AE006EB840393F851
:105580006132AB4204D107F8243090F8603203E076
:1055900090F8605207F824504B7090F862028870BF
:1055A00006E006EB8400F8E7641CE4B2082CB5D3EF
:1055B0001046BDE8F0810000E41500203E1E0020EA
:1055C0000549087810F0010F01D00020704740F025
:1055D00001000870012070472501002038B5C02463
:1055E00009E09DF8001034EA01000AD000290BD030
:1055F000002019F0CBFD684619F0B0FD002803D05B
:10560000EFE7684619F0AAFD38BD000010B5094C57
:105610002078FF2803D019F015FDFF202070072007
:10562000A0700549087820F001000870C0F3400020
:1056300010BD000024010020250100202DE9F04FBD
:1056400089B00746FE4C00262146A078FD4DDFF8C4
:10565000F8B30A784FF0FF0A04F1060904F10108D3
:10566000082880F07582DFE800F0040614202C8EF4
:10567000FDFCE67026710BF10C00FDF7A7FCE0784D
:10568000401CE07019F0D2FBA0600220A07000F076
:105690005FBA291D0BF10C00FDF7E2FB002846D094
:1056A000DBF80C0028600320A070352300220421C1
:1056B000E44819F0DBFD2070FF2800F04982042047
:1056C000A070207819F0BAFD002800F04182B9F8E6
:1056D0000000401CA9F8000099F8010019F086FEAE
:1056E00099F8000019F082FE012019F07FFE0020D9
:1056F00019F07CFE002019F079FE012019F076FEE9
:10570000002019F073FE002019F070FE002019F03F
:105710006DFE002019F06AFE002019F067FE0020DF
:1057200019F064FEE068B0B100F018FA16E019F064
:105730007DFBA1680022411AD1F57A7072EB060058
:1057400080F00682E078032801D3062000E00120E3
:10575000A07000F0FDB9206900F000FA002019F0F7
:1057600045FE607919F042FE002019F03FFE01204D
:1057700019F03CFE19F08AFC19F058FBA0600520D6
:10578000A07000F0E5B9104619F02EFD90B10DF1B2
:10579000100B0DF1110019F0E1FC04A819F0DEFC6A
:1057A000BDF81000B9F80010884212D019F05AFC68
:1057B00000F0CEB919F03AFBA1680022401AD0F5EA
:1057C0007A7072EB060080F0C3810620A07000F0B2
:1057D000BFB90BF1030019F0C1FC0BF1020019F085
:1057E000BDFC0BF1050019F0B9FC0BF1040019F038
:1057F000B5FC0BF1070019F0B1FC0BF1060019F034
:10580000ADFC0BF1090019F0A9FC0BF1080019F02F
:10581000A5FC0BF10B0019F0A1FC0BF10A0019F02B
:105820009DFCBDF81400411EADF81410C0B10DF17F
:105830001C09FFF7D3FE09F1010019F08FFC07A83E
:1058400019F08CFC09F1010019F088FC07A819F087
:1058500085FCBDF81400411EADF814100028E8D1F5
:1058600001E035E154E1BDF816000DF10409411ED7
:10587000ADF81610F0B3FFF7B1FE09F1010019F011
:105880006DFC01A819F06AFC09F1030019F066FC2F
:1058900009F1020019F062FC09F1070019F05EFC41
:1058A00009F1060019F05AFC09F1050019F056FC3F
:1058B00009F1040019F052FC09F1090019F04EFC3D
:1058C00009F1080019F04AFCBDF80400012807D1CD
:1058D000BDF80600012803D1BDF80C0004284CD007
:1058E000BDF80C00411EADF80C1058B108A819F015
:1058F00035FC00E00DE0BDF80C00411EADF80C10C9
:105900000028F3D1BDF81600411EADF8161000288E
:10591000B1D1BDF81800411EADF81810F0B3FFF773
:105920005DFE09F1010019F019FC01A819F016FC3F
:1059300009F1030019F012FC09F1020019F00EFC44
:1059400009F1070019F00AFC09F1060019F006FC3C
:1059500009F1050019F002FC09F1040019F0FEFB41
:1059600009F1090019F0FAFB09F1080019F0F6FB3A
:10597000BDF80400012815D01CE098F8000040F0A4
:10598000020088F800002F4819F0E8FB681C19F0A5
:10599000E5FBA81C19F0E2FBE81C00E021E019F08F
:1059A000DDFB8CE0BDF80600012803D1BDF80C003A
:1059B000042852D0BDF80C00411EADF80C1048B1BF
:1059C00008A819F0CBFBBDF80C00411EADF80C1077
:1059D0000028F5D1BDF81800411EADF818100028B8
:1059E0009DD1BDF81A00411EADF81A1038B3FFF76B
:1059F000F5FD09F1010019F0B1FB01A819F0AEFBAA
:105A000009F1030019F0AAFB09F1020019F0A6FB45
:105A100009F1070019F0A2FB09F1060019F09EFB3D
:105A200009F1050019F09AFB09F1040019F096FB41
:105A300009F1090019F092FB09F1080006E03EE0C7
:105A400024010020C4230020555C002019F086FBAF
:105A5000BDF80400012813D01AE098F8000040F0C7
:105A6000020088F800003C4819F078FB681C19F027
:105A700075FBA81C19F072FBE81C19F06FFB1EE007
:105A8000BDF80600012803D1BDF80C00042825D07C
:105A9000BDF80C00411EADF80C1048B108A819F073
:105AA0005DFBBDF80C00411EADF80C100028F5D1CF
:105AB000BDF81A00411EADF81A10002897D119F050
:105AC000D1FA207819F0BEFA84F800A00720A0705F
:105AD00098F8000010F0020F13D013E098F80000BF
:105AE00040F0020088F800001B4819F037FB681CE2
:105AF00019F034FBA81C19F031FBE81C19F02EFB3F
:105B0000DDE72E602868386009B00120BDE8F08F1D
:105B10002079022804D33E6009B00120BDE8F08F4F
:105B2000401C2071DBF8100090B1DBF80C104140F4
:105B30004840CBF810004840CBF80C00E670FF2A34
:105B400004D0104619F07EFA84F800A00120A0705D
:105B500009B00020BDE8F08FC42300202DE9F041FA
:105B60000646354615F8014B3CB12E2C05D02F2C9E
:105B700003D02C2C01D03E2CF4D1A81B401EC7B260
:105B8000384619F033FC3946304619F045FC3044AC
:105B9000461C2CB12F2C03D02C2C01D03E2CE1D153
:105BA000BDE8F041002019F021BC000070B50546A9
:105BB0000C460C49284615F03BFE0B4B5A1E30B1E3
:105BC000187840F0020018700720907070BDD56002
:105BD0000020106190705471187820F00200187045
:105BE00070BD0000C4230020250100202DE9F041F4
:105BF000DFF8C880074608EB07000C4690F838022B
:105C0000C00659D005213846FFF7A0F92C480721D6
:105C1000C619B1EB141F0AD198F83B01012810D026
:105C2000B07DC00603D502213846FFF78FF97D1CF1
:105C3000482C0DD020073DD498F83C0101280DD008
:105C400017E0A007EFD50221384615F035FCEEE746
:105C5000E8B2BDE8F041072100F088B9E00704D0C0
:105C6000E8B2082100F082F903E004213846FFF78A
:105C70006DF9A00702D5E8B220F0BEF960070CD597
:105C8000B07D800618D4E8B2102110F0CFFC384661
:105C9000BDE8F041032115F00FBCB07D80060BD5A7
:105CA000E8B2112110F0C2FC3846BDE8F0410321F2
:105CB000FFF74CB96007E3D4BDE8F081E41500209C
:105CC000801C0020014A515C1AF036BE148702087D
:105CD00070B5194C194D207820B101281ED01848F4
:105CE000E86170BD19F0A2F8286001202070002141
:105CF0004C201AF021FE134D134C6878015D54209E
:105D00001AF01AFEE878015D5C201AF015FE287979
:105D1000015DBDE8704064201AF00EBE19F086F8EF
:105D200029684FF4FA63411A0022591A72EB0200F3
:105D3000D7D20220207070BD7C000020E41D00201E
:105D4000FD6B0108E2860208E48602082DE9F041B5
:105D50007748D0B090F815137648002939D04168BB
:105D60007548FCF7FDFA754E30787178884200F07E
:105D7000DA80401C00F01F0400208DF810007048ED
:105D8000817890F805C00379C2788DE80E104378C9
:105D900002786CA144A820F0D5FB06EB4400C07843
:105DA000292851D2DFE800F0931A1A1A1A1A1A1A7F
:105DB0001A727272727272721A1A1A7272721A727B
:105DC000721A721A1A7272721A1A1A1A1A1A1A1A7B
:105DD0001A0001685848FCF7C3FAC4E706EB44050B
:105DE000A878401E272884BF00208DF8280103D8FA
:105DF000C0B24AA920F005FB4D4890F815030028D1
:105E000044A822D0FCF78AFA07464AA8FCF786FA8B
:105E100007EB0008E878544F07EBC0004068FCF738
:105E20007DFA4044B0F5807F51D244A904A8FCF724
:105E300041FA4AA904A8FCF73DFAE87807EBC0004C
:105E4000416804A8FCF736FA41E0FCF767FA074618
:105E50004AA8FCF763FA07EB0008E878424F57F8C6
:105E60003000FCF75BFA4044B0F5807F2FD244A9A4
:105E700004A8FCF71FFA4AA904A8FCF71BFAE87863
:105E800057F8301004A8FCF715FA20E0284890F8DD
:105E90001503002844A82CD0FCF740FA06EB440573
:105EA0008046E878304F07EBC0004068FCF736FAD0
:105EB0004044B0F5807F0AD244A904A8FCF7FAF95F
:105EC000E87807EBC000416804A8FCF7F3F91A482A
:105ED000FCF724FAC0F5007504A8FCF71FFA854208
:105EE00021D904A91448FCF7E5F950B02046BDE8D3
:105EF000F081FCF713FA06EB44058046E8781A4F68
:105F000057F83000FCF70AFA4044B0F5807FDED243
:105F100044A904A8FCF7CEF9E87857F8301004A893
:105F2000FCF7C8F9D3E7307850B0BDE8F081000045
:105F3000E4150020C883020834590020601D0020A9
:105F4000680000203230253032642D253032642D37
:105F50002530326420253032643A253032643A25C7
:105F60003032642020000000E08302082DE9F04177
:105F70002B4E07460D463068C14389074ED00104B9
:105F800002D520F400403060DFF89880D7B17C1E45
:105F9000082DE0B24FF000012FD015F08DFA08EB7C
:105FA000070090F83702C0F34110FEF75FFB30683E
:105FB00020F4C04040F0040030601B4801780B29F9
:105FC00022D025E0072D07D0082D0ED040F010007C
:105FD0003060062D0DD00EE098F83801FEF746FB34
:105FE000306840F010003060E2E740F03000306090
:105FF00001E00220D9E70120D7E715F05DFAE0B211
:10600000042115F059FAF6E7016E41F480010166AA
:1060100029463846BDE8F04110F008BBBDE8F081E4
:10602000801C0020E41500203815002010B504461F
:106030000B4890B0826822B10AA1684620F082FA2B
:1060400003E00DA1684620F07DFA10A1204615F06E
:106050006BFB81B26A46204615F082FB10B010BD82
:106060007C2200203C4572723E4552527C302564B1
:106070003C2F4572723E00003C4572723E455252C2
:106080007C30303C2F4572723E0000003C457272FD
:106090002F3E00002DE9F04104460FF039FA5C492B
:1060A0000A20487121785C4DB1FBF0F259498A5CB5
:1060B00042F01002EA722278B2FBF0F300FB1322E6
:1060C0008A5C42F010022A736278B2FBF0F300FBA4
:1060D00013228A5C2A7263780A2B02D342F01002E0
:1060E0002A72A278B2FBF0F28A5C42F010026A7265
:1060F000A278B2FBF0F300FB13228A5C42F010029C
:10610000AA72E278B2FBF0F28A5C6A74E278B2FBBF
:10611000F0F300FB13228A5CAA742279B2FBF0F23E
:106120008A5C42F01002EA742279B2FBF0F300FBC1
:1061300013228A5C2A75A379B3FBF0F3CE5C6E75EB
:10614000A379B3FBF0F700FB1730085CA875E07982
:1061500016281BD2DFE800F01A0B0B0B0B0B0B0BF6
:106160000B54484E131A1A1A0F1A1A1A1A1642F01A
:10617000100028750AE046F01000687506E002215C
:10618000302001E0602140201AF0D6FBE97A182087
:106190001AF0D2FB297B20201AF0CEFB297A0020AE
:1061A0001AF0CAFB697A08201AF0C6FBA97A1020F7
:1061B0001AF0C2FB697C4C201AF0BEFBA97C54206B
:1061C0001AF0BAFBE97C5C201AF0B6FB297D64204A
:1061D0001AF0B2FB697D6C201AF0AEFBA97DBDE818
:1061E000F04174201AF0A8BB012130201AF0A4FB62
:1061F00021210AE0012130201AF09EFB322104E027
:10620000012130201AF098FB30213820BCE7000033
:10621000801C002014870208E41D002010B50FF038
:1062200077F940214C201AF087FB402154201AF0C6
:1062300083FB40215C201AF07FFB4021BDE8104029
:1062400064201AF079BB2DE9F04F0D461446114633
:1062500010F062FDA220E080AC2060810020D726F3
:10626000D9210422A3274FF0050C4FF0D1084FF09D
:10627000CE094FF0CF0A4FF0D00B4FF0D20E292DA0
:1062800029D2DFE805F028191C1F152225152765DE
:106290005C5F313C41572A2D2F696C48454D515563
:1062A000704A46353A28777A7D74808374858700F2
:1062B000A4F80880BDE8F08FA4F80890FAE7A4F8E5
:1062C00008A0F7E7A4F808B0F4E7A4F808E0F1E7BD
:1062D000D32000E0D4202081ECE72681D8201DE0E7
:1062E000268159E0D52114E022806680D82119E06A
:1062F000F5211AE0E080208110E0F52234E02280D0
:10630000DA216180A780F5E72280DA22628009E045
:10631000DC21218102E0DD210DE027816081C9E7D8
:1063200022806680A180E5E7E6212180678004E085
:10633000DC2030E0B32121806080A080DAE7228079
:10634000062112E0228007216180A4F804C0D1E771
:106350002280A4F802C0F0E72280DE2105E0A4F844
:1063600000C0092101E0E62222806180E5E7A4F86F
:10637000088011E0A4F808900EE0A4F808A00BE053
:10638000A4F808B008E0A4F808E005E0D32002E093
:10639000D42000E0D520208161818BE72DE9F041F8
:1063A0002A4F2B4D0C2679682A782C46092847D28B
:1063B000DFE800F005112534293D383B3B0042F071
:1063C000010020F0020028700120A0710522214860
:1063D000FBF78EFF36E012F0010F4FF006060AD0F1
:1063E0001C4800F0A7FA40B1287840F0020028705D
:1063F0000220A07126E0A67124E0A67122E0BDE88B
:10640000F04111F031BE7869FBF7EBFF124D687077
:10641000B869FBF7E6FF2870A67113E0BDE8F0410C
:1064200011F0BEBD0B20A0710CE0A6710AE0A671B0
:10643000A078FE2806D016F0F1FCFE20A07001E046
:106440000520A0710120BDE8F0810000F4230020A8
:1064500038010020480100204201002010B5002032
:1064600014F04AFB40F29C61144814F03BFC144CBD
:106470002068010206D513490A68134B02F4E06252
:106480001A430A6020F00300206012F081FA1048DD
:106490000E490162002141770F490E48C86113215E
:1064A000002010F0C3F8208810F4C04F04D10B482E
:1064B000017841F00401017010BD0000E4150020D6
:1064C000801C00200CED00E00400FA05F9450108ED
:1064D000C0150020FD6B0108E41D00206E000020A7
:1064E0002DE9F0434C4900204C4C0A784B7802EBE4
:1064F000820203EB4202D7B2494A0A2501268046AE
:106500004FF0020C4FF064090E2F7AD2DFE807F04B
:1065100079070A0F122326292C5379795D6394F8A1
:10652000153302E094F816335B1C8B704BE094F843
:1065300017335CE094F8BA30B3FBF9F48C7009FBC4
:106540001434B4FBF5F4CC70B3FBF5F405FB143351
:106550000B7103212CE094F8183348E094F81933B8
:1065600045E094F81A33E0E72C4B42F21076B3F88A
:106570005836B3FBF6F406FB14368C704FF47A747D
:10658000B6FBF4F6CE70B3FBF4F604FB16364C46BD
:10659000B6FBF4F60E71B3FBF9F609FB1634B4FB47
:1065A000F5F44C71B3FBF5F405FB14338B71052145
:1065B0005171BDE8F08394F87030012B01D18E70D9
:1065C00001E081F802805671F3E7144B93F89A3694
:1065D000AA2BF6D0F3E7114B93F89B36632B03D924
:1065E0000E4C632384F89B360C4B93F89B36B3FB1D
:1065F000F5F405FB14338C70CB7082F805C0D8E736
:10660000FFE7A7F13203262B03D8E31993F8B13241
:10661000EDE70120CDE70000C0150020E4150020C3
:10662000700000202DE9F047DFF8289100244B4648
:1066300099F8000099F8011000EB800001EB400090
:10664000C7B2987893F803C000EB80010CEB4106C9
:10665000414A751E93F80480F1B20E2F6CD2DFE828
:1066600007F06B070C1419272C3136556B6B5C67E0
:1066700002286BD282F8150369E0401E082865D213
:1066800082F8160319F082FA61E00A2D5ED282F8D0
:1066900017135CE0642148430CEB8C0100EB4100D4
:1066A0004044A0F10B01F52950D282F8BA004EE027
:1066B000622D4BD282F8181349E0072D46D282F89A
:1066C000191344E0022841D282F81A033FE042F253
:1066D000107250430CEB4C02C2EBCC1200EBC20028
:1066E00008EBC80202EB081200EB820299F80500E1
:1066F00099F8061000EB800002EB40000844B0F56A
:10670000803F23D21449A1F8580620E0012801D087
:1067100030B9022082F8700019E0012801D010B1D0
:1067200014E0552000E0AA200B4981F89A060EE0FB
:10673000094880F89B160AE0A7F13200272805D8FF
:10674000102E03D2D01980F8B11200E001242046A7
:10675000BDE8F087C0150020E4150020012181402C
:10676000024842688A43426070470000840000206B
:106770000449D1E90020904202D008600CF06CBFBF
:1067800070470000840000200121814002484268D7
:106790005140416070470000840000200121814089
:1067A00002484268114341607047000084000020A5
:1067B00010B5002103231522084617F0BBF807493E
:1067C0004870FE2809D0FE2088700020C870C8716B
:1067D000087014200A31088010BDFEE7380100203F
:1067E0002DE9F8434E4D687817F03EF80A2700244B
:1067F000C8B1687817F052F84FF00108002838D077
:1068000018F014FBE8606946687816F09DFC454E68
:1068100000B3E8799DF80020411CC9B2E9713254F7
:106820001F2910D010E0EC716F71EC703C480470BF
:106830002C71A878FE2803D016F0F0FAFE20A8707C
:106840000120BDE8F883EC716946687816F07CFC9D
:106850000028DED19DF800000A281CD1E8793454C4
:10686000EC7111F0C1FA3048006811F0A7FA6871B4
:1068700011E0E87878B118F0D9FAE968401A2B49A4
:10688000401A74F1000006D318F0D0FAE860022034
:10689000687185F80380E87805283DD2DFE800F0CC
:1068A00003243C3C0700AC7118F0C0FAE86068783B
:1068B00017F014F80646DFF87890A87959F8200008
:1068C000FBF72CFD864202D20120BDE8F883A879AF
:1068D00059F82010687817F063FA687816F014FCFD
:1068E0000D20A87185F8038068790A2814D0FFF775
:1068F00055FD042158B1A8790D2801D0E97003E0B5
:106900006879022800D1EC706F712C7104E0A879CD
:106910000D2801D0E970CAE70120BDE8F883000026
:1069200038010020D0230020F423002020BF0200E3
:1069300048A8020810B50C460146052206A0FBF740
:1069400002FD28B90522214603A0FBF7FCFC08B193
:10695000002010BD012010BD6D6569616E00000052
:1069600010B5012806D002281CD003281ED0092803
:1069700028D11EE00EF0F4FD0CF0F0FF4FF47A7415
:10698000204620F0D3FD0CF0E9FF204620F0CEFD9C
:106990000CF0E4FF204620F0C9FD0CF0DFFF0EF004
:1069A000B7FD0FE00420FDF761FE0BE0FCF723F9D3
:1069B00008E0FEF78BFB04480168044A01F4E0613B
:1069C00011430160012010BD0CED00E00400FA0548
:1069D00078B400250D8000950278431C002A2ED043
:1069E0004FF6FF743C2A02D0402A08D00DE09DF8F3
:1069F000000040F00100009018460C8005E09DF872
:106A000000C04CF0020CCDF800C09DF800C01CF096
:106A1000030F03D1202A1AD02C2A18D02C2A0ED0EA
:106A20001CF0010F04D01CF0020F01D03E2A06D04A
:106A30000A88521C0A8013F8012B002AD2D19DF833
:106A4000002012F0020F00D10D8078BC704718466C
:106A5000F1E700002DE9F05F04460E46608800284B
:106A600035D0FE277188328811442288114448406D
:106A70001FFA80F80025DFF888A1DFF880910AF579
:106A8000257B89F8005005EB450000EBC5000AEBBB
:106A9000800090F824100D2922D004291AD0B0F8D3
:106AA000270040451CD115F0DBF86088BBF81210B8
:106AB000884215D12088BBF81010884210D1306868
:106AC000DBF8181088420BD10120BDE8F09F0020B0
:106AD000BDE8F09FB0F827006188884200D12F46BA
:106AE000681CC5B20F2DCCD3FE2F24D089F80070BE
:106AF00015F0B6F899F8000000EB400101EBC00179
:106B00000AEB8100A0F827803E483268C0F8C8210F
:106B10007268C0F8CC213289A0F8D0212088ABF867
:106B200010006088ABF812005AF82100CBF80C0076
:106B30000120BDE8F09F607B10F0020F07D0DFF866
:106B4000C880B8F8380028B10020BDE8F09F0020C8
:106B5000BDE8F09F002505EB850008EB80010A8A5F
:106B6000CAB163889A4212D14989228891420ED1D2
:106B700058F820003168884209D118F05FF905EB18
:106B8000850108EB810148820020BDE8F09F681C68
:106B900085B2032DDFD3002789F8007007EB47008B
:106BA00000EBC7000AEB800090F8250010F0080FFA
:106BB0001CD015F055F8BBF812006188884215D139
:106BC00005EB850008EB8005306828607068686018
:106BD00030892881208868816068E8606088288220
:106BE00018F02CF968820020BDE8F09F781CC7B22D
:106BF0000F2FD1D30020BDE8F09F0000A20100209C
:106C0000E4510020C8520020A454002070B48446EF
:106C100017480C680068844202D1FF2070BC70479E
:106C2000FF23144A0020BCF80250D689AE4208D196
:106C30009389BCF80060B34202D11368A342EDD03F
:106C400003461C32401CC0B21028EED3FF2B0CD0E0
:106C5000084AC3EBC30002EB800004604A6842604C
:106C600009890181BCF80010818170BC1846704709
:106C7000555C0020E456002078B400250D80009576
:106C80000278431C002A2ED04FF6FF743C2A02D013
:106C9000402A08D00DE09DF8000040F0010000906F
:106CA00018460C8005E09DF800C04CF0020CCDF8B1
:106CB00000C09DF800C01CF0030F03D1202A1AD099
:106CC0002C2A18D02C2A0ED01CF0010F04D01CF056
:106CD000020F01D03E2A06D00A88521C0A8013F8FF
:106CE000012B002AD2D19DF8002012F0020F00D112
:106CF0000D8078BC70471846F1E700B503460020C8
:106D0000D873184621F08CF80021585C20B1481C3B
:106D1000C1B20F29F9D300BD0F29FCD220200A46A9
:106D2000491CC9B298540F29F9D300BDF0B59FB0E2
:106D300016460C4607467C2269464FF4A04013F0E5
:106D400059FF00206D46295CFF2903D0401CC0B2CA
:106D50007C28F8D348B145F25C0101EB40102022B9
:106D6000294613F047FF002008E001201FB0F0BDC6
:106D70003918401C695C04F8011BC0B2B042F7D35B
:106D80000020F3E72DE9F0431746804638449FB0D2
:106D90000D46202842D84FF4A0497C226946484637
:106DA00013F028FF00246E46305DFF2804D0641CD9
:106DB000E4B27C2CF8D301E07C2C0AD300242022FE
:106DC000314645F6DC7013F015FF484613F09AFE85
:106DD00008E03CB145F25C0000EB44102022314653
:106DE00013F008FF002006E008EB000115F8012B66
:106DF000401C7254C0B2B842F6D304F5A04013F060
:106E00007BFE572013F032FF45F27C0000EB44106C
:106E100013F072FE2021684613F064FF1FB0BDE836
:106E2000F083000070B50E460446002512E080286D
:106E300001D9208840BA00F017F80246701908A15D
:106E40001FF080FB2D1D2078ADB2802801D2641C7C
:106E500000E0A41C20780028E9D17055284670BDB8
:106E6000253034580000000030B500231A46802831
:106E700011D30B4C9918490834F82150854203D995
:106E8000A1F101018AB203E006D201F101018BB246
:106E90009342EFD9002030BD04EB8100408830BD23
:106EA000448102083FB50DA292E83800D2680392EF
:106EB0008DE838006B460AE003EB121212780A7074
:106EC00010F8012B02F00F029A5C4A70891C0278BC
:106ED000002AF1D1002008703FBD0000303132336C
:106EE0003435363738394142434445462DE9F84375
:106EF00001213D2011F00CF901214B4800F0ECF884
:106F000001214A4800F0E8F843F6F070ADF80000BF
:106F10001026474F8DF8036002248DF80240694621
:106F2000384600F08DF840213846FBF765FE4FF4F7
:106F30004040ADF8000048258DF8035069463846BA
:106F400000F07EF80F20ADF800008DF80240002020
:106F50008DF803006946384600F072F84FF01808C3
:106F6000ADF8008014208DF80300324F8DF80240F8
:106F70006946384600F064F84FF47040ADF8000000
:106F80008DF803608DF802406946384600F058F8E5
:106F90004FF00109ADF800908DF803508DF80240D4
:106FA0006946384600F04CF82020ADF800008DF816
:106FB00003506946384600F043F849F20210ADF834
:106FC000000003278DF802708DF803601A4E6946A1
:106FD000304600F035F84FF42060ADF800008DF831
:106FE00002708DF803806946304600F029F860028F
:106FF000ADF800008DF802708DF8035069463046F8
:1070000000F01EF80420ADF800008DF802402820A2
:107010008DF803006946094800F012F8074910315D
:10702000C1F80090BDE8F883000130000002300094
:1070300000100140000C0140000801400014014014
:10704000F0B5CC78002204F00F03E40601D58C786B
:1070500023430C784FF00F0C4FF0010EDCB10568A4
:107060000E880EFA02F42640A64210D196000CFAC1
:1070700006F725EA070703FA06F5CE783D43282EE2
:1070800002D0482E02D002E0446100E00461521CAC
:10709000082AE5D305600A88FF2A1CD94468002223
:1070A00002F108060EFA06F50E882E40AE420ED109
:1070B00096000CFA06F7BC4303FA06F7CE783C4379
:1070C000282E00D14561CE78482E00D10561521C92
:1070D000082AE5D34460F0BDF0B5104D6B68440D4F
:1070E000260184B2C0F30157B440C0F30342032F1A
:1070F00005D0C0020AD503209040834307E06868AA
:1071000023F0706220F07060686002E0A34343F0F7
:10711000706201B122436A60F0BD000000000140CE
:107120002DE9FC5FDFF8D4A2B34C0AF2C650DFF8B9
:10713000D082B4F808C0019098F80C000025411ED8
:10714000D8F860200AF2F6532E464FF00F0B4FF09E
:107150000B0E4FF47A77C9B242F480290AF2266AFC
:107160000093BCF1110F7DD2DFE80CF0090F162758
:107170002E3A414A516794CDD4E2F0EEED0022F46C
:107180008040C8F860000120D0E03A4603219DA06D
:1071900002F0C6F80220C9E098F802200323382A3A
:1071A00009D0B8F80420002A06D120B188F80C10C4
:1071B0003A4694A001E123811AE13A46012197A0C1
:1071C00002F0AEF80420B1E098F80200162803D0CF
:1071D000B8F8040010B10BE10720A7E00520A5E0F6
:1071E0003A46012190A002F09BF806209EE098F814
:1071F00002003828F0D0B8F804000028ECD0F7E0FE
:107200003A4601218BA002F08BF808208EE0B8F8F6
:10721000041009200029B7D098F802102B2938D083
:1072200098F802002C286BD098F80200322867D01A
:1072300098F90200401C76D1DAE081A18448FBF77E
:107240008FF883480199FBF735F86C4890F8F605FC
:1072500038B180A17E48FBF72DF87D480099FBF7F7
:1072600029F800E0B9E0654890F8260638B179A120
:107270007748FBF71FF851467548FBF71BF876A1D6
:107280007348FBF717F83A460121714802F048F8B5
:107290000A204BE098F80210382931D0B8F80410D1
:1072A000002989D160B366A16948FBF759F868489D
:1072B0000199FAF7FFFF514890F8F60538B165A13A
:1072C0006348FAF7F7FF62480099FAF7F3FF4B4873
:1072D00090F8260638B15FA15D48FAF7EBFF5146FA
:1072E0005B48FAF7E7FF5CA15948FAF7E3FF98F823
:1072F0000C003A46401EC1B288F80C1054485CE0BD
:10730000A4F808E074E03A46012154A002F008F81D
:107310000C200BE098F802100D20382904D0B8F8A2
:10732000041019B164E026E0A8F8046020815FE051
:10733000B8F8040000285BD13A460A213DA001F0CC
:10734000EFFF0E20F2E722E018E0FFE798F80220B6
:107350002E2A10D098F802202F2A0CD098F802205C
:10736000332A08D0B8F804204ABB20B188F80C10A2
:107370003A4630A021E0A4F808B039E03A463C2172
:1073800039A0C8F8609001F0CBFF1020CEE798F844
:1073900002304B2B03D0B8F804203AB128E0267015
:1073A00022F400300125C8F8600017E040B1C8F8A9
:1073B000609088F80C103A462BA001F0B1FF17E05E
:1073C0002078401CC0B220700F2809D229A010F0EC
:1073D00079FC17F02BFDC8F84C000225268107E048
:1073E00026702681032588F801602549C8F8081011
:1073F0002846BDE8FC9F000018000020E41500208E
:107400003815002041542B51494D55583D313B2BE7
:1074100051494E44493D310D0000000041542B4379
:10742000474154543F0D000041542B4347415454AD
:107430003D310D0041542B514953544154450D00E9
:1074400041542B51495245474150503D00000000E6
:10745000600500202C0000000D00000041542B515D
:10746000494143540D00000041542B51494C4F43B6
:1074700049500D0041542B514944454143540D009E
:107480003D9300082DE9FE4FCA487F25CA4CD0F82D
:107490005A06002835D0C948C078C00714D0206EDD
:1074A000C10210D520F4801020664FF47A720121B9
:1074B000C3A001F035FFC64890F80804C007FAD011
:1074C000C4A017F003FB657094F90110C0480127B0
:1074D0004030CB4E4FF0000A4FF003084FF0020B44
:1074E00047F230594FF4FA620090102971D2DFE868
:1074F00001F00D16222A445159718CACB7D4E5FA2B
:10750000F8F76570BFA017F0E1FADDE786F80080B4
:10751000206E20F4801020666770C1A045E14FF412
:107520007A720121A6A001F0FBFEA94890F8080498
:10753000C007FAD0AFE04FF47A720321C0A001F087
:10754000EFFE4046CAE0A07833280AD0A088002881
:107550003DD1207B38B1401EC1B221734FF47A7205
:107560008AE00520BAE0206E20F4804040F400302C
:10757000206604206070B5A017E1FFF7D1FD012857
:1075800004D0022823D16570B9A00EE105206070F7
:10759000BDA00AE14FF47A720321C2A001F0C0FE3F
:1075A00006209BE0A07838280BD0A08800280ED1B8
:1075B000207B58B1401EC1B221734FF47A72B9A03A
:1075C0005BE04FF47A70A080072087E06570BDE82B
:1075D000FE8FD6E07748774A764990F85C06B2F895
:1075E0005E2691F85D168DE807007248B4A190F808
:1075F0005B3690F85A2676481EF0A4FF4A460121D1
:10760000734801F08DFE082068E0A078092718284B
:1076100007D0A07819280DD0A0880028D7D167708E
:10762000D5E7B1A017F052FAB8484078B070A4F886
:1076300004A0F4E7B6A017F049FA30780028C5D0C6
:10764000401E3070A4F804A025E0A0880028BED118
:1076500084F8557003217AA001F062FE0A203DE013
:1076600094F8550002280DD0A0880028AFD1207BC7
:1076700060B1401EC1B2217371A003B0BDE8F04FEC
:1076800001F04EBE86F800800B2027E030780028FD
:107690009CD0401E3070584620E0022110F036F990
:1076A00002B2B280A2A14A481EF04CFF4FF47A7297
:1076B0000121474801F034FE0C20607003F026FAE7
:1076C000A078112802D0A0880028F7D1B08881B214
:1076D000009810F021FBA4F804900D20607076E76C
:1076E00036E019E0FFE7A0781C280ED0A0781D280E
:1076F00005D0A078132802D0A088002890D1206E51
:1077000020F4000020668EA01FE096A017F0DEF99E
:10771000A4F804900E20E1E794F85A0088B19BA0E9
:1077200017F0D4F994F85A004FF47A72401E84F896
:107730005A009E48032107709DA001F0F1FD0F2023
:10774000CCE7A0880028CAD19EA017F0BFF93DE77A
:10775000A078362805D0A0880028C0D16570A2A0E6
:1077600023E04FF0FF324FF40071009810F0C6F99B
:107770008E4800780028EAD1206E40F48010206600
:1077800024E717F053FB206584F801A0A248A0600D
:10779000206EC002A3D4707810B1401E707016E73E
:1077A0000F2070709D48A0609DA0BDE8FE4F17F0AF
:1077B0008DB90000E4150020381500206400002079
:1077C00041542B5149434C4F53453D310D0000006E
:1077D0006005002045746865726E6574204F4B2CFF
:1077E0002047505253205032502073657276657294
:1077F00020646973636F6E6163740D0A000000009A
:107800004C00002047736D20503250207365727613
:107810006572206970206572726F722E0D0A000009
:1078200067707273206C6F67696E205032502073DE
:1078300065727665722073746172740D0A000000BF
:1078400041542B514953544154450D006770727394
:10785000206572726F722C6E656564207265636F4D
:107860006E6669672067707273210D0A0000000060
:107870007265636F6E6669672067707273206661F8
:10788000696C210D0A0000007265636F6E6669679E
:1078900020677072732073756363657373210D0ABB
:1078A0000000000041542B5149444E5349503D3093
:1078B0003B2B5149484541443D313B0D0000000000
:1078C00041542B51494F50454E3D312C2254435089
:1078D000222C2225642E25642E25642E2564222C3C
:1078E000222564220D0000006770727320636F6EA2
:1078F0006E61637420503250207365727665722019
:10790000737563636573730D0A000000DC1C00204F
:107910006770727320636F6E6E61637420503250B3
:1079200020736572766572206661696C0D0A0000CD
:1079300041542B514953454E443D312C25640D0093
:10794000677072732073656E642064617461207463
:107950006F2070327020736572766572206661697F
:107960006C0D0A00677072732073656E6420646129
:10797000746120746F207032702073657276657246
:1079800020737563636573730D0A0000677072730B
:107990002072656365697665205032502073657288
:1079A00076657220646174610D0A00001D0200207A
:1079B00041542B514952443D302C312C312C35331C
:1079C000360D000067707273207761697420503241
:1079D00050207365727665722064617461207469E9
:1079E0006D656F75740D0A0067707273206C6F6738
:1079F000696E2070327020736572766572206661E0
:107A0000696C2C736572766572206461746120659F
:107A100072726F72200D0A00D59700083D9300081E
:107A200067707273206C6F67696E2070327020739C
:107A30006572766572206661696C2C20696E697466
:107A40002067736D206D6F64756C650D0A00000012
:107A50002DE9F84FAA48AB4C4FF07F06C078C0071D
:107A600003D1A948D0F85A06A0B9206EC10210D59A
:107A700020F4801020664FF47A720121A3A001F057
:107A80004FFCA64890F80804C007FAD0A4A017F04D
:107A90001DF8667094F90110A048DFF8B8924030E4
:107AA0000627AD4D4FF0010A4FF003084FF4FA627C
:107AB00047F2305B00900C2972D2DFE801F0060C2F
:107AC00014294354779CC9D7EAFF85F8008084F8CD
:107AD00001A0A2A0A6E084F855A00321A6A001F071
:107AE0001FFC0220D3E094F85500022871D0A08832
:107AF00000286FD1207B20B1401EC1B221739EA00F
:107B0000EAE0206E20F48010206666709DA089E077
:107B1000A9780FF05BFF02B2AA8099F80110A8784B
:107B2000814203D0401C00F01F00A8709CA17B483C
:107B30001EF008FD4FF47A720121784801F0F0FB45
:107B40000420607002F0E2FFA078112802D0A08823
:107B50000028F7D1A88881B2009810F0DDF8A4F8C9
:107B600004B0052093E0A0781C2813D0A0781D282D
:107B700005D0A078132802D0A08800285FD1206EFD
:107B800020F4000020668AA016F0A0FF28780028C4
:107B900029D106E08FA016F099FFA4F804B04DE0BB
:107BA000A5E0206E20F4801020664FE094F85A0083
:107BB00088B192A016F08AFF94F85A004FF47A72B6
:107BC000401E84F85A00032194A001F0A9FB07206D
:107BD0005DE08AE033E0A088002830D194A016F060
:107BE00075FF287818B1401E287050464FE099A0C4
:107BF00016F06CFFD5E7A078362806D0A0880028BC
:107C00001DD194F85A0008B318E04FF0FF324FF43A
:107C1000007100980FF072FFA880002806DD082090
:107C2000607094A0BDE8F84F16F050BF10F16301EA
:107C300001D0002854D198A016F048FF6770BDE825
:107C4000F88F99F80100A97888424ED16670F6E75E
:107C5000B5F9042052A131481EF074FC4FF47A7239
:107C600001212E4801F05CFB0920607002F04EFFFC
:107C7000A078112802D0A0880028F7D1A88881B266
:107C8000009810F049F840F6B830A0800A206070E3
:107C9000D5E7A0781C2809D0A0781D2820D0A0788E
:107CA00013281DD0A088D8B1C9E707E04FF47A7235
:107CB0000F2181A001F034FB0B20E8E7A0784A28CF
:107CC0000ED0A0880028BAD1207B48B1401EC1B296
:107CD00021734FF47A7278A0BDE8F84F01F020BB11
:107CE00094F85A000028ACD0A8E74046CFE717F038
:107CF0009DF82065002060707348A0609FE7000039
:107D00006400002038150020E415002041542B5158
:107D100049434C4F53453D310D00000060050020A4
:107D200045746865726E6574204F4B2C206F72200D
:107D300050325020736572766572206970206572CA
:107D4000726F722C206770727320636C6F73650D95
:107D50000A000000DC1C00204C00002067707273D9
:107D6000205032502073656E642070756C736520EE
:107D700073746172740D0A0041542B51495354417C
:107D800054450D00677072732050325020636F6E3F
:107D90006E616374206572726F720D0A00000000DC
:107DA00041542B514953454E443D312C25640D001F
:107DB000677072732073656E6420646174612074EF
:107DC0006F2050325020736572766572206661694B
:107DD0006C0D0A00677072732073656E64206461B5
:107DE000746120746F205032502073657276657212
:107DF00020737563636573730D0A00006770727397
:107E00002072656365697665642050325020736521
:107E10007276657220646174610D0A0041542B51C1
:107E20004952443D302C312C312C3533360D000075
:107E300067707273207761697420503250207365C7
:107E40007276657220646174612074696D656F7506
:107E5000740D0A00677072732020503250207365D1
:107E60007276657220646973636F6E6163740D0A64
:107E700000000000677072732050325020736572EA
:107E80007665722072657475726E20584D4C206450
:107E90006174610D0A0000006770727320503250E7
:107EA00020736572766572206461746120657272F8
:107EB0006F720D0A0000000041542B514953414399
:107EC0004B3D310D00000000D59700082DE9FF5F04
:107ED000FA48FB4C8078012814D1B4F860004004C3
:107EE00010D54FF47A720121F6A001F019FA206E34
:107EF00020F480402066F74890F80804C007FAD0C4
:107F00001320607094F901C0F248DFF8D483143074
:107F100000270121F04EF14D4FF4FA624FF0030BB0
:107F20004FF0110AA8F102090090BCF1130F7DD2A5
:107F3000DFE80CF00A151B232B41596886AED3DE0F
:107F4000F8F7F6F5F4F3F20098F8000020F0FF00DF
:107F500088F80000206E20F48040206669E001214E
:107F6000D8A001F0DDF9022016E1A078302802D077
:107F7000A08800285ED158460EE14FF47A720221A3
:107F8000D8A001F0CDF9042006E1A07833281ED056
:107F9000A08800284ED1207B28B1401EC1B2217399
:107FA0004FF47A72B0E0206E20F4804040F400304C
:107FB00020660520F0E0FFF7B3F8012807D002287B
:107FC00038D196F8BC00012803D013200CE106201C
:107FD000E2E02878697888422CD004B0C448BDE833
:107FE000F05F01F0F3BD96F8BB004FF0640201288A
:107FF0004FF0030104D0BFA001F092F90720CBE0BD
:10800000C3A0F9E7A0780821382817D0A088002855
:1080100010D1207B90B196F8BB10A0F1010001298E
:10802000C1B221734FF0640206D000E0B6E1B1A006
:108030006BE06170BDE8FF9FB5A066E0A780F8E740
:10804000A0880028F6D196F8BB00012811D0B6F818
:10805000A600A14B00907533B4A2B5A19D481EF0B7
:1080600071FA43F6982201219A4801F059F9092042
:1080700092E071367078B6F83530F278B1788DE8E4
:108080000F003378A9A2B1A192481EF05BFAE8E78D
:10809000A078182806D0A078192805D0A088002834
:1080A00001D0C7E7A780EDE098F80000C0F3820395
:1080B000032B08D24FF0005303EB70104FEAF0602F
:1080C00088F80000B5E796F8BC00012881D0A949DE
:1080D0004FF46160A1F85800D6E0A0880028A9D12B
:1080E00084F8547003217FA001F01AF90B2053E0AB
:1080F00094F8540002280DD0A08800289AD1207B43
:1081000088B1401EC1B2217376A004B0BDE8F05F13
:1081100001F006B90C203FE0C7E0C0E083E06FE06B
:108120004EE028E00AE098F80000C0F38202032A3B
:1081300074D396F8BC000128C8D0A5E028786A78E6
:10814000904203D08B4AB2F858203AB389F80470B1
:108150004D46009811F0AEF8687199F8052086A197
:108160005C481EF0EFF94FF47A720121594801F092
:10817000D7F80D20607002F0C9FCA078112802D059
:10818000A0880028F7D199F8051000980FF0C4FDD9
:1081900042F21070A0800E2060704BE7401C00F08F
:1081A0001F0089F8030005EB400089F80410C3782C
:1081B00081784E460122009810F0E4FF7071CCE700
:1081C000A0781C2817D0A0781D2802D0A0880028ED
:1081D000E3D198F80000C0F38202032A56D396F840
:1081E000BC000128A8D05046607062494FF461601D
:1081F000A1F858001EE747F23050A0800F20CBE7CF
:1082000094F8590058B1401E84F859004FF47A721E
:1082100003215DA001F084F81020BDE736E0A088BE
:10822000002880D006E7A0783628F8D129484030C9
:1082300011F0A4F802280AD0032806D0042804D09C
:10824000052802D0A0781A28E9D1A780E7E7A780FF
:1082500098F8001021F0E00188F80010206E0F213E
:1082600040F48040206689F801104249A1F8587016
:1082700099F8041011B199F80300287028786978EA
:10828000884201D00A2087E7504685E74FF0005228
:1082900002EB70104FEAF06088F800006BE60121F5
:1082A00008A001F03DF8122076E7A078302802D02F
:1082B000A08800289ED113206EE7000064000020F3
:1082C0003815002041542B5149434C4F53453D3004
:1082D0000D00000060050020E4150020DC1C0020DB
:1082E0001A00002041542B514953544154450D006C
:1082F0004D9D000841542B5149444E5349503D3146
:108300003B2B5149484541443D313B0D00000000A5
:1083100041542B5149444E5349503D303B2B514918
:10832000484541443D313B0D00000000544350009E
:1083300041542B51494F50454E3D302C222573223C
:108340002C222573222C222564220D0041542B510E
:10835000494F50454E3D302C222573222C22256456
:108360002E25642E25642E2564222C222564220DC0
:1083700000000000801C002041542B514953454E01
:10838000443D302C25640D0041542B514952443D4D
:10839000302C312C302C3533360D000067700A48F4
:1083A000A060B4F8600040043FF57BAE99F801008E
:1083B00018B1401E89F801003CE60F2089F8010041
:1083C0000248A06036E60000D59700083D930008FB
:1083D0002DE9F05FBE4C94F90180BF4DBD480027E8
:1083E0006A79D0F800B0521C204602F0FF0ABB4A5E
:1083F000007B0826411E92F800C052784FF0010E13
:108400004FF01409C9B2B8F10E0F6ED2DFE808F0D0
:1084100007152D354553646E8CA0C1FEF1F0AD48B3
:108420002F702BF4C04101606420A08003202070D5
:1084300084F801E00021AA4835E1A08800282AD16B
:10844000A8486F714BF4001190F830012871A148D1
:1084500001600520FEF7A2F90420FEF77FF9A2498A
:108460004FF48050086002203DE04FF47A720321FF
:108470009EA000F055FF032035E0A3780422382B9E
:1084800008D0A388002B06D120B121734FF47A7253
:1084900096A0A2E06270BDE8F09F3C23062299A15D
:1084A0009E481EF04FF84FF47A7203219B4800F06B
:1084B00037FF052017E0A2780621382A0AD0A288C3
:1084C000002AE8D130B13C2306228EA193481EF049
:1084D00039F87BE06170DEE74FF47A72032190A0F7
:1084E00000F01EFF07206070D5E7E0E0A278382A90
:1084F00008D0A288002ACED120B121734FF47A721D
:1085000087A06AE06670C6E700EBC00301EB430397
:1085100093F8E8300A2B04D285F800E00920607057
:1085200006E0401C687100E06E4968790428EBD3CE
:108530006A4994457ED068790428ACD3287910B173
:10854000401E287102E00A7084F801906F71A2E762
:10855000A08800289FD17CA17048F9F701FF6F48DF
:10856000F9F7DCFE6D490144687900EBC0025D4813
:1085700000EB4200E8300FF091FC74A16748F9F776
:1085800099FE4FF47A720321644800F0C9FE0A2074
:10859000A9E7A178382924D0A18800299BD150B31C
:1085A00069A15E48F9F7DCFE5C48F9F7B7FE5B4964
:1085B0000144687900EBC0024A4800EB4200E83011
:1085C0000FF06CFC61A15548F9F774FE207B4FF465
:1085D0007A72401EC1B251482173BDE8F05F00F0CD
:1085E0009FBE84F82C704EF66020A0800B207AE7A6
:1085F00044E02CE00AE0FFE755A00FF063FB41F2F6
:108600008830A0806879401C68717BE7A0780C28CE
:10861000BED0A0780A2813D0A088002897D14CA0FB
:108620000FF050FB2D480178407881420DD06879D9
:10863000401C00E009E0687141F28830A08061E7E9
:10864000944502D085F805A0F6E748464BE7A078A8
:108650000D250A280DD000F0D1FB01289ED13CA0A9
:108660000FF030FB2D4890F80804C007FAD0657071
:1086700011E70021384817F075F9F8E794450ED056
:1086800085F805A041F28830A08002F0E9FD0620BF
:10869000FBF7ECFF0520FEF781F8667001E084F837
:1086A00001902D480121BDE8F05F17F05BB902F0A1
:1086B000D7FD0520FEF752F80648016821F40011A5
:1086C000016017F063FA67702448A060E3E60000D9
:1086D00038150020801C0020310000201E1D0020C5
:1086E00020810208E41500201408014041542B5158
:1086F00041554443483D303B2B5153494445543D3B
:10870000303B0D0041542B514D49433D302C2564E5
:108710003B2B434C564C3D25643B0D00600500202F
:1087200041542B51544F4E454445543D342C312C2B
:10873000332C332C36353533363B2B51544F4E4585
:108740004445543D310D0000415444003B0D0000B0
:108750004154480D00000000008C0208D597000825
:10876000F0B50026054630463346344615E02F78EE
:108770009F40274307F07F0401F8014B2C78C3F199
:108780000707FC40401C5B1C072B04D1401C01F870
:10879000014B00231C466D1C761C9642E7DB002231
:1087A0000A70F0BDF0B500252B462E460FE013F001
:1087B000070412D00778C4F1080C07FA0CF72F430E
:1087C00001F8017B0578E540761C401C5B1C934258
:1087D000EDDB002008703046F0BD0578F5E70000BD
:1087E00010B5012186B088030FF092FC1B4C204687
:1087F00016F068FF00214FF4E1300090ADF808104A
:10880000ADF804100C20ADF80610ADF80C10ADF862
:108810000A006946204616F0C9FF012240F226618F
:10882000204616F0ABFF012240F22551204616F0FB
:10883000A5FF0121204616F03AFF01208DF8110016
:1088400002218DF812108DF8130025208DF81000EC
:1088500004A80EF011F906B010BD00000038014068
:108860000148006870470000AC01002038B50C20BA
:108870000AF0F4FF0DF012F900F0F0006FF01301B0
:1088800001EB9000C4B20CB3072100200DF018F9E1
:10889000601EC4B20DF002F9A8B101280ED0022862
:1088A00017D0022C0FD30DF0F9F80546AC420AD3CD
:1088B000294600200DF004F9601BC4B22000A4F189
:1088C0000101CCB2E6D140F2B45038BD4FF406708D
:1088D00038BD032CF7D3002000900DF0DFF80428FA
:1088E00007D10DF0DBF88DF801000DF0D7F88DF809
:1088F0000000BDF80000B0F5067FE4D340F2B451AB
:108900008842E5D9084638BD00200D4A014602EBF1
:108910004003401CB3F88030C0B219440828F6D395
:10892000C80840F6B211884201D20220704740F6D2
:108930001F41884201D2012070470020704700008B
:108940003203002038B512F039F804460F481049B8
:1089500090F9D10251F820000E49F9F75CFDF9F7C2
:1089600090FD204400906846F9F7DEFD027D0A493B
:10897000643A0A70027C521C4A70027B8A70027A46
:10898000CA7002790A710078487138BDE415002078
:10899000288702080000614568000020014801683E
:1089A00041607047AC010020064841780078814260
:1089B00006D104488430007A400701D40020704773
:1089C00001207047C404002010B540687C21F9F7ED
:1089D0009BFC002800D0407810BD10B54FF0FF344C
:1089E00040687C21F9F790FC38B110F8011F11B1F3
:1089F000F9F7F7FC0446204610BD6FF0010010BDEA
:108A000010B540687C21F9F77FFC002800D0401C9D
:108A100010BD000070B55C212248F9F740FC2248E7
:108A20000021234A81702148D0612348214A0262F3
:108A3000FF2202774177214800681A4C800620689F
:108A400002D540F0200001E020F020001C49206009
:108A50004FF4807048611B4DC00128600020FDF775
:108A60007DFE164908200C3108600420FDF776FED3
:108A7000A81428600520FDF771FE0120FDF76EFEA9
:108A8000206820F4001020600220FDF787FE0320FC
:108A9000FDF784FE0620FDF781FEBDE8704007204B
:108AA000FDF77CBE801C002064000020D15C000823
:108AB000E41D0020F9450108C0150020080C014004
:108AC000001001401408014010B516F0AFF90B4931
:108AD0004AF6C8730022096D411A591A72EB020056
:108AE00005D30748074940788978884204D006486A
:108AF00001F06CF8012010BD002010BD38150020D9
:108B0000DC1C00204C000020517A0008054AD0717E
:108B100031B1012802D00220907170470320FBE799
:108B20000020F9E7180000202DE9F05F854D0024B2
:108B30002946A879844FDFF81482CA792646072887
:108B40007ED2DFE800F0041CFA3195AFD80008EBC4
:108B5000020191F85900002872D0401E81F8590096
:108B600079487BA140381DF0EDFC774840380FF084
:108B7000A9F80120A87116F059F92861DEE098F8EB
:108B8000020036280AD016F051F9296941F28832DC
:108B9000411A0020511AB04152D3CFE0012A01D02E
:108BA0000220A6E00320A4E004226EA13846F9F7D3
:108BB000CAFB0028D0D004226CA13846F9F7C3FBC9
:108BC0000028C9D004226BA13846F9F7BCFB002865
:108BD00036D15C49381D0C310DF09CFDD7E9028976
:108BE000E968AA4678181030C7F83002056807F11E
:108BF0001000834618F070F9DAF80C005F49384429
:108C00000674FF200870584618F076F80028DFD167
:108C10005846F9F783FB5646CAF80C0000280FDDCA
:108C20000146584618F070F952A0391D00683860A6
:108C3000F0680DF039FDC7E90289F068384400E0BA
:108C40007BE01030C7F830020560F3683E4814330B
:108C5000F360F2794AA140381DF074FC16F0E6F892
:108C60003061394840380FF02DF80420B07165E0CC
:108C700001F04CFF98F80200112809D016F0D6F840
:108C800029694FF47A72411A891A76F10000EFD3FC
:108C9000A88981B238460FF03FF816F0C7F828616E
:108CA000052026E098F802001C2812D098F802004F
:108CB0001D2842D098F8020013283ED016F0B6F8CE
:108CC000296940F6B832401A0021101AB14134D354
:108CD00034E01D482FA140381DF034FC16F0A6F8F2
:108CE00028610A2088F80C00174840380EF0EAFF87
:108CF0000620A87122E098F802004A281DD016F03C
:108D000095F829694FF47A72411A0020511AB0413E
:108D100014D216F08BF8286198F80C0068B1401E48
:108D200088F80C000848EA791AA140381DF00AFCBE
:108D3000054840380EF0C6FF00E001242046BDE89B
:108D4000F09F000018000020A0050020381500202A
:108D500041542B514952443D302C312C25642C3543
:108D600033360D00256D61490000000040616C4103
:108D7000000000004069654D00000000B8000020C0
:108D800041542B514953454E443D25642C25640DD7
:108D90000000000041542B51495341434B3D256491
:108DA0000D00000070B586B016460D46044614222C
:108DB0000DA16846F9F75AFA002069460CE02278BE
:108DC00001EB121212782A7014F8012B02F00F0234
:108DD0008A5C6A70AD1C401CB042F0DB0020287039
:108DE00006B0700070BD0000303132333435363794
:108DF0003839414243444546000000002DE9F05F08
:108E0000E14C94F82C2020460025DFF880930527BC
:108E1000DF4EDFF8808390F82D10072A72D00CDC2B
:108E20004FF0FF0A42F210704FF01D0B15D2DFE831
:108E300002F01A27303B467F93000B2A72D006DCE3
:108E4000082A70D0092A6FD00A2A06D14BE10C2AD1
:108E50006BD01D2A6AD01E2A69D0F17888F80010DC
:108E60000120BDE8F09F75700021CB4816F07AFD17
:108E700040F6B830A08098F80000F07001207EE144
:108E8000A088002876D10021C44816F06BFD02208E
:108E900075E1FFF789FD0028F4D1757099F831016B
:108EA000012868D103206AE10121BD4816F05AFD6E
:108EB000A58084F82DA084F82E5004205FE1FF29BE
:108EC00021D0A080B04894F82E202F30115494F86F
:108ED0002E10491CC9B284F82E10042907D304218E
:108EE0000EF0C2FF002803DD757084F82C7090E04E
:108EF0007078401CC0B27070032844D8032084F8F6
:108F00002C0086E0A8E0FFF74FFD0028BAD1A0882A
:108F10000028B7D17078401CC0B270700328C1D946
:108F200058462CE109E1B8E0CEE010E11DE122E174
:108F3000FFF73AFD0028A5D199F8D2024FF00101C0
:108F4000062807D0974816F00DFDA58084F82DA0BF
:108F5000062014E19448F6E7FF2971D075700622C7
:108F600084F82C208B4A5578894A527932320A2962
:108F70004FD201E0A7E0DDE0DFE801F005070E20B9
:108F80002429383E47555846B9E7F570D0B2FAF76C
:108F9000D5FF002185480CE000217F4816F0E2FC57
:108FA00098F80000B07098F80110884204D10021B0
:108FB0007F4816F0D7FC2CE00720A0E7D0B212F0D3
:108FC000B3FE26E0F570D0B212F092FF21E07949AD
:108FD000086800F00303012B01D0030602D520F03E
:108FE00083000860D0B212F0C7FF12E00120FBF747
:108FF0003DFB00217048DCE70520FBF737FB002133
:109000006E4816F0AFFC082079E799F8D2120629CD
:1090100002D084F82DA0B4E0A0800021684816F0AA
:10902000A1FC0A206BE74EF66020A0800520FBF72C
:109030001DFB0021634816F095FC0B205FE7FFE75E
:10904000FFF7B2FC00283ED17078401CC0B27070AF
:1090500003283FF665AF6DE0FFF7A6FC98BB98F8D4
:109060000120B078824213D0401C00F01F00B07085
:1090700008EB4000544AC1788078FDF7E4F8524983
:109080004FF6FE70888100214F4816F06BFC78E0A7
:1090900000214E4816F066FC4CE0FFF785FC90B9C5
:1090A00099F83E0100EB4001C1EBC0104FF6FF7193
:1090B00001EAC000A0800520FDF750FB0120FDF76C
:1090C0006DFB09205BE037E00E2900D1A580A08868
:1090D00090BB0520FDF762FB0120FDF73FFB06205A
:1090E000FBF7C4FA26E03A4A4FF40046012910780B
:1090F00001D069B11CE040F0020010700122344937
:109100000020FDF73FFE33480660002132480CE0A6
:1091100020F00200107001222D490020FDF732FEE0
:109120002C48001D066000212C4816F01BFCA58071
:10913000A08808B984F82C7023E0FFF735FC00BB49
:109140004EF66020A08002F0A5F80C2017E00E2952
:1091500000D1A580A088A0B902F082F80620FBF714
:1091600085FA0520FDF71AFBE4E701211C4816F0FB
:10917000F9FB1E2003E0FFF717FC10B91F2084F84D
:109180002C0000206DE6000038150020E4150020BA
:10919000310000201E1D0020008C0208E687020816
:1091A000388C02081A8C0208288C0208468C0208A7
:1091B0005A8C0208801C0020808C02084E8C020809
:1091C000528C0208568C0208A40400204A8C020823
:1091D0007800002010080140A88B0208AE8B02081E
:1091E000428C020830B50346002006E01C785D780A
:1091F0000D704C709B1C891C801C9042F6DBD007C4
:1092000003D0462001F8020C521C002008701046C2
:1092100030BD000001480EF055BD00006005002083
:109220002DE9F041044602210AF032FA04EB400530
:10923000AD1C022128460AF02BFA00F0FF08AD1CF5
:10924000022128460AF024FA0446AD1C02212846D1
:109250000AF01EFA314FAD1C4FF000063870E007DF
:1092600008D0621CB91C2846FFF7BCFF3819641CE3
:10927000867004E02246B91C2846FFF7B3FF254458
:10928000AD1C022128460AF003FA7870103502213D
:1092900028460AF0FDF94FEA40004FF47A7190FB3E
:1092A000F1F201FB120405F102055FEA48600FD5F7
:1092B0000120F875287830280AD16878362802D03D
:1092C000352803D004E00E3C0E3501E00C3C0C3593
:1092D000DFF848807978C4F3470008F11808B875BA
:1092E000224649B129464046F8F7C0FF38190676AC
:1092F00038190676BDE8F081414628461EF066F929
:109300000446024629464046FFF72AFA28460DF051
:1093100033FA29464046F9F723F8E9E760050020CB
:1093200070B5054C0D46FF211646A1700EF0CAFC23
:109330002573A68070BD0000381500202DE9F05F70
:10934000D74C94F9018020460026056E007B4FF42F
:10935000807E411E4FF47A724FF4FA6C41F2883BE2
:109360004FF012094FF0140AC9B245F02007B8F1C6
:10937000240F6FD2DFE808F0121E252F3A454F5A0E
:10938000676F7589959BA8AEBCC4CCD2F1F0EFEEA7
:10939000EDECEBEAE9E8E7E66E6EF2F825F4C040A2
:1093A00020F01F0020F40000267040F400302066FA
:1093B00001205BE1BBA00EF085FC6420A0800220B0
:1093C00054E1A08800286AD1B8A00EF07BFC64208C
:1093D000A08003204AE1A088002860D1B6A00EF04A
:1093E00071FC40F6B830A08004203FE1A08800283E
:1093F00055D1B449C1F800E040F6B830A08005204E
:1094000034E1A08800284AD1AE49091DC1F800E026
:10941000A28006202AE1A088002840D1AA494FF462
:1094200000700861A4F804C007201FE1A08800288C
:1094300035D1A5494FF400704861A4F804B0FF206D
:10944000A070082012E1A08810B1A078002826D1D1
:1094500009200BE11CE10A219CA0FFF761FF0A2013
:1094600004E1A378382B06D0A388002B17D150B184
:10947000217396A006E125F02000206644F62060C6
:10948000A0800B20F2E0276630E0A1880C200029A4
:109490008FD0A17802298CD0A178252989D0BDE868
:1094A000F09F0A218AA0FFF73BFF0D20DEE0A378A2
:1094B000382B07D0A388002BF1D10028E3D02173EB
:1094C00083A0DFE00E20D1E00A2184A0FFF728FF6F
:1094D0000F20CBE0A378382B06D0A388002BDED159
:1094E00020B121737DA0CDE01020BFE06670D6E7EB
:1094F000E8030BD401217EA0FFF712FF1120B5E095
:10950000A0780B2802D0A0880028C8D14846ADE03A
:1095100003217AA0FFF704FF1320A7E0A378012B13
:1095200006D0A388002BBAD130B1217373A0A9E073
:1095300025F04000206621E045F040002066D5E798
:1095400012E00BE056E04FE092E08AE07BE074E04E
:1095500065E05EE03BE033E019E011E003216AA042
:10956000FFF7DEFE232081E0A378372B06D0A38807
:10957000002B94D110B1217363A083E0504675E0B5
:1095800062460A216EA0FFF7CBFE15206EE0A2789E
:109590003A2A0ED0A378424A3B2B126E42F48072D4
:1095A0000CD0A388002BA2D140B12173624664A0E5
:1095B00068E025F480702066162057E0226695E763
:1095C00062460A216348FFF7ABFE17204EE0A378FE
:1095D000382B07D0A388002B89D1002886D021738F
:1095E0005C484FE01E2041E00A215BA0FFF798FE97
:1095F0001F203BE0A278262A09D0A288002A84D125
:1096000000289CD0217340F6B83253A03AE01820CD
:109610002CE00A215BA0FFF783FE192026E0A27848
:10962000382A08D0A288002AA3D1002887D0217325
:109630005A4654A026E01A2018E00A215EA0FFF73F
:109640006FFE1B2012E0A278042A08D0A288002A0C
:109650008FD10028B3D021735A4657A012E01C20A6
:1096600004E00A2157A0FFF75BFE1D20607016E79B
:10967000A378052B0AD0A388002BF8D100289ED010
:10968000217350A0BDE8F05FFFF74ABEFF20EDE771
:1096900045F42040A664206666704D48A060FEE652
:1096A000381500204154480D0000000041542B5152
:1096B0004944454143540D0041542B51504F5744A8
:1096C0003D310D00100801400010014041540D00D3
:1096D000415458343B45303B0D00000041542B4968
:1096E00050523D3131353230303B26570D000000AD
:1096F00041542B43434C4B3F0D00000041542B433E
:1097000050494E3F0D00000041542B4352534D3DF4
:109710003231342C32383533392C302C302C313234
:109720002C22464646464646464646464646464617
:1097300046464646464646464646220D000000003E
:1097400041542B435245473F3B2B435245473D3104
:109750000D0000005881020841542B43545A553DD6
:10976000313B2B514E49545A3D313B2B51494E49C7
:10977000535441543B2B514D4F535441543D310DA3
:109780000000000041542B434E4D493D322C312CFA
:10979000302C302C303B2B43504D533D22534D2227
:1097A0002C22534D222C22534D223B2B434D474418
:1097B0003D312C343B0D000041542B435343413F7A
:1097C0000D00000041542B434F50533F0D0000004B
:1097D000D59700082DE9F047C14C94F90180234644
:1097E000C04E1A7B0A27501EC1B20025186E4FF4D6
:1097F0007A794FF0FF3CB8F10D0F7DD2DFE808F029
:10980000071F264BFCFBFAF9F8F7F6F5F4000121E7
:1098100021706170B449B54AC97892F89B2691428B
:109820000AD1800206D5AF4800F0D0F9206E20F4AE
:1098300000102066AEA02AE040F40010F9E74A4686
:109840000A21B1A0FFF76CFD0220FEE0A3783A2BBD
:109850000FD0A378A2483B2B006E40F4807010D04C
:10986000A388002B79D172B121734FF4FA62A6A0BC
:10987000F7E020F48070206641F28830A080032059
:10988000E3E020F01F0020666570A2A0A660BDE89E
:10989000F04715F01BB994F859000C2728B10021A6
:1098A0000846FFF733F9A2A007E094F85A0038B150
:1098B00000210120FFF72AF9A4A015F007F9E5E03F
:1098C000AA48AB49894F02784078DFF8A8A28242C3
:1098D0000FD0BAF8582050465AB997F87020012A8C
:1098E0000DD097F8BC20012A0ED04FF46162A0F889
:1098F00058208846487800E0F0E038B115E08878D4
:109900000028F6D19C4849E09C4847E015F08EFAC3
:10991000A16C97F8BA20411AA2FB0920511AA8415C
:1099200003D297F87000012807D0206EC00215D42A
:1099300098F80300C00704D014E015F077FAA0648B
:10994000E0E715F073FA216D47F23052401A00211A
:10995000101AA94106D28A4820E043E0FFF7B4F884
:1099600000283FD1874801784078814201D086485D
:1099700014E094F8210000F00F01B1EB101F01D0AA
:1099800082480BE0824801784078814201D08148CA
:1099900004E0BAF84000D04620B17F48BDE8F04767
:1099A00000F014B998F84200C00726D097F8E800F4
:1099B0000A2815D2794E7577206E20F48000206633
:1099C00015F034FA4949B0611222E8313046F8F70F
:1099D0004DFC734800F0FAF8734972483562C8616B
:1099E00088F84250BDE8F08774E068E05BE04FE043
:1099F00044E02CE023E012E00AE0A08830B1B4F8A3
:109A000060008004EED46570A660EBE704201CE0E3
:109A10004A460A2165A0FFF783FC052015E0A378DC
:109A2000062B07D0A388002BDCD12AB121734A462C
:109A30005EA016E0062008E040F020001CE04A4648
:109A400003215CA0FFF76CFC07206070CAE7A378D5
:109A5000012B0AD0A388002BC4D15AB121734A46E6
:109A600054A0BDE8F047FFF75BBC20F04000206643
:109A70000820EAE740F040002066C4E7C00305D5AF
:109A800000F016F9A4F804900920DEE76770A9E752
:109A9000A178382903D0A0880028F7D0A2E720F4C5
:109AA00080302066F2E7000406D54A46012144A032
:109AB000FFF736FC0B20C8E784F801C092E7A178D5
:109AC0000B2903D0A0880028F6D08BE720F40040B3
:109AD0002066F1E7FFF728F8012883D1657081E758
:109AE000381500203D93000868000020E415002090
:109AF00047736D20696E207374616E646279206DA6
:109B00006F64652E0D0A000041542B435245473FB8
:109B10000D00000047736D20435245472065727267
:109B20006F722C47736D20696E69740D0A00000016
:109B30006770727320726563656976656420434D52
:109B40005320646174610D0A000000006770727335
:109B500020726563656976656420503250207365B4
:109B60007276657220646174610D0A00DC1C00204D
:109B700064000020801C0020CD7E00084D9D000860
:109B800085740008A21D0020C9A70008D5A50008FB
:109B90001E1D0020D183000849A90008C01500201F
:109BA000E5510108554C0008E41D002041542B43A9
:109BB00053510D0041542B4350494E3F0D000000BE
:109BC00041542B43434C4B3F0D00000002490022FF
:109BD0004A7088607047000038150020334910B57E
:109BE00001F20A4091F80A1409075ED02F4991F852
:109BF0000A140278491E61F303020270007800071C
:109C000053D12A480146B0F8D42F01F2094091F807
:109C1000091440F22D130909244C594304EB410166
:109C2000A1F864260178037809094A1C62F3071336
:109C30000370224602F5816392F8082461F344021E
:109C40001A7001780522B2EB111F05D8214691F850
:109C5000091421F0F0010170144991F809140378F6
:109C600001F00F020021B2EB131F0ED00F4890F845
:109C7000090440F22D12000950430C4A04EB400045
:109C800000F20C40C2F8D00F0CE0084AC2F8D01F16
:109C900092F80824C2F34303044A92F8092463F3B8
:109CA000071202700148A0F8D41F10BD6005002003
:109CB0001FB50948817844790379C2788DE81E0080
:109CC0004378027805A110481CF03CFC04B00E4813
:109CD000BDE810400DF0F6BF6800002041542B4352
:109CE000434C4B3D22253032642F253032642F25E2
:109CF0003032642C253032643A253032643A2530D3
:109D000032642B3030220D006005002010B5094967
:109D100000F0DCFB044608A10648F8F7CBFA22461F
:109D200006A109481CF00EFCBDE8104006480DF0E5
:109D3000C9BF0000600500201A00000041542B43F9
:109D40004D47533D25640D009C1500202DE9F04F33
:109D5000E64C85B094F901202046E54D90F80CC002
:109D6000DFF89093ACF10100C1B228780626864650
:109D700000EBC00309EB4300BD3099F818834FF0A6
:109D8000000A4FF0130B42F21077142A73D2DFE867
:109D900002F00A10202B3A487694AED5EAFEFDFC7C
:109DA000FBFAF9F872F76420A080022020700120ED
:109DB0007EE1A08800284BD1CFA00DF083FF4FF4A7
:109DC0007A70A08099F8E500687085F800A00220FC
:109DD0006EE1A08800283BD14FF47A720321C8A01D
:109DE000FFF79EFA032063E1A2780420382ADFD02F
:109DF000A288002A2CD1BCF1000FD9D021734FF4D6
:109E00007A72BFA063E143460022C3A1C8481CF098
:109E100099FB4FF47A720321C548FFF781FA0520B8
:109E200046E1A078382812D0A088002810D1BCF1D3
:109E3000000F0CD043460022B7A1BD481CF082FBA6
:109E4000207B4FF47A72401EC1B22173DDE0667050
:109E500005B0BDE8F08F00EBC00102EB410191F8C5
:109E6000BD10502901D00A2906D207206070287839
:109E7000022808D2ECE733E1401C287000E04A4693
:109E800028780228E7D3687838B1A0F1010010F0F3
:109E9000FF00687085F800A0DAD1A64D286841015E
:109EA00006D440F080602860182100200CF0BEFB32
:109EB0004FF46160A5F858000EE1A1880029C7D1D0
:109EC00069460DF0EBFF9CA19948F8F749FA6946FD
:109ED0009748F8F7EFF999A19548F8F7EBF94FF49F
:109EE0007A7203219248FFF71BFA0820E0E0A1787C
:109EF00038291ED0A1880029AAD1BCF1000F26D094
:109F000069460DF0CBFF8CA18948F8F729FA69461C
:109F10008748F8F7CFF989A18548F8F7CBF9207B76
:109F20004FF47A72401EC1B221738148FFF7F8F9ED
:109F30008EE74EF66020A0800920B9E0A0780C28BA
:109F400009D0A0780A283ED0A088002880D16AA035
:109F50000DF0B8FE3FE04EF66020A080012009F031
:109F600059FB0A206070A0780A2831D0A08870B30D
:109F700009F02EFB0128DBD1022009F04BFB07E0A2
:109F8000ACE097E08DE050E044E030E013E006E024
:109F90000320A8700B20607069A014F097FD714831
:109FA0000178407881427AD0E870FAF7EBFCFAF752
:109FB00073FD0C20607041F2883203215C48FFF78A
:109FC000AFF90D2074E0A7800EF1010006E007E074
:109FD000022009F01FFBA7802878401C287036E774
:109FE00061A014F073FD022009F014FBAFE7A07824
:109FF0004FF4FA6241280AD0A08840B1A0784228E4
:10A0000096D1BCF1000F4AD0217349485FE0A2808D
:10A010000E204DE0A08800288AD140F6B830A080FC
:10A02000012009F0F7FA0F206070A08838B109F01C
:10A03000CFFA022810D0A0780A28C9D008E7022059
:10A0400009F0E8FA52A014F041FDA8780028CDD01C
:10A05000401EA8700C202BE056A014F037FD3549A7
:10A060000868420106D520F0806008601A210020AF
:10A070000CF0DCFA022009F0CDFA3A49EA780878C7
:10A08000904201D0401C087000F01F000870497811
:10A09000884204D00320A8700B2009E0FFE71020BD
:10A0A00006E04FF47A72022113A0FFF739F911206C
:10A0B0006070CDE6A07838280ED0A0880028BDD1E9
:10A0C000BCF1000F08D021734FF47A720AA005B0DA
:10A0D000BDE8F04FFFF724B95846E9E71220607059
:10A0E00084F801A03D48A060B2E6000038150020C9
:10A0F0002C000020E41500204154480D0000000011
:10A1000041542B5141554443483D303B2B5153461C
:10A11000523D373B0D00000041542B514D49433D0A
:10A12000302C25643B2B434C564C3D25643B0D00A5
:10A1300060050020801C0020415444003B0D0000BD
:10A14000446574656374656420416C61726D20437D
:10A15000656E7465722048616E647368616B65201A
:10A160000D0A0000DC1C0020416C61726D2043650B
:10A170006E74657220576169742048616E647368FB
:10A18000616B652054696D656F7574200D0A000060
:10A19000416C61726D2043656E7465722057616910
:10A1A0007420456E7465722054696D656F757420F6
:10A1B0000D0A0000416C61726D2043656E7465721A
:10A1C000204D6573736167652053656E6420537518
:10A1D0006363657373200D0A00000000D5970008C3
:10A1E0002DE9F047744C94F901C02046734E007B72
:10A1F0000B25411E32684FF000094FF004084FF460
:10A200007A77C9B2BCF10B0F7ED2DFE80CF00615ED
:10A2100025393C475767838DB10022F4C040306038
:10A220006420A08084F8008001206070BDE8F047C1
:10A230000021634815F096BBA0780A2809D0A088B1
:10A24000002807D13A4602215EA0FFF769F80220F4
:10A2500022E06570BDE8F087A3780322382B0DD08B
:10A26000A3780A2BF5D0A378132BF2D0A388002B68
:10A27000F0D118B121733A4652A067E06270E9E765
:10A2800084F80180E6E7A0780A28E2D03A46032164
:10A290004EA0FFF745F805206070DBE7A2780A2A98
:10A2A000D7D0A3780622382BE8D0A388002BD1D1B1
:10A2B0000028E3D021733A4644A047E0A0780A285A
:10A2C000C7D03C23062247A14C481CF03BF93A4634
:10A2D00003214A48FFF724F80720DDE7A1780A297F
:10A2E000B7D0A2780821382A12D0A288002AB1D18A
:10A2F00070B13C2306223BA140481CF023F9207B8F
:10A30000401EC1B2217300E042E03A463B481DE0E6
:10A3100061709FE7A0780A289BD03A46032138A0B5
:10A32000FEF7FEFF0920B7E7A2780A2A91D0A378AA
:10A33000224A0A25382B126842F400120AD0A38858
:10A34000002B87D168B121733A462DA0BDE8F047B4
:10A35000FEF7E6BF84F82C9005203260FCF71EFA69
:10A3600077E705203260FCF719FA84F82C9070E743
:10A37000A0780A280BD00EF0F1FB01288DD12AA07D
:10A380000DF0A0FC1D4890F80804C007FAD06570D5
:10A390000021274815F0E6FA00F062FF0520FCF7DF
:10A3A000DDF9306820F40010306015F0EFFB84F820
:10A3B00001902048A0604DE738150020801C002047
:10A3C000208102084154410D0000000041542B51EE
:10A3D00041554443483D303B2B5153494445543D3E
:10A3E000303B0D0041542B514D49433D302C2564E9
:10A3F0003B2B434C564C3D25643B0D006005002033
:10A4000041542B51544F4E454445543D342C312C2E
:10A41000332C332C36353533363B2B51544F4E4588
:10A420004445543D310D00004154480D00000000EA
:10A43000008C0208D597000870B5FEF7D1F9214DC0
:10A440000024A5F6D8702C66A0F80644A0F80444B1
:10A45000A0F8D44F00F5816190F8080420F01E00A8
:10A460000870A5F6D87101F2094091F8091421F09D
:10A470000F010170017821F0F001103101700078B6
:10A4800040F22D1100094843A5F6D87101EB4000B8
:10A4900000F20C40C1F8D00F084600F20A4190F8D3
:10A4A0000A0420F00F000870022009F0B3F86C7065
:10A4B0000548A86095F8210020F0FF0085F82100EC
:10A4C00070BD0000381500203D9300082DE9F043D1
:10A4D00005463F48ADF5017D0C468046F7F71EFF67
:10A4E0000646C00758D0701C00EBD070012101EB6C
:10A4F00060008DF8F40191208DF8F50102222146CB
:10A500007DA8FEF74FFC0746E11932464046FEF7AC
:10A5100069FE0744A81CF7F701FF804611208DF85B
:10A52000F4014FF000098DF8F5918DF8F681287847
:10A530008DF8F701E11904227DA8FEF733FCC61956
:10A54000A1194246A81CFEF74DFE06448DF8F49171
:10A5500068788DF8F501A8208DF8F601687818352F
:10A56000E0B169462846FCF75DFC0546C0F34700AC
:10A570008DF8F701A11904227DA8FEF713FC06440B
:10A58000A0196946F7F796FE7019C01B0DF5017DFD
:10A59000C0F34F00BDE8F0833046A5E72846F7F743
:10A5A000BDFE8DF8F7010422A1197DA8FEF7FAFB84
:10A5B00006442846F7F7B2FE421C69462846FEF7D5
:10A5C000F1F80246A1196846FEF7ECFB3044DCE7DF
:10A5D000451500202DE9F05F6B4C94F901C023462E
:10A5E0004FF00109187B93F82120411E09EB121747
:10A5F0000A2607F007084FF0000A4FF0060B4FF449
:10A600007A75C9B29844BCF10C0F74D2DFE80CF033
:10A61000060D17262D3A48626774829A40F6B830C4
:10A62000A08084F800B048468AE0A088002813D1B2
:10A630002A46022155A0FEF773FE022080E0A3788F
:10A640000322382B07D0A388002B05D118B1217322
:10A650002A464EA08CE06270BDE8F09F2A46022197
:10A660004DA0FEF75DFE04206AE0A3780522382B9A
:10A67000F1D0A388002BEFD10028ECD021732A461B
:10A6800045A075E098F8222047A14A481BF05AFFE0
:10A6900040F6B83202214748FEF742FE58464FE0E6
:10A6A000A178152910D0A1880029D5D180B198F8BA
:10A6B00022203DA13F481BF045FF207B40F6B832E9
:10A6C000401EC1B2217352E084F82CA0072037E06D
:10A6D0006670C1E70EF08CFE0028F9D1BCE7A088B7
:10A6E00010B1A0781128B7D1FEF794FD46F2A8105A
:10A6F000A080092024E041E0A078122805D0A078AD
:10A70000132802D0A0880028A6D1206E20F40000D3
:10A710002066DDE767F30712C2F3021060F3071249
:10A7200004EB121084F8212090F8222022A1214865
:10A730001BF008FF2A4602211E48FEF7F1FD0B2000
:10A74000607089E7A3780C21382B15D0A388002BE3
:10A7500082D188B104EB121017A190F8222015487D
:10A760001BF0F0FE207B2A46401EC1B22173114827
:10A77000BDE8F05FFEF7D4BD61706DE784F801A01D
:10A780001048A06068E700003815002041542B43B2
:10A790004D47463D300D000041542B435343533D3C
:10A7A0002255435332220D0041542B434D47523D15
:10A7B00025640D006005002041542B434D47443D66
:10A7C00025640D00D59700082DE9F047514C94F908
:10A7D00001002146DFF840910F7B504A791E504D11
:10A7E0004FF000084FF0050C4FF47A76C9B20B28F1
:10A7F00073D2DFE800F0060C16232A525D657389D8
:10A8000086006420A08084F800C0012056E0A08863
:10A8100000283ED13246022142A0FEF781FD0220EF
:10A820004CE0A2780320382A48D0A288002A30D1F0
:10A83000002F43D0217332463AA012E03246022163
:10A840003BA0FEF76DFD042038E0A2783248382A9C
:10A8500040780AD0A288002A1BD137B12173324632
:10A8600033A0BDE8F047FEF75BBD6870287085F83F
:10A87000028043E000EBC00102EB410191F8E810D7
:10A88000502901D00A2906D206206070A878042831
:10A8900006D2BDE8F087401CA870A8780428E9D348
:10A8A000297889F8001040F6B830A0800A2005E029
:10A8B0006878F9F735FC2870A68007206070E8E713
:10A8C000A08810B1A0781128E3D11D480DF0FAF945
:10A8D00046F2A810A0800820F0E715E0A078122822
:10A8E00005D0A078132802D0A0880028D1D1A8785C
:10A8F000401CA870206E20F40000206684F801C07F
:10A90000C7E7A0880028C4D184F801800D48A06062
:10A91000BFE7000038150020A21D0020E41500202C
:10A920004800002041542B434D47463D300D000068
:10A9300041542B435343533D2255435332220D0080
:10A9400060050020D59700082DE9F05F634C94F96D
:10A9500001802046DFF888B190F80CC00527ACF1E3
:10A960000100C1B20126BBF84000DFF878E15E4A81
:10A970004FF47A754FF00A0A4FF00009B8F10B0F47
:10A980006FD2DFE808F0060C16242B727F8591A6A3
:10A99000A3006420A08027706670BDE8F09FA088A7
:10A9A0000028FAD12A46022150A0FEF7B9FC022065
:10A9B0006CE0A2780320382A68D0A288002AECD163
:10A9C000BCF1000F62D021732A4648A012E02A464B
:10A9D000022149A0FEF7A4FC042057E0A378382BFD
:10A9E0000CD0A388002BD8D1BCF1000F16D0217356
:10A9F0002A4641A0BDE8F05FFEF792BC4B4682F8C4
:10AA00000190517806FA01F528420FD1491CC9B2CC
:10AA100051701029F5D30CE0137055E04B4682F8C5
:10AA20000190517806FA01F5284204D0C8B21028E6
:10AA3000F2D350462AE0491CC9B251701029F0D314
:10AA4000F7E701EBC10305EB430393F8E830502B24
:10AA500001D00A2B06D2062161701178042908D290
:10AA60009BE736E0491C117000E075461178042917
:10AA7000E7D352789640B043ABF8400040F6B83088
:10AA8000A080D6E70DF026FDA5800720607084E742
:10AA9000A08810B1A0781128E2D1FEF7BBFB46F2E6
:10AAA000A810A0800820F1E7A078122805D0A0788F
:10AAB000132802D0A0880028D2D11078401C107032
:10AAC000206E20F400002066677066E7A0880028EA
:10AAD000C6D184F801900C48A0605EE738150020CC
:10AAE000801C0020E41500203C00002041542B4332
:10AAF0004D47463D300D000041542B435343533DD9
:10AB00002255435332220D00D59700082DE9F04F0E
:10AB100091B008F023FFFE4890F80804C0F3430208
:10AB2000FB4800F20941109190F8090400F00F0071
:10AB3000824273D0F64890F8090400F00F06761CA4
:10AB4000052E00D3002640F22D1006FB00F1F04840
:10AB500000EB410505F20C4083460BF0F5FDED4C92
:10AB6000071E4FF0FF00A0704FF0000926DBDFF852
:10AB7000A883584658F82710F7F7A8FB8246F81E16
:10AB800034286FD2DFE800F03E5573906EFDFDFC77
:10AB9000B5FBFBFCFCFC6E6E6EFAF96EF8F86EF716
:10ABA000F76E6E6EF6F7F66EF76E6E6EB5F56EF4C6
:10ABB0006E6E6E6E6E6EF36E6EF2F1F03920A070F6
:10ABC000D34890F80904109966F303000870206ECA
:10ABD000400316D5D1A15846F7F778FB801C0546EF
:10ABE000CEA1F7F773FB80F800906946284610F075
:10ABF0001FFE012805D1206E20F4802020664B2006
:10AC0000A070FBE2C6A15846F7F760FB407A3128F6
:10AC100005D0352803D0302803D0B2E2F3E23A2041
:10AC20003AE2206E20F01F0040F4807020663B2046
:10AC300032E2BDA15846F7F749FB2221F7F764FB42
:10AC4000431C002001461A5C222A0CD02B2A03D078
:10AC50006718491C7A73C9B2401C80B21328F2D31A
:10AC6000042019E28CE2214481F80D90F8E7B0A1AC
:10AC70005846F7F72BFBB24F08B1B2A10AE0B3A1D7
:10AC80005846F7F723FB20B9B3A15846F7F71EFB48
:10AC900040B1B5A13846F7F763FBB64981F8F695A0
:10ACA00081F826960520F7E1B3A15846F7F70EFB89
:10ACB0008279216E303A62F304012166C079A0F1F5
:10ACC0003002092A08D801EB8103102202EB43026B
:10ACD000104460F304012166084601F01F010429B5
:10ACE00002D240F0800001E020F0800020660620C3
:10ACF000D2E1A3A15846F7F7E9FA08B1A0A100E014
:10AD0000A1A15846F7F7E2FAA1A1F7F7DFFA4178D7
:10AD10008278303901EB81016FF02F0303EB4101A1
:10AD200011449C4FC9B28E4639700179427930394D
:10AD300001EB810103EB41011144C9B279708B46EB
:10AD4000C179027A303901EB810103EB41011144F1
:10AD5000CAB2BA70817A90F80BC0303901EB810128
:10AD600003EB410161440DE0CEE1B8E196E184E1FD
:10AD700052E176E07BE161E14CE13DE1AAE0A7E050
:10AD80009CE08BE0C9B2F97090F80D8090F80EC08D
:10AD9000A8F1300808EB880803EB4808C44487F89A
:10ADA00004C090F8108090F811C0A8F1300808EBAA
:10ADB000880803EB4808C44487F805C0C77C90F8AE
:10ADC00014C0303F07EB870703EB4703807C6344E5
:10ADD000C3F387032B2802D02D281ED03CE06D4FF3
:10ADE000C818C0B2F870182836D31838F870521C3A
:10ADF000BA70594670460AF015FDB97888422BD2D0
:10AE00000121B9707878401CC0B278700C2823D921
:10AE100079703878401C38701EE05E4F994202D33A
:10AE2000C81AF87018E0C3F118000844F870012A35
:10AE300002D9521EBA700FE0BBF1010F02D9ABF17B
:10AE4000010003E0AEF1010038700C207870C1B24F
:10AE500038780AF0E7FCB8704E4810F003FB0B207E
:10AE60001AE12D494022E4316846F7F7FFF94AA17B
:10AE70005846F7F72BFA00F10B0B0027E8460222A1
:10AE800058F827105846F7F75EFA20B17F1CFFB23A
:10AE9000102FF4D375E184F82D7072E12078012829
:10AEA00008D040A00CF00EFF194890F80804C00725
:10AEB000FAD066E13D48FEF789FE62E139A00CF068
:10AEC00001FF134890F80804C007FAD00A20E3E015
:10AED0000C20E1E094F8210035A100F00F0758465E
:10AEE000F7F7F4F910F80C1F202900D1401C017865
:10AEF0003039CAB202704178A1F13003092B06D86B
:10AF000002EB8203D02202EB43021144017057E0AE
:10AF10006005002038150020B48102080D0A0000E9
:10AF20002B435245473A20002B435343413A0000FC
:10AF30004348494E41204D4F42494C4500000000D6
:10AF4000AA1B002022434D4E4554220043484E2D5B
:10AF5000554E49434F4D00004348494E4120554E00
:10AF600049434F4D0000000022554E494E455422A2
:10AF700000000000E41500202B4353513A0000006C
:10AF80002B43434C4B3A00002B514E49545A3A0044
:10AF900022000000680000202B51544F4E454445CC
:10AFA000543A20004154480D00000000E1A100087F
:10AFB0002B434D54493A2022534D222C00000000CF
:10AFC0007F1C94F8212007F00701B1EB121F0AD073
:10AFD0006218007882F8220094F8210061F30300DF
:10AFE00084F82100CDE0027888A18B481BF0AAFAF2
:10AFF00089480CF067FEC4E05846D8F85410F7F7BB
:10B0000065F9AFF2E801F7F761F9801CFEF708F97E
:10B01000152041E018203FE008F1A807584639689C
:10B02000F7F754F980463868F7F778F910F8080010
:10B03000352801D042202FE041202DE0AFF224112D
:10B040005846F7F743F98078A0F1300105290CD86C
:10B05000302802D0312804D007E0206E20F4804050
:10B0600002E0206E20F4801020661A2014E0206E8A
:10B0700020F4804040F40030F4E768A15846F7F728
:10B0800025F92C21F7F740F9401C2C21F7F73CF962
:10B090008078302875D14A20A07072E0002762A124
:10B0A0005846F7F713F98346AFF29011F7F70EF908
:10B0B000804680F800905FA15846F7F707F908B17D
:10B0C000022000E00120E1197F1CFFB281F854004A
:10B0D00008F1010B052FE2D38AF8009051E058A146
:10B0E0005846F7F7F3F82C21F7F70EF9401C2C21FE
:10B0F000F7F70AF94078A0F13001052941D8534902
:10B10000425C521C42543CE04FF0000850A15846AB
:10B11000F7F7DCF850B12C21F7F7F6F8401C2C219A
:10B12000F7F7F2F8401C4FF6FF730EE03A48C0F80C
:10B130004090C0F8449024E008EB880203EA420201
:10B14000303A11441FFA81F8401C0178A1F1300215
:10B15000092AF1D9B8F5067F0BD8AFF24021F7F7ED
:10B16000B5F8811C05D02C4842464030F7F77EF8F0
:10B1700004E02948C0F84090C0F844908AF8009054
:10B18000A77035A15046F7F7A1F860B132A150463B
:10B19000F7F79CF810F8041F4F2904D141784B2988
:10B1A00001D100F1020A2CA15046F7F78FF8F0B157
:10B1B00029A15046F7F78AF8811CB5F864064B1BA5
:10B1C00040F26462C01A00F20C405053002006E0C6
:10B1D0002B1811F8012B401C83F80C2480B2B5F811
:10B1E00064268242F4D8284480F80C9406E00A4889
:10B1F00090F80904109966F30300087094F90200AE
:10B2000011B0BDE8F08F3920FAE7000041542B431C
:10B210004D47443D25640D00600500202B514953E6
:10B2200041434B3A200000002B51495354415445AF
:10B230003A200000434F4E4E454354454400000021
:10B240002B51495244493A2000000000611500206A
:10B250002B514952443A20000D0A0D0A000000000B
:10B2600010B50120FBF77AFA0849094A086820F46A
:10B27000801008604FF48051116010F4F01F04D169
:10B28000BDE810400020FBF769BA10BD801C00200B
:10B290001408014010B50020FBF780FA0420FBF7EA
:10B2A0005DFA0520FBF75AFA0849082008600848AB
:10B2B000016841F48011016006494FF48050086034
:10B2C000BDE810400120FBF769BA0000140C0140F2
:10B2D000801C00201008014070B5184C0D46064631
:10B2E00004F23B31F7F721F828B904F24B31284634
:10B2F000F7F71BF8A0B1124890F8570048B111A118
:10B300003046F7F712F820B910A12846F7F70DF8E4
:10B3100030B104F21B313046F7F707F858B901E0B5
:10B32000802070BD04F22B312846F6F7FEFF00287E
:10B3300004BF812070BD002070BD0000E415002016
:10B34000801C002061646D696E0000003030303078
:10B3500030300000F0B5AF4CAF4D85B020781422EE
:10B3600000EB800101EBC00005EB80106946007E18
:10B370000AF0D4FFA948007848B1022800F0808084
:10B38000A7A090E80E108DE80E10006904900D2221
:10B39000A6A16846F6F7D7FF002800F079800C22B6
:10B3A000A6A16846F6F7CFFF002800F075800F22AF
:10B3B000A6A16846F6F7C7FF002873D00B22A7A105
:10B3C0006846F6F7C0FF002870D00A22A6A168469A
:10B3D000F6F7B9FF00286DD00D22A6A16846F6F752
:10B3E000B2FF00286AD00C22A6A16846F6F7ABFF90
:10B3F000002867D00822A7A16846F6F7A4FF002816
:10B4000064D00822A6A16846F6F79DFF002861D007
:10B410000D22A6A16846F6F796FF00285ED00A2204
:10B420007FA16846F6F78FFF002800F0DF800A2230
:10B43000A2A16846F6F787FF002800F0DB800D2206
:10B44000A1A16846F6F77FFF00287CD00922A2A1BF
:10B450006846F6F778FF002876D00922A1A1684651
:10B46000F6F771FF002870D00922A1A16846F6F70F
:10B470006AFF002814BF002002F076F805B0F0BD86
:10B480008EA090E80E108DE80E10006904907EE703
:10B4900001F03CFF05B0F0BD01F004FA05B0F0BDCD
:10B4A00000E003E000F016FA05B0F0BD00F0E8FFA0
:10B4B00005B0F0BD02F0DCF905B0F0BD03F016F9FF
:10B4C00005B0F0BD03F0FCFA05B0F0BD03F05EFD81
:10B4D00005B0F0BD01F096FB05B0F0BD874E2078B9
:10B4E00006EB4000407812F0D9F90746207806EBC9
:10B4F0004000407811F018FF3918207800EB8002E6
:10B5000002EBC00205EB82121268914253D306EBA4
:10B510004000407812F0C2F9217801EB810202EB81
:10B52000C10105EB8111096888423EBF012005B0C9
:10B53000F0BD002918BF724E3DD0207800EB80018D
:10B5400001EBC00002E059E05CE05FE005EB801039
:10B550001E30102107F0F0F868BB207800EB800166
:10B5600001EBC00005EB80102E3040F20E3107F0E9
:10B57000F3F800BB207800EB800101EBC00005EB85
:10B5800080101E305FA1F6F7D0FE50B9207800EB96
:10B59000800101EBC00005EB80102E301CF0CDFBCC
:10B5A0003070207800EB800101EBC00005EB8010CB
:10B5B00000680028C1D1207800EB800101EBC000B9
:10B5C00052A105EB80100A68C0F81E204A68C0F836
:10B5D00022208A68C0F8262089894185002180F8C8
:10B5E0002C100821017705B00020F0BD02F034FED8
:10B5F00005B0F0BD01F0D2FC05B0F0BD00F00CFCD0
:10B6000005B0F0BD00F0B8FD05B0F0BD02F0A8FB3C
:10B6100005B0F0BD5401002010240020D801002006
:10B620005570646174652E68746D000052656D6FAD
:10B6300074654374722E68746D00000050617373FA
:10B64000776F72642E68746D00000000416C617247
:10B650006D43656E7465722E68746D004E65747707
:10B660006F726B2E68746D004F7074696F6E2E6808
:10B67000746D00005573657250686F6E652E687446
:10B680006D000000576972656C6573732E68746D88
:10B69000000000005A6F6E652E68746D0000000097
:10B6A000524649442E68746D00000000537973744B
:10B6B000656D4C6F672E68746D0000005265626F97
:10B6C0006F742E68746D0000416C61726D45766513
:10B6D0006E742E68746D0000456D61696C2E68741F
:10B6E0006D00000054696D65722E68746D00000075
:10B6F000536D6172742E68746D0000005501002056
:10B70000EE01002067657450616765002F537973FF
:10B7100074656D4C6F672E68746D00002DE9F04301
:10B720008DB02E4FDFF8B880387800EB800101EB48
:10B73000C00108EB8111C97E11F0800F4AD17E1C37
:10B7400006EB400006224078002111F051FD4FF039
:10B750000009CDF80090CDF8049038784B4606EB00
:10B760004000022240781F4911F0CEFBC01C00F0BF
:10B77000FC04242C00D3242402AD94B13878042294
:10B7800006EB40002946407811F032FD03232A469B
:10B7900004212846F8F78EFE201F84B2ED1C002CF1
:10B7A000ECD185F8009002A801783A2904D0611CF8
:10B7B0008CB2401C282CF7D380F80090411C02A8C2
:10B7C000FFF78AFD397801EB810202EBC10108EB3A
:10B7D0008111C8760DB0BDE8F0830000540100204F
:10B7E000102400207CA80208F0B585B0194D002473
:10B7F0006F1E009401943878234605EB4000022226
:10B800004078154911F080FB0246144E0A2A0BD3EA
:10B810003878022100EB800202EBC00006EB8010BA
:10B820000177046005B0F0BD387802A905EB40004F
:10B83000407811F0DDFC02A90C5402A8F6F7DEFDF9
:10B84000397801EB810202EBC10106EB811108603E
:10B8500005B0F0BD550100207CA80208102400208E
:10B86000012803D0022803D1FFF7BEBFFFF756BF60
:10B87000704700002DE9F041124C00252570661C30
:10B88000DFF84480FF27207806F810500F48002189
:10B890000823B0F85826084612F04CF8217806EB39
:10B8A0004102507001EB810000EBC10008EB8010F9
:10B8B00007764776481CC0B220700228E3D3257073
:10B8C000BDE8F0815401002010240020E415002080
:10B8D000002070472DE9F04FFC4FFB4E00253878D3
:10B8E00087B006EB40002C46407811F0D7FF804629
:10B8F000387806EB4000407811F016FD08EB0001A7
:10B900003878DFF8CC8300EB800202EBC00208EB52
:10B9100082124FF001091268AA469142C0F040829B
:10B9200006EB4000407811F0B9FF397801EB810255
:10B9300002EBC10108EB8111096888423EBF01207A
:10B9400007B0BDE8F08F4FF0020B002918BFE14EA1
:10B9500000F02A82387800EB800101EBC00008EB90
:10B9600080101E30102106F0E7FE002840F01882FB
:10B97000387800EB800101EBC00008EB80102E301E
:10B9800040F20E3106F0E8FE002840F009823878D7
:10B9900000EB800101EBC00008EB80101E30CEA14F
:10B9A000F6F7C3FC0028387800EB800101EBC000FB
:10B9B00008EB80107DD01E30CAA1F6F7B6FC002837
:10B9C000387800EB800101EBC00008EB801071D0EB
:10B9D0001E30C7A1F6F7A9FC0028387800EB8001DB
:10B9E00001EBC00008EB801065D01E30C4A1F6F753
:10B9F0009CFC0028387800EB800101EBC00008EBCC
:10BA0000801071D01E30C2A1F6F78FFC0028387864
:10BA100000EB800101EBC00008EB801071D01E30FC
:10BA2000BEA1F6F782FC0028387800EB800101EB1C
:10BA3000C00008EB80107CD01E30BBA1F6F775FC6F
:10BA40000028387800EB800101EBC00008EB801083
:10BA500070D01E30B7A1F6F768FC0028387800EBEC
:10BA6000800101EBC00008EB801000F0F5801E3073
:10BA7000B3A1F6F75AFC0028387800EB800101EBFF
:10BA8000C00008EB801000F0F3801E30AEA1F6F786
:10BA90004CFC0028387800EB800101EBC00008EB7B
:10BAA000801000F0FB801E30A9A1F6F73EFC0028B4
:10BAB00002E005E019E02BE000F0508100F061B9F0
:10BAC00090F82E00312896F8BC0006D002281CBF42
:10BAD000012486F8BCB000F054B901281CBF012431
:10BAE00086F8BC9000F04DB935E090F82E00312872
:10BAF00096F8700006D002281CBF012486F870B0AA
:10BB00003FE147E001281CBF012486F8709038E12E
:10BB100000F12E0168461CF024F900285ED006F1E1
:10BB2000BD0168461BF0BEFE002842D101240098EA
:10BB300001E03FE054E0C6F8BD000198C6F8C1003E
:10BB40000298C6F8C5000398C6F8C900BDF81000F1
:10BB5000A6F8CD0015E100F12E0168461CF001F9B0
:10BB6000D8B306F1CF0168461BF09CFE002820D117
:10BB70000098C6F8CF000198C6F8D3000298C6F81E
:10BB8000D7000398C6F8DB00BDF810000124A6F822
:10BB9000DF00F6E02E301CF0D0F8411E8DF80000DA
:10BBA0000F291BD296F8E51081421CBF012486F8AC
:10BBB000E500E6E000F12E0168461CF051F860B1A6
:10BBC0000422694606F1E100F6F7BDFB00284ED0DD
:10BBD00000980124C6F8E100D3E0FFE70125D0E09A
:10BBE0002E3005A90FF024FE01280DD0387800EB87
:10BBF000800101EBC00008EB80102E3006F17501CA
:10BC0000F6F793FB98B116E0042205A906F171003E
:10BC1000F6F799FB10B996F8BB0040BB86F8BB90CD
:10BC20000598C6F87100012486F875A0A9E096F879
:10BC3000BB0001281BD186F8BBA0C6F871A03878DC
:10BC4000012400EB800101EBC00008EB801000F143
:10BC50002E0106F1750034E02E30F6F7C2FBB6F87F
:10BC6000A61080B281421CBFA6F8A600012488E07D
:10BC700000F12E0106F1A800F6F757FB18B338784B
:10BC8000012400EB800101EBC00008EB801000F103
:10BC90002E0106F1A800F6F763FB72E000F12E0119
:10BCA00006F1B100F6F741FB68B13878012400EBEA
:10BCB000800101EBC00008EB801000F12E0106F1BD
:10BCC000B100F6F74DFB5CE0550100205401002067
:10BCD00010240020E415002050686F6E65456E61E9
:10BCE000626C65005443504950456E61626C65005A
:10BCF00043656E74657250686F6E653100000000B8
:10BD000043656E74657250686F6E653200000000A6
:10BD100043656E746572436E7400000043656E7413
:10BD2000657249440000000043656E7465724950B5
:10BD30000000000043656E746572506F72740000FD
:10BD40004C6F674E616D65004C6F67507377640090
:10BD500050756C736554696D65000000387800EBB0
:10BD6000800101EBC00008EB80102E301BF0E5FFD6
:10BD70008DF8000096F8BA1081421CBF012486F8A5
:10BD8000BA00387800EB800101EBC00008EB8010AE
:10BD9000006800287FF4DEAD012D01D025B106E05A
:10BDA000164880F80E9002E0144880F80EB0012C7E
:10BDB00007D100200EF0A0FE40F29C6110480EF06A
:10BDC00091FF387800EB800101EBC0000DA108EB7A
:10BDD00080100A68C0F81E204A68C0F822208A68CD
:10BDE000C0F82620C968C0F82A1080F82EA00821C3
:10BDF000017707B00020BDE8F08F0000D8010020D7
:10BE0000E41500202F416C61726D43656E7465729C
:10BE10002E68746D000000002DE9F05FBF4FBE4E2C
:10BE2000002538782C4606EB4000407811F036FDAE
:10BE30008046387806EB4000407811F075FA08EB40
:10BE400000013878DFF8D88200EB800202EBC002F4
:10BE500008EB821212689142C0F0338106EB400079
:10BE6000407811F01BFD397801EB810202EBC10132
:10BE700008EB8111096888423CBF0120BDE8F09FB2
:10BE8000002900F02281DFF89C92DFF89CA209F2E1
:10BE9000E2264FF0220B387800EB800101EBC00066
:10BEA00008EB80101E30102106F046FC002840F000
:10BEB0000881387800EB800101EBC00008EB8010AE
:10BEC0002E3040F20E3106F047FC002840F0F98099
:10BED000387800EB800101EBC00008EB80101E30C9
:10BEE00092A1F6F722FA0028387800EB800101EBE6
:10BEF000C00008EB80102DD01E308FA1F6F715FA88
:10BF00000028387800EB800101EBC00008EB8010BE
:10BF100026D01E308AA1F6F708FA0028387800EB00
:10BF2000800101EBC00008EB80104FD01E3085A1CE
:10BF3000F6F7FBF90028387800EB800101EBC00030
:10BF400008EB801064D01E3080A1F6F7EEF90028CF
:10BF50007ED0A7E02E301BF0F0FE8AF80000A1E0B2
:10BF60002E307DA1F6F7E1F9002816BF9AF80000FF
:10BF7000022500284BD0387800EB800101EBC0008F
:10BF800008EB80102E301BF0D8FE9AF800108A5D66
:10BF900082423CD0012488550A291CBF0B290C2958
:10BFA00035D199F8EB0210F0010F0BD199F8EC02A2
:10BFB00010F0010F06D199F8ED0210F0010F08BF43
:10BFC000022000D0012089F837016BE000F82DBF76
:10BFD00063A1F6F76FF9387800EB800101EBC00040
:10BFE00008EB80102D3009F2C651F6F79EF90028B3
:10BFF00058D0387800EB800101EBC00008EB8010CE
:10C0000000F12D0109F2C650F6F7AAF9012449E022
:10C0100000F82DBF52A1F6F74DF9387800EB8001FA
:10C0200001EBC00008EB80102D3009F2F651F6F755
:10C030007CF9B8B3387800EB800101EBC00008EB65
:10C04000801000F12D0109F2F650F6F789F900E0B1
:10C0500001E0012426E0387800EB800101EBC0000C
:10C0600008EB80103EA100F82DBFF6F723F93878D1
:10C0700000EB800101EBC00008EB80102D3009F2CD
:10C080002661F6F752F968B1387800EB800101EBD0
:10C09000C00008EB801000F12D0109F22660F6F7D0
:10C0A0005FF90124387800EB800101EBC00008EB58
:10C0B0008010006800287FF4EEAE012D01D025B17C
:10C0C00006E028490120887302E02649022088738F
:10C0D000012C07D100200EF00FFD40F29C611148A9
:10C0E0000EF000FE387800EB800101EBC0001EA1CD
:10C0F00008EB80100A68C0F81E204A68C0F82220A9
:10C100008A68C0F82620C968C0F82A10082101777B
:10C110000020BDE8F09F00005501002054010020E0
:10C1200010240020E4150020EE01002053656C650A
:10C1300063744576656E7400626F785F706172003B
:10C1400061706E007573657200000000706173733A
:10C15000776F7264000000004765745061720000E0
:10C1600022000000D80100202F416C61726D4576DD
:10C17000656E742E68746D002DE9F047AE4DAD4FBD
:10C180004FF000082878444607EB4000407811F053
:10C1900085FB0646287807EB4000407811F0C4F88C
:10C1A00031182878A54E00EB800202EBC00206EBA6
:10C1B0008212DFF88C9212689142C0F0138107EB73
:10C1C0004000407811F06AFB297801EB810202EB14
:10C1D000C10106EB8111096888423CBF0120BDE81E
:10C1E000F087002918BF974F00F0FE80287800EBF9
:10C1F000800101EBC00006EB80101E30102106F01C
:10C200009BFA002840F0EE80287800EB800101EBDB
:10C21000C00006EB80102E3040F20E3106F09CFA82
:10C22000002840F0DF80287800EB800101EBC0009F
:10C2300006EB80101E3084A1F6F777F800282878E6
:10C2400000EB800101EBC00006EB80103AD01E30FD
:10C250007FA1F6F76AF80028287800EB800101EB4F
:10C26000C00006EB801044D01E307BA1F6F75DF8CD
:10C270000028287800EB800101EBC00006EB80105D
:10C2800045D01E3076A1F6F750F80028287800EB4C
:10C29000800101EBC00006EB80104CD01E3072A173
:10C2A000F6F743F80028287800EB800101EBC00086
:10C2B00006EB801055D01E306DA1F6F736F8002839
:10C2C00063D07DE000F12E0107F29C40F6F72DF8D7
:10C2D000002875D02878012400EB800101EBC00014
:10C2E00006EB801000F12E0107F29C40F6F738F8BB
:10C2F00066E02E30F6F775F8524980B2B1F8CC14EA
:10C3000081425DD04F490124A1F8CC0458E000F1EE
:10C310002E0107F2CE40F6F708F808B3287801247A
:10C3200000EB800101EBC00006EB801000F12E0154
:10C3300007F2CE4012E000F12E0107F2FE40F5F7C1
:10C34000F4FF68B12878012400EB800101EBC00004
:10C3500006EB801000F12E0107F2FE40F6F700F820
:10C360002EE000F12E0107F21650F5F7DEFF38B38C
:10C370002878012400EB800101EBC00006EB80105F
:10C3800000F12E0107F21650E8E7287800EB800153
:10C3900001EBC00006EB801000F12E0107F24650C1
:10C3A000F5F7C3FF60B12878012400EB800101EBB1
:10C3B000C00006EB801000F12E0107F24650CDE7D9
:10C3C000287800EB800101EBC00006EB80100068CC
:10C3D00000287FF40BAFB8F1010F03D0B8F1000FC4
:10C3E00002D004E0012000E0022089F80E00012CB8
:10C3F00007D100200EF080FB40F29C6111480EF046
:10C4000071FC287800EB800101EBC00019A106EB5C
:10C4100080100A68C0F81E204A68C0F822200989E6
:10C42000C184002180F82810082101770020BDE890
:10C43000F087000055010020540100201024002046
:10C44000D8010020E4150020736572766572000043
:10C45000706F727400000000757365720000000058
:10C46000706173730000000066726F6D0000000061
:10C47000746F00002F456D61696C2E68746D00004B
:10C480002DE9F04FF14FF04C4FF0000A387883B0AF
:10C4900004EB40005546407811F000FA0646387823
:10C4A00004EB4000407810F03FFF31183878DFF897
:10C4B000A08300EB800202EBC00208EB821212683C
:10C4C0009142C0F0968104EB4000407811F0E6F90B
:10C4D000397801EB810202EBC10108EB8111096897
:10C4E00088423EBF012003B0BDE8F08F002900F074
:10C4F0008481D84E4FF0300BE946387800EB80014C
:10C5000001EBC00008EB80101E30102106F014F97A
:10C51000002840F06E81387800EB800101EBC0000C
:10C5200008EB80102E3040F20E3106F015F900288D
:10C5300040F05F81387800EB800101EBC00008EB30
:10C5400080101E30C4A1F5F7F0FE0028387800EB0B
:10C55000800101EBC00056D008EB80101E30BFA157
:10C56000F5F7E3FE0028387800EB800101EBC0000E
:10C5700008EB80107ED01E30BAA1F5F7D6FE002859
:10C58000387800EB800101EBC00008EB801072D01E
:10C590001E30B5A1F5F7C9FE0028387800EB800100
:10C5A00001EBC00008EB801067D01E30B0A1F5F79A
:10C5B000BCFE0028387800EB800101EBC00008EBDE
:10C5C000801070D01E30ACA1F5F7AFFE002838788F
:10C5D00000EB800101EBC00008EB80107ED01E3024
:10C5E000A7A1F5F7A2FE0028387800EB800101EB47
:10C5F000C00008EB801072D01E30A3A1F5F795FEA5
:10C6000000286DD0E3E008EB801303F12E01002039
:10C610000A788AB3A2F1300CBCF10A0F24BFA2F150
:10C62000410CBCF1060F06D3A2F1610CBCF1060F60
:10C6300041F10001ECD203EB000C401C491CC0B2DC
:10C640008CF81E200C28E3D30024387800EB8001FE
:10C6500001EBC00008EB801000EB4400817F8DF8F7
:10C660000910C07F8DF8080002981AF0D3FF09F86E
:10C67000040003E022E051E016E061E0601CC4B277
:10C68000062CE2D3062206F16A016846F5F75BFE46
:10C69000002842D00099C6F86A10BDF804100125A0
:10C6A000A6F86E1093E05DE00C28CDD21918401C5E
:10C6B000C0B281F81EB00C28F8D3C5E72E30FAF7C7
:10C6C0001CFB3878102200EB800101EBC00008EB66
:10C6D000801000F12E0106F15A0002E04DE057E013
:10C6E00061E0F5F730FE002871D03878012500EBC5
:10C6F000800101EBC00008EB8010D0F82E10C6F8C6
:10C700005A10D0F83210C6F85E10D0F83610C6F8BD
:10C710006210D0F83A00C6F8660058E02E3069463C
:10C720000FF086F8012864D1042206F1460168461C
:10C73000F5F709FE00B300980125C6F8460046E06B
:10C740002E3069460FF074F8012852D1042206F108
:10C750004E016846F5F7F7FD70B100980125C6F85F
:10C760004E0034E02E3069460FF062F8012840D1C7
:10C7700000980125C6F84A0029E02E3069460FF0DE
:10C7800057F8012835D100980125C6F852001EE05F
:10C790002E3069460FF04CF801282AD10098012567
:10C7A000C6F8560013E0387800EB800101EBC000BA
:10C7B00008EB80102E30F5F714FE264980B2B1F850
:10C7C0005816814203D023490125A1F8580638782C
:10C7D00000EB800101EBC00008EB8010006800282E
:10C7E0007FF48BAEBAF1010F03D0BAF1000F04D081
:10C7F00006E027480121817302E025480221817368
:10C80000012D07D100200EF077F940F29C6111480C
:10C810000EF068FA387800EB800101EBC0001DA132
:10C8200008EB80100A68C0F81E204A68C0F8222071
:10C830008968C0F82610002180F82A1008210177A5
:10C8400003B00020BDE8F08F550100205401002006
:10C8500010240020E41500206D6163006E616D6599
:10C8600000000000697000006761746577617900FD
:10C870006D61736B00000000646E73310000000096
:10C88000646E733200000000776562506F7274004E
:10C89000D80100202F4E6574776F726B2E68746D0F
:10C8A000000000002DE9F84FBC4EDFF8EC820025B7
:10C8B00030782C4608EB4000407810F0EFFF074638
:10C8C000307808EB4000407810F02EFD39183078B1
:10C8D000B34F00EB800202EBC00207EB8212DFF8DD
:10C8E000C4A212689142C0F02F8108EB400040784A
:10C8F00010F0D4FF317801EB810202EBC10107EBAC
:10C900008111096888423CBF0120BDE8F88F0029E9
:10C910001CBFDFF89482DFF8949200F01781307822
:10C9200000EB800101EBC00007EB80101E301021EE
:10C9300005F002FF002840F00781307800EB80010D
:10C9400001EBC00007EB80102E3040F20E3105F0F5
:10C9500003FF002840F0F880307800EB800101EB05
:10C96000C00007EB80101E3091A1F5F7DEFC002817
:10C97000307800EB800101EBC00007EB80103AD06B
:10C980001E308DA1F5F7D1FC0028307800EB800136
:10C9900001EBC00007EB801042D01E3088A1F5F7F4
:10C9A000C4FC0028307800EB800101EBC00007EBED
:10C9B00080104CD01E3085A1F5F7B7FC00283078E8
:10C9C00000EB800101EBC00007EB801054D01E305B
:10C9D00081A1F5F7AAFC0028307800EB800101EB7B
:10C9E000C00007EB80105CD01E307DA1F5F79DFCE8
:10C9F00000285CD099E000F12E0108F23B30F5F7F9
:10CA000094FC002852D03078012400EB800101EB27
:10CA1000C00007EB801000F12E0108F23B3013E05C
:10CA200000F12E0108F24B30F5F77FFC00287CD096
:10CA30003078012400EB800101EBC00007EB80108F
:10CA400000F12E0108F24B30F5F78AFC6DE000F1A1
:10CA50002E0108F21B30F5F768FC002865D030780D
:10CA6000012400EB800101EBC00007EB801000F116
:10CA70002E0108F21B30E7E700F12E0108F22B30FF
:10CA8000F5F753FC002850D03078012400EB8001EA
:10CA900001EBC00007EB801000F12E0108F22B30F3
:10CAA000D2E72E301BF049F989F800003DE03078DC
:10CAB000062200EB800101EBC00007EB80102E3056
:10CAC0004AA1F5F740FC002816BF99F8000002259E
:10CAD00000282AD0317808EB800001EB810202EBBC
:10CAE000C10107EB8111801C91F82E20303A8DF89E
:10CAF000002091F82F20303A8DF8012091F8302055
:10CB0000303A8DF8022091F83110042230398DF836
:10CB100003106946F5F717FC38B199F80000009941
:10CB200008EB80000124C0F80210307800EB80018F
:10CB300001EBC00007EB8010006800287FF4EFAE27
:10CB4000012D01D015B104E0012000E002208AF897
:10CB50000E00012C07D100200DF0CEFF40F29C61A9
:10CB600011480EF0BFF8307800EB800101EBC000F7
:10CB700020A107EB80100A68C0F81E204A68C0F8A0
:10CB800022208A68C0F826208989418508210177FA
:10CB90000020BDE8F88F000055010020540100205E
:10CBA00010240020D8010020E4150020EE01002010
:10CBB00041646D4E616D650041646D507377640032
:10CBC0004D61737465724E616D6500004D617374E3
:10CBD000657250737764000073656C5573657200FD
:10CBE0005573657250737764000000004765745098
:10CBF000617200002F50617373776F72642E6874D6
:10CC00006D0000002DE9F05FCE4DCF4EDFF83C9374
:10CC10002878022700EB800101EBC00006EB8010B2
:10CC2000012490F83E134FF0040B4FF00008A9F1D7
:10CC3000160A062980F08281DFE801F0030A34E554
:10CC4000FDFC80F83E43C24880F8008000F045B902
:10CC50001E30102105F070FD022800F04181287877
:10CC600000EB800101EBC00006EB80101E30B9A183
:10CC7000F5F75BFB50B1287800EB800101EBC000B9
:10CC800006EB801080F83E7300F027B92878032166
:10CC900000EB800202EBC00006EB801080F83E1330
:10CCA00000F01BB92E3040F20E3105F055FD022880
:10CCB00000F01681287800EB800101EBC00006EB44
:10CCC0008010A7A180F83E431E30F5F72EFB002808
:10CCD000287800EB800101EBC00006EB801021D02A
:10CCE0001E30A1A1F5F721FB00282878A04F00EB0A
:10CCF000800101EBC00006EB801022D01E309DA108
:10CD0000F5F713FB002850D0287800EB800101EBE9
:10CD1000C00006EB80100168002908BF80F83EB310
:10CD200000F0DBB82E301BF008F889F800002878F6
:10CD300000EB800101EBC00006EB801080F83E4361
:10CD4000CBE02E308EA1F5F7F0FAA8B199F80000EB
:10CD5000002849D0287800EB800101EBC00006EBE9
:10CD600080102E30F5F74AFB99F8001007EB81028E
:10CD7000C2F8F40158B1B0E02878052100EB800238
:10CD800002EBC00006EB801080F83E13A5E0481EC1
:10CD900007EBE00100F0070091F8F62104FA00F03B
:10CDA00022EA000081F8F60197E099F800000028D7
:10CDB0001AD0297801EB810202EBC10106EB811147
:10CDC00091F82E10302910D0421E07EBE20302F03A
:10CDD000070293F8F6C104FA02F24CEA020283F861
:10CDE000F621694A3039815477E0401E07EBE001B3
:10CDF00000F0070091F8F62104FA00F022EA0000A2
:10CE000081F8F60169E00068002818BF5F4F52D032
:10CE1000287807EB4000407810F040FD04005FD018
:10CE2000B4F5477F88BF4FF447742246287800EB5B
:10CE3000800101E06DE062E001EBC00107EB400022
:10CE400006EB81112031407810F0D2F9297801EBFE
:10CE5000810202EBC10106EB81110A68101A0A195E
:10CE60000860D07F25283ED0907F25281CBF82F8FF
:10CE7000208000203CD09AF80920002A08BF01F148
:10CE8000200405D0012A0CBF01F11F0401F11E048A
:10CE90008AF80900204605F04DFE21462C48F5F79A
:10CEA00009FA287800EB800101EBC00006EB801046
:10CEB00000680028ACD18AF8098099F8000024495C
:10CEC000401EC0B20BF074FB287800EB800101EB30
:10CED000C00006EB801080F83EB30220BDE8F09F52
:10CEE0000120BDE8F09FC877012082F81F80C2E7CB
:10CEF0008877D07FC877022082F81E80BBE78AF847
:10CF00000E7000200DF0F8FD40F29C6118480DF005
:10CF1000E9FE287800EB800101EBC0001CA106EBC4
:10CF200080100A68C0F81E204A68C0F822200989CB
:10CF3000C184082101770020BDE8F09F0020BDE8F2
:10CF4000F09F00005401002010240020EE0100207A
:10CF5000345B0020524649445F4D73670000000077
:10CF6000526669644E6F0000436F64650000000004
:10CF7000E415002046756E6374696F6E0000000052
:10CF80004765745061720000B618002055010020FA
:10CF90002F524649442E68746D0000002DE9F04F71
:10CFA000CC4FDFF8348300263878CC4D00EB80017D
:10CFB00001EBC00108EB8111DFF8249391F83E23C7
:10CFC000C1B034464FF0010B4FF6FF7A9AB1012AF7
:10CFD00050D0022A71D0C3A089F80EB00268C1F8FF
:10CFE0001E204268C1F822208068C1F8260008206F
:10CFF000087700F06AB905EB40000094019440788E
:10D0000000230622BAA10FF07FFF504500F0CD802B
:10D01000022089F80000C9F81C4000940194387877
:10D02000002305EB400002224078B3A10FF06CFF13
:10D03000504500F0BA80397801EB810202EBC10261
:10D0400008EB821213681B1A9B1F801C136082B2AC
:10D0500005EB41000021407810F0CAF8397801EB67
:10D06000810202EBC10108EB81110A68101A086005
:10D0700081F83EB3009401943878002305EB40001A
:10D08000042240789DA10FF03FFF50454FD0001D76
:10D0900082B23878002105EB4000407810F0A8F803
:10D0A000397801EB810202EBC10108EB81110A68BA
:10D0B000101A0860022081F83E03387805EB400022
:10D0C000407810F0EBFB0446387800EB800101EB70
:10D0D000C00008EB80100168A14238BF0C4649F23D
:10D0E0008000814288BF0126002C55D0802C34BF9F
:10D0F0002046802082B23878784B00EB800101EB2B
:10D10000C00103EB400008EB81111E31407810F0A4
:10D110006FF80546387800EB800101EBC00008EBA2
:10D1200080100168491B641B01609EBB1CE03878BD
:10D1300005EB4000407810F0B1FB001F82B2387858
:10D14000002105EB4000407810F052F8397801EBEF
:10D15000810202EBC10108EB81110A68101A086014
:10D1600041B00120BDE8F08FD9F81C0000F5801017
:10D170000DF0C2FC387800EB800101EBC00008EB39
:10D1800080101E3029460DF0ADFDD9F81C00284452
:10D19000C9F81C00002CA9D1387800EB800101EB04
:10D1A000C00008EB8010006818B141B00120BDE854
:10D1B000F08F80220126694650030DF01BFD9DF87B
:10D1C0000000562804BF9DF802002E285FD14AA116
:10D1D0006846F5F77BF800281CBF801C002156D05C
:10D1E00003782201412B34BF303A373A9C18491C4E
:10D1F000401CC9B2082924BF00252946F0D3037872
:10D200000AEA0512412B34BF303A373A1A4401F189
:10D210000101C9B295B200F101000429EFD3A2B215
:10D22000384939480DF0E6FC21463648F7F76AFCE4
:10D23000A84226D1002630460DF05EFC40F29C61EB
:10D2400030480DF04FFD06F089FB4FF4005448F6CE
:10D25000FF7504F580104FF48072694680300DF040
:10D26000C9FC20460DF048FC4FF4807168460DF073
:10D2700039FD04F58074AC42EBD306F06FFB0BF084
:10D2800087FB002E04BF022089F80E0007D089F822
:10D290000EB040F29C621B4900200DF0ABFC3878C8
:10D2A000032100EB800202EBC00008EB801080F845
:10D2B0003E130CA10A684B688968C0F81E20C0F8AC
:10D2C0002230C0F826100821017741B00020BDE8C7
:10D2D000F08F000054010020102400205501002090
:10D2E000D80100202F5265626F6F742E68746D0034
:10D2F000436F6E66696700000D0A00000D0A0D0A93
:10D3000000000000E4150020800010002DE9F04727
:10D31000844E834D0024307805EB4000407810F0B7
:10D32000BDFA0746307805EB400040780FF0FCFF6F
:10D33000391830787C4F00EB800202EBC00207EB1B
:10D340008212DFF8E89112689142C0F0C98005EBC3
:10D350004000407810F0A2FA317801EB810202EB34
:10D36000C10107EB8111096888423CBF0120BDE87B
:10D37000F087002971D06E4DDFF8B8816FF02F0A69
:10D38000307800EB800101EBC00007EB80101E300D
:10D39000102105F0D1F900287DD1307800EB800113
:10D3A00001EBC00007EB80102E3040F20E3105F08B
:10D3B000D3F900286FD1307800EB800101EBC00079
:10D3C00007EB80101E305CA1F4F7AFFF0028307827
:10D3D00000EB800101EBC00007EB801012D01E3083
:10D3E00057A1F4F7A2FF0028307800EB800101EB91
:10D3F000C00007EB801023D01E3054A1F4F795FF36
:10D4000060B33EE090F82E00312809D032280CD0CD
:10D4100033280FD0342804BF4620F6F78FFD30E0C4
:10D4200046200EF081FC60BB08E046200EF0A4FD13
:10D4300038BB03E046200EF05BFD10BB012420E06A
:10D4400090F82F1090F82E00303800EB80000AEB97
:10D450004000084488F8000013E043E0FFE798F834
:10D46000000070B1317801EB810202EBC10107EBE2
:10D47000811191F82E10312914D0322918BF0224BD
:10D480001FD0307800EB800101EBC00007EB80106B
:10D490000068002800E023E07FF472AF012C1FD069
:10D4A00004B322E0415D11F0080FEAD1162109F022
:10D4B000BDF898F800000121401EC0B20DF0FCFF3D
:10D4C000DFE7415D11F0080FDBD0192109F0AEF85C
:10D4D00098F800000121401EC0B2F7F737FDD0E7F1
:10D4E000012000E0022089F80E00307800EB800176
:10D4F00001EBC00018A107EB80100A68C0F81E20DD
:10D500004A68C0F822208A68C0F8262089894185A7
:10D51000002180F82C10082101770020BDE8F08759
:10D52000550100205401002010240020D8010020C3
:10D53000951C0020EE0100204374726C0000000076
:10D540004279706173734E756D00000042797061AD
:10D5500073734F70740000002F52656D6F746543D4
:10D5600074722E68746D00002DE9F04F87B0DFF8FB
:10D57000D49200200590B24C99F8000004EB4000D2
:10D58000407810F08BF9054699F8000004EB400054
:10D5900040780FF0C9FE291899F80000DFF8A8A21A
:10D5A00000EB800202EBC0020AEB8212DFF89CB2B1
:10D5B00012689142C0F0428104EB4000407810F0C4
:10D5C0006DF999F8001001EB810202EBC1010AEB41
:10D5D0008112116888423EBF012007B0BDE8F08F7C
:10D5E00092F83E0320B1012800F0F48000F0F9B871
:10D5F000002918BFE84600F0F48099F8000000EB1D
:10D60000800101EBC0000AEB80101E30102105F0F4
:10D6100093F8002840F0128199F8000000EB800197
:10D6200001EBC0000AEB80102E3040F20E3105F005
:10D6300093F8002840F0028199F8000000EB800187
:10D6400001EBC0000AEB80101E3081A1F4F76DFEE3
:10D6500000287DD199F80000002500EB800101EB46
:10D66000C0000AEB801000F12E060024305D2C284B
:10D670000DD0601C44B2102CF8DB5DB1012D10D030
:10D68000022D13D0032D1BD0042D21D027E0002024
:10D690003055F2E730461AF050FB401E8BF80D0073
:10D6A0001DE031466846F4F75BFE18E0307830281C
:10D6B00008BF022713D031280CBF012704270EE032
:10D6C000314608F110001AF065FB002870D106E021
:10D6D000314608F112001AF05DFB002868D13019BC
:10D6E000461C681C45B2052DBFDB9BF80D005A4C4B
:10D6F00000EB800004EB800000F25B3114226846EE
:10D70000F4F721FEE0B19BF80D00009900EB8000DA
:10D7100004EB8000C0F85B130199C0F85F13029915
:10D72000C0F863130399C0F867130499C0F86B132A
:10D7300000200DF0E1F940F29C6120460DF0D2FA94
:10D74000042F36D09BF80D00434A00F1280100E079
:10D750002FE002EBD10201F0070192F840210124F1
:10D7600004FA01F10A4269D0022F04BF3B4AF021BA
:10D7700004D0012F04BF394AF42101D10EF040F941
:10D7800037489BF80D2003211044817111F04EFBA6
:10D79000CBF8200099F8000000EB800101EBC000FD
:10D7A0000AEB801080F83E4307B00220BDE8F08FFE
:10D7B00044E099F8000000EB800101EBC0000AEBA7
:10D7C0008010006800287FF418AF0598012835D034
:10D7D00038B109E022489BF80D10084480790328ED
:10D7E0001CD002208BF80E0099F8000000EB80019D
:10D7F00001EBC0001BA10AEB80100A68C0F81E20D4
:10D800004A68C0F822200989C184002180F82810C4
:10D810000821017707B00020BDE8F08F11F006FB6A
:10D82000DBF8201041F28832431A0021D21A71EB42
:10D83000010022BF022007B0BDE8F08F0120D1E730
:10D84000550100205401002010240020D8010020A0
:10D850007377536D61727400E4150020C3360108BC
:10D86000801C00202F536D6172742E68746D00004F
:10D870002DE9F05FFE4FFD4E002538782C4606EB73
:10D880004000407810F00AF88046387806EB4000F7
:10D8900040780FF049FD08EB00013878DFF8D483B9
:10D8A00000EB800202EBC00208EB8212DFF8C8A393
:10D8B00012689142C0F0268206EB400040780FF0DB
:10D8C000EDFF397801EB810202EBC10108EB811118
:10D8D000096888423CBF0120BDE8F09F002900F0A4
:10D8E0001382DFF89893E64E4FF6FF7B387800EB13
:10D8F000800101EBC00008EB80101E30102104F005
:10D900001BFF002840F0FE81387800EB800101EB1E
:10D91000C00008EB80102E3040F20E3104F01CFFE6
:10D92000002840F0EF81387800EB800101EBC00067
:10D9300008EB80101E30D3A1F4F7F7FC00283878EC
:10D9400000EB800101EBC00008EB80107ED01E30A0
:10D95000CEA1F4F7EAFC0028387800EB800101EB57
:10D96000C00008EB801072D01E30CBA1F4F7DDFCB4
:10D970000028387800EB800101EBC00008EB801034
:10D9800066D01E30C7A1F4F7D0FC0028387800EB31
:10D99000800101EBC00008EB801074D01E30C3A1E1
:10D9A000F4F7C3FC0028387800EB800101EBC000DD
:10D9B00008EB801068D01E30BFA1F4F7B6FC002839
:10D9C000387800EB800101EBC00008EB801078D0C4
:10D9D0001E30BBA1F4F7A9FC002873D0387800EB07
:10D9E000800101EBC00008EB80101E30B6A1F4F7F7
:10D9F0009CFC002867D0387800EB800101EBC00068
:10DA000008EB80101E30B3A1F4F78FFC002878D00B
:10DA1000387800EB800101EBC00008EB80101E306D
:10DA2000AFA1F4F782FC00286CD0387800EB8001BD
:10DA300001EBC00008EB80101E30ACA1F4F775FCC0
:10DA4000002871D0387800EB800102E00CE01CE087
:10DA50002AE001EBC00008EB80101E30A6A1F4F70D
:10DA600064FC002873D0F0E02E301AF0C2F9B0F553
:10DA7000807F29D296F83211C0B281421CBF0124A6
:10DA800086F83201E1E021E030E02E301AF0B1F901
:10DA9000B0F5807F18D296F83311C0B281421CBF16
:10DAA000012486F83301D0E02E301AF046F91F2801
:10DAB0000AD296F8341181421CBF012486F8340141
:10DAC000C3E020E031E043E00125BEE02E301AF053
:10DAD00034F996F83511814260D086F83501012479
:10DAE000C0EB00108000A9F84C00AEE02E301AF018
:10DAF00024F996F83A1181421CBF012486F83A01B4
:10DB0000A3E05BE06CE02E301AF073F9B6F8E61093
:10DB1000814243D0A6F8E600C0EB00100BEA80007B
:10DB20000124A9F84A0090E06CE0387896F83611A4
:10DB300000EB800202EBC00008EB801090F82E0092
:10DB4000303881421CBF012486F836017DE06BE04D
:10DB5000387896F8371100EB800202EBC00008EB32
:10DB6000801090F82E00303881426ED0C0B201246F
:10DB700086F83701012896F8EB0210D020F001005A
:10DB800086F8EB0296F8EC0220F0010086F8EC0231
:10DB900096F8ED0220F0010086F8ED0255E040F025
:10DBA000010086F8EB0296F8EC0240F0010086F8DE
:10DBB000EC0296F8ED0240F00100EDE7387896F8B7
:10DBC000391100EB800202EBC00008EB801090F8E6
:10DBD0002E00303881421CBF012486F8390134E020
:10DBE000387896F83B1100EB800202EBC00008EB9E
:10DBF000801090F82E00303881421CBF012486F836
:10DC00003B0122E0387896F83C1100EB800202EBF1
:10DC1000C00008EB801090F82E00303881421CBF05
:10DC2000012486F83C0110E0387896F83D1100EBAD
:10DC3000800202EBC00008EB801090F82E00303814
:10DC400081421CBF012486F83D01387800EB800139
:10DC500001EBC00008EB8010006800287FF446AE9E
:10DC6000012D4FD005B152E04EE0000055010020DB
:10DC70005401002010240020D8010020801C002026
:10DC8000E4150020496E64656C6179004F75744439
:10DC9000656C61790000000042656C6C54696D65CB
:10DCA00000000000776C734C6F73650041435F4464
:10DCB0006574656374000000436F6D6D00000000C3
:10DCC00041726D436C65770041726D5265706F7281
:10DCD00074000000466F72636541726D00000000C1
:10DCE000446F6F724465746563740000776C73549D
:10DCF000616D706572000000416C61726D4C696D00
:10DD000069740000012000E002208AF80E00012C56
:10DD100007D100200CF0F0FE40F29C610C480CF0A2
:10DD2000E1FF387800EB800101EBC00009A108EBAE
:10DD300080100A684B688968C0F81E20C0F822303D
:10DD4000C0F82610082101770020BDE8F09F0000F0
:10DD5000E41500202F4F7074696F6E2E68746D008B
:10DD60002DE9F84FFF4FFE4D4FF00008387844463C
:10DD700005EB400040780FF091FD0646387805EB42
:10DD8000400040780FF0D0FA31183878F64E00EBAA
:10DD9000800202EBC00206EB82124FF0010A126809
:10DDA0009142C0F0258205EB400040780FF076FDEF
:10DDB000397801EB810202EBC10106EB81110968A0
:10DDC00088423CBF0120BDE8F88F4FF002090029CE
:10DDD0001CBFDFF898B3E64D00F00E82387800EBF8
:10DDE000800101EBC00006EB80101E30102104F012
:10DDF000A3FC002840F0FC81387800EB800101EBA7
:10DE0000C00006EB80102E3040F20E3104F0A4FC6E
:10DE1000002840F0ED81387800EB800101EBC00074
:10DE200006EB80101E30D3A1F4F77FFA0028387873
:10DE300000EB800101EBC00006EB80107ED01E30AD
:10DE4000CEA1F4F772FA0028387800EB800101EBDC
:10DE5000C00006EB801070D01E30C9A1F4F765FA3F
:10DE60000028387800EB800101EBC00006EB801041
:10DE70007CD01E30C4A1F4F758FA0028387800EBA3
:10DE8000800101EBC00006EB801070D01E30C1A1F4
:10DE9000F4F74BFA0028387800EB800101EBC00062
:10DEA00006EB80107AD01E30BDA1F4F73EFA0028B0
:10DEB000387800EB800101EBC00006EB80106ED0DB
:10DEC0001E30BAA1F4F731FA0028387800EB80014F
:10DED00001EBC00006EB80107BD01E30B6A1F4F73A
:10DEE00024FA0028387800EB800101EBC00006EB33
:10DEF00080106FD01E30B3A1F4F717FA00283878DD
:10DF000000EB800101EBC00006EB801079D01E30E1
:10DF1000AFA1F4F70AFA0028387800EB800101EB92
:10DF2000C00006EB80106DD01E30ACA1F4F7FDF9F7
:10DF3000002868D000F000B900E019E000F12E01DF
:10DF400005F29120F4F7F1F9002800F0F580387817
:10DF5000012400EB800101EBC00006EB801000F112
:10DF60002E0105F29120F4F7FBF9E5E018E032E02C
:10DF70002E3019F0E2FE95F9D112814240D00124F1
:10DF800085F8D102FAF7DEFC97480DF06BFADBF862
:10DF9000600040F48030CBF86000CDE034E048E031
:10DFA00090F82E00312807D095F8900202281CBF67
:10DFB000012485F89092BFE08C48016841F48051BB
:10DFC000016095F8900201281CBF012485F890A2F9
:10DFD000B2E043E057E000F12E01684619F0DAFEA6
:10DFE000002878D1022205F520716846F4F7ABF9D4
:10DFF00000281CBFBDF80000A5F8800200D0012455
:10E000009AE054E068E07CE000F12E01684619F0E7
:10E01000C1FE00285FD1022205F282216846F4F792
:10E0200092F900281CBFBDF80000A5F88202E6D1D5
:10E0300082E000F12E01684619F0ACFE00284AD1BA
:10E04000022205F521716846F4F77DF900281CBF0E
:10E05000BDF80000A5F88402D1D16DE000F12E01D9
:10E06000684619F097FE002835D1022205F2862174
:10E070006846F4F768F900281CBFBDF80000A5F851
:10E080008602BCD158E000F12E01684619F082FEEC
:10E0900008BB022205F522716846F4F754F90028FE
:10E0A0001CBFBDF80000A5F88802A8D144E000F12B
:10E0B0002E01684619F06EFE68B9022205F28A2127
:10E0C0006846F4F740F900281CBFBDF80000A5F829
:10E0D0008A0294D130E041E000F12E01684619F047
:10E0E00059FED8BB022205F523716846F4F72BF9D7
:10E0F00000281CBFBDF80000A5F88C027FF47FAF9C
:10E100001AE0387800EB800101EBC00006EB8010CC
:10E1100000F12E01684619F03DFEF8B9022205F221
:10E120008E216846F4F70FF900281CBFBDF80000E7
:10E13000A5F88E027FF463AF387800EB800101EB25
:10E14000C00006EB8010006800287FF447AEB8F1ED
:10E15000010F4DD0B8F1000F4ED050E048E0000064
:10E160005501002054010020102400203815002003
:10E17000E41500207365727665720000474D540007
:10E18000626F785F7061720041726D54696D6531C4
:10E190000000000044697361726D54696D6531005F
:10E1A00041726D54696D653200000000446973610D
:10E1B000726D54696D65320041726D54696D6533DD
:10E1C0000000000044697361726D54696D6533002D
:10E1D00041726D54696D65340000000044697361DB
:10E1E000726D54696D34000068000020801C0020AE
:10E1F000144880F80EA002E0124880F80E90012C1E
:10E2000007D100200CF078FC40F29C610E480CF025
:10E2100069FD387800EB800101EBC0000BA106EB33
:10E2200080100A68C0F81E204A68C0F822200989B8
:10E23000C184002180F82810082101770020BDE862
:10E24000F88F0000D8010020E41500202F54696DDC
:10E2500065722E68746D00002DE9F04FDFF81484AC
:10E26000DFF8149483B098F80000022700EB8001D7
:10E2700001EBC00109EB81114FF6FF7691F83E13D7
:10E28000FE4CDFF8FCA329B1012960D002297CD023
:10E2900000F0D9B9002504EB4000009501954078C5
:10E2A0002B460722F7A10EF02FFEB04209D0012025
:10E2B0008AF800008AF80C00CAF818508AF80A5048
:10E2C00014E00095019598F80000002304EB40004D
:10E2D00007224078EDA10EF017FEB04200F06C81ED
:10E2E0008AF80C70CAF818508AF80A5000950195FF
:10E2F00098F80000002304EB400002224078E5A1DA
:10E300000EF002FEB04200F0578198F8001001EBC9
:10E31000810202EBC10209EB821213681B1A9B1FD8
:10E32000801C136082B204EB4100002140780EF0A3
:10E330005FFF98F8001001EB810202EBC10109EBCD
:10E3400081110A68101A0860012081F83E0300203C
:10E350000090019098F80000002304EB4000042294
:10E360004078CDA10EF0D0FDB0425FD0001D82B24A
:10E3700098F80000002104EB400040780EF038FFD0
:10E3800098F8001001EB810200E008E002EBC10107
:10E3900009EB81110A68101A086081F83E7398F839
:10E3A000000004EB400040780FF078FA064698F839
:10E3B000000000EB800101EBC00009EB8010016858
:10E3C000B14238BF0E469AF80C0010F0010F4DD044
:10E3D000B1F5482F02D901208AF80A00002E00F07A
:10E3E000E180802E34BF3046802082B298F8000051
:10E3F000A24B00EB800101EBC00103EB400009EBF5
:10E4000081111E3140780EF0F3FE054698F80000A9
:10E4100000EB800101EBC00009EB80110868401B94
:10E4200008609AF80A00761B40B3B8E098F800003C
:10E4300004EB400040780FF031FA001F82B298F8E8
:10E440000000002104EB400040780EF0D1FE98F867
:10E45000001001EB810202EBC10109EB81110A6896
:10E46000101A086003B00120BDE8F08F00F0020030
:10E47000002818BFB1F5801FB0D9ACE79AF80C009E
:10E4800010F0010F4CD010F0800F2ED184A001F1BC
:10E490001E0B0090F3F742FFC7B2BD4228BF002415
:10E4A0001BD31ADD0BEB04003A460099F3F74BFF40
:10E4B00028B1601C84B2281BB842F3DC0DE01BEBD2
:10E4C00004000AD007F0B0FE8AF80B009AF80C009E
:10E4D00040F080008AF80C0002E001208AF80A006F
:10E4E0009AF80C0010F0800F59D0DAF8180000F5F7
:10E4F00060300CF001FB98F800002A4600EB800128
:10E5000001EBC00009EB801000F11E019AF80B002E
:10E5100008F032F8DAF818002844CAF818003EE08B
:10E5200010F0020F3BD010F0800F21D15EA001F15E
:10E530001E0B0090F3F7F2FEC7B2BD4228BF0024C5
:10E5400016D315DD0BEB04003A460099F3F7FBFEFA
:10E5500028B1601C84B2281BB842F3DC08E01BEB36
:10E56000040005D09AF80C0040F080008AF80C00F6
:10E57000DAF8180000F580100CF0BEFA98F80000E8
:10E58000294600EB800202EBC00009EB80101E3030
:10E590000CF0A8FBDAF818002844CAF81800002E7E
:10E5A0007FF41FAF98F8000000EB800101EBC00082
:10E5B00009EB8010016819B103B00120BDE8F08FAC
:10E5C000032480F83E439AF80A00D8BB9AF80C005E
:10E5D00010F0010F0BD08AF80040012007F0D4FFA3
:10E5E0009AF80B0007F012FE8AF80E400FE010F0C8
:10E5F000020F0CD010F0800F25D030480CF07CFAC0
:10E600000F212FA00CF06EFB04208AF80E000020D2
:10E610008AF80C0098F8000000EB800101EBC000C4
:10E620002BA109EB80100A684B688968C0F81E208E
:10E63000C0F82230C0F826100821017703B000206E
:10E64000BDE8F08FFFE700208AF80C0001208AF86F
:10E650000E0098F8000000EB800101EBC0001CA147
:10E6600009EB80100A68C0F81E204A68C0F8222012
:10E67000896833E054010020102400205501002057
:10E68000D80100207755706461746500735570641B
:10E69000617465000D0A00000D0A0D0A00000000FB
:10E6A0004D50465300000000343230393233313996
:10E6B00037383034313731323732000000F01F0044
:10E6C00073797374656D20757064617465202100C1
:10E6D0002F5570646174652E68746D00C0F8261043
:10E6E0000821017703B00020BDE8F08F2DE9F04349
:10E6F000DD4FDC4E0025387887B006EB40002C4615
:10E7000040780FF0CBF88046387806EB4000407830
:10E710000EF00AFE08EB00013878DFF8508300EBBA
:10E72000800202EBC00208EB8212DFF84493126809
:10E730009142C0F06B8106EB400040780FF0AEF8DC
:10E74000397801EB810202EBC10108EB8111096804
:10E7500088423EBF012007B0BDE8F083002918BF02
:10E76000C44E00F05581387800EB800101EBC00009
:10E7700008EB80101E30102103F0DEFF002840F06F
:10E780004581387800EB800101EBC00008EB801078
:10E790002E3040F20E3103F0DFFF002840F03681CA
:10E7A000387800EB800101EBC00008EB80101E30D0
:10E7B000B1A1F3F7BAFD0028387800EB800101EB36
:10E7C000C00008EB801054D01E30ADA1F3F7ADFDB2
:10E7D0000028387800EB800101EBC00008EB8010C6
:10E7E0005BD01E30A8A1F3F7A0FD0028387800EB1D
:10E7F000800101EBC00008EB80106FD01E30A4A197
:10E80000F3F793FD0028387800EB800101EBC0009E
:10E8100008EB801079D01E309FA1F3F786FD002809
:10E82000387800EB800101EBC00008EB80106BD062
:10E830001E309BA1F3F779FD0028387800EB8001AA
:10E8400001EBC00008EB80107ED01E3095A1F3F7DD
:10E850006CFD0028387800EB800101EBC00008EB6C
:10E86000801072D01E3091A1F3F75FFD00286ED0AA
:10E87000BDE000F12E01684619F073FA00287DD042
:10E8800006F1E801684619F00DF800285BD1012473
:10E890001222694606F1E80032E000F12E016846D6
:10E8A00019F05FFA002869D006F1FA01684618F0FD
:10E8B000F9FF002847D10098C6F8FA000198C6F879
:10E8C000FE000298C6F802010398C6F80601BDF8DA
:10E8D00010000124A6F80A0189E0FFE700F12E01EB
:10E8E000684619F03EFA88B306F58671684618F056
:10E8F000D9FF00287BD101241222694606F58670D3
:10E90000F3F7B4FC73E000E022E000F12E0168466A
:10E9100019F027FAD0B106F58F71684618F0C2FFDA
:10E92000002864D10098C6F81E010198C6F822019B
:10E930000298C6F826010398C6F82A01BDF810000F
:10E940000124A6F82E0152E012E026E016E032E0A3
:10E950002E3019F0F2F9411E8DF800000F290DD26A
:10E9600096F8301181421CBF012486F830013EE048
:10E970002E3005A90CF05CFF012801D0012536E0FE
:10E98000042206F25A6105A8F3F7DDFC78B3394892
:10E9900005990124C0F85A1629E02E30F3F721FD1D
:10E9A000344980B2B1F85E1681421CBF3149A1F8EA
:10E9B0005E061BD11BE03878112200EB800101EBD1
:10E9C000C00008EB80102E3006F5CC61F3F7BBFCDD
:10E9D00068B1387800EB800101EBC00008EB8010D3
:10E9E00000F12E0106F5CC60F3F7BAFC012438786B
:10E9F00000EB800101EBC00008EB801000680028EC
:10EA00007FF4B1AE012D01D015B104E0012000E08A
:10EA1000022089F80E00012C07D100200CF06CF8C0
:10EA200040F29C6113480CF05DF9387800EB8001EE
:10EA300001EBC0001EA108EB80100A68C0F81E2080
:10EA40004A68C0F822208A68C0F826208989418552
:10EA5000002180F82C100821017707B00020BDE8C4
:10EA6000F0830000550100205401002010240020F4
:10EA7000D8010020E415002050686F6E6531000059
:10EA800050686F6E6532000050686F6E653300002D
:10EA900050686F6E653400004469616C436E7400A9
:10EAA00069700000706F727400000000707764007D
:10EAB0002F5573657250686F6E652E68746D000017
:10EAC0002DE9F84FDFF8F4B30027FB489BF800105E
:10EAD000B94600EB41003E463D463C46B8464078CC
:10EAE0000EF0DCFE8246F4489BF8001000EB41007B
:10EAF00040780EF019FC0AEB00029BF8000000EBD6
:10EB0000800101EBC003EE4901EB831109688A42E1
:10EB1000C0F00082E849DA4601EB400040780EF090
:10EB2000BDFE02469AF8000000EB800101EBC00038
:10EB3000E34901EB8010006882423CBF0120BDE840
:10EB4000F88F00281CBFDFF87CB34FF0010A00F0FB
:10EB5000E581DA48007800EB800101EBC001D8487C
:10EB600000EB81101E30102103F0E6FD002840F07C
:10EB7000D181D248007800EB800101EBC001D04880
:10EB800000EB81102E3040F20E3103F0E5FD00283D
:10EB900040F0C081C948007800EB800101EBC00162
:10EBA000C74800EB81101E30C7A1F3F7BEFB002859
:10EBB000C248007800EB800101EBC001C04800EBC7
:10EBC000811043D01E30C3A1F3F7AFFB0028BB4830
:10EBD000007800EB800101EBC001B94800EB811027
:10EBE00046D01E30BDA1F3F7A0FB0028B348007843
:10EBF00000EB800101EBC001B14800EB81107FD038
:10EC00001E30B9A1F3F791FB0028AC48007800EB67
:10EC1000800101EBC001AA4800EB81106FD01E30CB
:10EC2000B4A1F3F782FB0028A448007800EB800130
:10EC300001EBC001A24800EB811072D01E30B0A1E0
:10EC4000F3F773FB00286DD000F024B990F82E1074
:10EC5000302900F01F812E3019F06FF80646B9F107
:10EC6000000F04BF8BF800608BF801A000F012B910
:10EC70002E30A5A1F3F759FB68B3002E00F00A81EE
:10EC8000701EC6B28D48007800EB800101EBC00118
:10EC90008B4800EB811090F82E1029B300F12E0163
:10ECA000684618F0F2FF002873D099480AFA06F275
:10ECB0004FF0010890F84011114380F8401106EB25
:10ECC00046010844BDF80010A0F848119DF8021054
:10ECD00080F84A11DEE08BF800604FF0010902274E
:10ECE0008BF801A0D6E00BE089480AFA06F24FF053
:10ECF000010890F84011914380F84011CAE012E0F9
:10ED000090F82E10302943D02E3019F016F8054611
:10ED1000B9F1000F3CD18BF8005002208BF80100B4
:10ED2000B8E04EE05EE02E3077A1F3F7FEFA88B34C
:10ED3000002D2DD0E81DC5B26048007800EB8001A1
:10ED400001EBC0015E4800EB811090F82E1049B332
:10ED500000F12E01684618F098FF002819D06C4A7F
:10ED600005F0070302EBD5000AFA03F390F840110F
:10ED70004FF00108194380F8401105EB450010449D
:10ED8000BDF80010A0F848119DF8021080F84A1153
:10ED900080E07EE0FFE702274FF001098BF800508A
:10EDA00038461CE05A4805F0070200EBD5000AFA85
:10EDB00002F290F840114FF00108914380F84011A1
:10EDC00068E090F82E10302964D02E3018F0B5FF8E
:10EDD0000446B9F1000F5DD18BF8004003208BF899
:10EDE000010057E03548007800EB800101EBC001DD
:10EDF000334800EB81102E3043A1F3F796FA002838
:10EE000004BF4FF001090227E6D094B304F12700B4
:10EE1000C4B22A48007800EB800101EBC001284809
:10EE200000EB811090F82E1021B300F12E016846FE
:10EE300018F02BFF68B3364A04F0070302EBD40046
:10EE40000AFA03F390F840114FF00108194380F8D3
:10EE500040119DF8010070388DF8010004EB44006A
:10EE60001044BDF80010A0F848119DF8021080F879
:10EE70004A110FE0264804F0070200EBD4000AFA1A
:10EE800002F290F840114FF00108914380F84011D0
:10EE900000E001270948007800EB800101EBC00188
:10EEA000074800EB8110006800287FF452AE012F64
:10EEB00030D007B135E031E0550100205401002089
:10EEC00010240020EE01002072656D6F74654E6F96
:10EED0000000000072656D6F746500006465746504
:10EEE00063746F724E6F00006465746563746F7253
:10EEF000000000007377697463684E6F00000000C3
:10EF0000737769746368000047657450617200002C
:10EF1000E415002015490120887302E013480221FE
:10EF20008173B8F1010F07D100200BF0E5FD40F22D
:10EF30009C610F480BF0D6FE0E48007800EB800174
:10EF400001EBC0010C4800EB81100CA10A68C0F86D
:10EF50001E204A68C0F822208A68C0F826208989C5
:10EF60004185082101770020BDE8F88FD8010020F5
:10EF7000E415002054010020102400202F5769724E
:10EF8000656C6573732E68746D0000002DE9F05F89
:10EF9000DFF878B40027DFF870849BF80000B946EA
:10EFA00008EB40003C463D463E4640780EF076FC7D
:10EFB00082469BF8000008EB400040780EF0B4F960
:10EFC0000AEB00019BF80000DFF844A400EB80028C
:10EFD00002EBC0020AEB821212689142C0F0ED818E
:10EFE00008EB400040780EF059FC01469BF8000009
:10EFF00000EB800202EBC0000AEB80100068814247
:10F000003CBF0120BDE8F09F002818BFDFF8048452
:10F0100000F0D7819BF8000000EB800101EBC000FD
:10F020000AEB80101E30102103F086FB002840F010
:10F03000C4819BF8000000EB800101EBC0000AEBEB
:10F0400080102E3040F20E3103F086FB002840F095
:10F05000B4819BF8000000EB800101EBC0000AEBDB
:10F0600080101E30ECA1F3F760F900289BF8000037
:10F0700000EB800101EBC0000AEB801079D01E305C
:10F08000E7A1F3F752F900289BF8000000EB80019C
:10F0900001EBC0000AEB80106AD01E30E3A1F3F749
:10F0A00044F9002878D09BF8000000EB800101EBC8
:10F0B000C0000AEB80101E30DFA1F3F736F90028FC
:10F0C0006BD09BF8000000EB800101EBC0000AEB65
:10F0D00080101E30DBA1F3F728F900287ED09BF8C2
:10F0E000000000EB800101EBC0000AEB80101E3035
:10F0F000D6A1F3F71AF9002871D09BF8000000EBB5
:10F10000800101EBC0000AEB80101E30D2A1F3F7A2
:10F110000CF900289BF8000000EB800101EBC00017
:10F120000AEB80107DD01E30CEA1F3F7FEF8002848
:10F130009BF8000000EB800101EBC0000AEB80109F
:10F1400070D01E30CAA1F3F7F0F800286BD09BF8FE
:10F15000000000EB800101EBC0000AEB80101E30C4
:10F16000C6A1F3F7E2F800287CD000F010B900E067
:10F1700014E090F82E10302900F009812E3018F09C
:10F18000DCFD0446B9F1000F40F00181BE485A2170
:10F190000470417000F0FBB80DE031E02E30BBA1EF
:10F1A000F3F7C3F8002840F0F280B7485A21047002
:10F1B000417000F009B9002C40D09BF8000008EB2A
:10F1C000040200EB800C0CEBC00092F837120AEB43
:10F1D000801001F01F0390F82E0001E02FE047E0BF
:10F1E000303883422AD060F30401012682F83712B6
:10F1F00011F01F0F22D1601EC0B2F5F777FEC6E0F6
:10F20000002C1BD008EB04029BF8000092F8371288
:10F2100000EB800C0CEBC000C1F341130AEB801033
:10F2200002E036E045E068E090F82E003038834296
:10F2300004D060F34611012682F83712A7E0002CB3
:10F2400074D09BF8000000EB800101EBC0000AEBDA
:10F2500080102E3018F071FD08EB040191F8712632
:10F26000824200E063E01CBF81F8710601268EE057
:10F27000002C5BD09BF8000000EB800101EBC0008C
:10F280000AEB801000F12E01601EC0B217F0C6F824
:10F290007DE090F82E10302979D02E3018F04DFDF9
:10F2A0000546B9F1000F72D1774956200D704870AC
:10F2B0006DE02E3075A1F3F738F8C8B1002D66D097
:10F2C0009BF8000000EB800101EBC0000AEB80100E
:10F2D0002E3018F032FD08EB850191F85C22824255
:10F2E00055D028289CBF012681F85C024FD91CE02C
:10F2F000654956200D70487066E0BDB19BF800006E
:10F3000000EB800101EBC0000AEB80102E3018F0FA
:10F3100014FD08EB850191F85D22824237D0282840
:10F320009CBF012681F85D0231D901272FE075B31A
:10F330009BF8000000EB800101EBC0000AEB80109D
:10F340002E3018F056FDFF2888BF012709D808EB9A
:10F350008501C0B291F85E2282421CBF012681F86D
:10F360005E0208EB850090F85E1200291FBF90F83E
:10F370005C12002990F85D12002990F85F1216D0F7
:10F3800001291CBF0126314601D080F85F129BF88D
:10F39000000000EB800101EBC0000AEB8010006868
:10F3A00000287FF437AE012F07D057B10CE00229B7
:10F3B0001CBF01260221E8D1E9E736490120887304
:10F3C00002E0344902208873012E07D100200BF09F
:10F3D00093FB40F29C610F480BF084FC9BF800000B
:10F3E00000EB800101EBC0002BA10AEB80100A6842
:10F3F000C0F81E204A68C0F822200989C18408216B
:10F4000001770020BDE8F09F550100205401002045
:10F4100010240020E41500207A6F6E654E6F000006
:10F420005A6E476574506172000000005A6F6E6535
:10F4300054797065000000005A6F6E6542656C6C0F
:10F440000000000053776974636800005A6F6E65AE
:10F450004E616D65000000004F7665726C61705AF8
:10F460006F6E65004F766C705A6F6E6531000000EC
:10F470004F766C705A6F6E65320000004F766C707C
:10F4800054696D6500000000EE010020476574506E
:10F4900061720000D80100202F5A6F6E652E6874CB
:10F4A0006D000000B0F5837F00F0318254DCDB2872
:10F4B0007ED037DCC6287CD025DCBC287AD018DC8E
:10F4C000B62878D00CDC2B2876D004DC032874D046
:10F4D0002A2873D1B9E02C2871D02D286ED1BAE03A
:10F4E000B7286DD0B9286CD0BA286BD0BB2865D1AD
:10F4F000BDE0BD38092861D2DFE800F0BEC0C2C45B
:10F50000C6C9CBCDD000C738142857D2DFE800F0E9
:10F51000DDDCDBDAD9D8D7D6D5D4D3D2D191D0CFD0
:10F52000CECDCCCBDC382A2848D2DFE800F0F5F489
:10F53000F3F2F1F0EFEEEDECEBEAE9E8E7E6E5E413
:10F54000E3E2E1E0DFDEDDDCDBDAD9D8D7D6D58255
:10F550008282D4D3D2D1D0CFB0F5987F00F063822D
:10F560001ADCA0F20710292863D2DFE800F0FDFCC6
:10F57000FBFAF9F8F7F662F5F4F3F2F1F0EFEEEDDD
:10F58000ECEBEAE9E8E7E6E5E4E3E2E1E0DFDEDD33
:10F59000DCDBDAD9D8D7D60040F24512A0F245110B
:10F5A000904200F082821BDCA0F2311014280AE0A5
:10F5B00032E176E05EE050E049E044E039E048E0E6
:10F5C0004DE04EE050E034D2DFE800F0FDFCFBFA05
:10F5D000F9F8F7F6F5F4F3F2F1F0EFEE33EDECEBCA
:10F5E0000A2900F0808207DC23D2DFE801F022F54F
:10F5F000F4F3F2F1F0EFEEED172900F084820CDC69
:10F600000B2900F073820C2900F07382132900F09B
:10F61000738216290DD100F073BA182900F0768292
:10F62000192900F07682652900F07682662900F0BB
:10F630007682FE48411E0422097800EB4100FCA1BD
:10F6400040780EF005BB02F011BA02F0E5B901F006
:10F650008DBC01F0A3BB01F033BD00F093BD01F000
:10F66000EDBE012001F02ABC022001F027BC0320DE
:10F6700001F024BC01F0F2BE01F0EABA01F0F8BAE0
:10F6800000F074BA01F004BB002002F0D1B901F01F
:10F69000AFBA01F00DBB012002F0CAB9022002F09E
:10F6A000C7B9032061E0B4E0B1E0ADE0A9E0A5E0B6
:10F6B000A1E09DE099E095E091E070E06CE068E009
:10F6C00064E060E05CE058E054E050E01BE116E1EB
:10F6D00011E10DE109E105E101E1FDE0F9E0F5E00D
:10F6E000F1E0EDE0E9E0E5E0E1E0DDE0D9E0D5E002
:10F6F000D1E0CDE0C9E0C5E0C1E0BDE0B9E0B5E0F2
:10F70000B1E0ADE0A9E0A5E0A1E09DE099E095E0E1
:10F7100091E08DE089E085E081E081E17DE179E1C2
:10F7200075E171E16EE16BE168E164E160E15CE18A
:10F7300058E154E150E14CE148E144E141E13CE170
:10F7400037E132E12DE128E123E11EE119E114E185
:10F750000FE10AE105E100E1FBE0F6E0F1E0ECE0B9
:10F76000E7E0E2E0DDE0D8E0D3E002F061B90420B8
:10F7700002F05EB9052002F05BB9062002F058B92C
:10F78000072002F055B9082002F052B9092002F012
:10F790004FB90A2002F04CB90B2002F049B90C20F5
:10F7A0001BE07FE17CE177E173E16FE16CE168E10F
:10F7B00064E160E15CE158E154E150E14CE148E191
:10F7C00044E140E13CE139E18AE186E182E17EE128
:10F7D0007AE176E172E16EE16AE102F029B90D2089
:10F7E00002F026B90E2002F023B90F2002F020B952
:10F7F000102002F01DB9012000F0A6BB022000F08D
:10F80000A3BB032000F0A0BB042000F09DBB00F0D0
:10F810003FBC012000F0D0BB022000F0CDBB032094
:10F8200000F0CABB042000F0C7BB052000F0C4BB39
:10F83000012000F02BBE022000F028BE032000F0C3
:10F8400025BE042000F022BE052000F01FBE0620C9
:10F8500000F01CBE072000F019BE012000F09EBE83
:10F86000022000F09BBE032000F098BE042000F0B0
:10F8700095BE052000F092BE062000F08FBE072046
:10F8800000F08CBE082000F089BE092000F086BE82
:10F890000A2000F083BE0B2000F080BE0C2000F098
:10F8A0007DBE0D2000F07ABE0E2000F077BE0F2046
:10F8B00000F074BE102000F071BE112000F06EBE8A
:10F8C000122000F06BBE012001F028B9022001F0E7
:10F8D00025B9032001F022B9042001F01FB9052049
:10F8E00001F01CB9012001F0F3B9022001F0F0B9D8
:10F8F000032001F0EDB90821012001F0D3BD202142
:10F90000022001F0CFBD1021032001F0CBBD01F09A
:10F910004FBE0021012001F0CDBE0121084601F0BB
:10F92000C9BE0221012001F0C5BE0321012001F062
:10F93000C1BE0421012001F0BDBE0521012001F05E
:10F94000B9BE0621012001F0B5BE0721012001F05A
:10F95000B1BE0121022001F0ADBE0221084601F036
:10F96000A9BE0321022001F0A5BE0121032001F060
:10F97000A1BE0221032001F09DBE0321084601F033
:10F9800099BE0421032001F095BE0521032001F05A
:10F9900091BE0621032001F08DBE0721032001F056
:10F9A00089BE0821032001F085BE0021042001F05A
:10F9B00081BE0021052001F07DBE0021062001F05E
:10F9C00079BE01F0FBB90A2000F0D4BE002000F09F
:10F9D000D1BE012000F0CEBE022000F0CBBE03203D
:10F9E00000F0C8BE042000F0C5BE052000F0C2BE75
:10F9F000012001F035BC022001F032BC01F070BBE7
:10FA000001F0EABF00F0D6B8012000F065B902208D
:10FA100000F062B9032000F05FB9042000F05CB987
:10FA2000012000F05BBF022006E00000550100202D
:10FA3000214445460000000000F050BF00F0E8BF40
:10FA4000012000F04DBC022000F04ABC032000F071
:10FA500047BC042000F044BC052000F041BC062057
:10FA600000F03EBC012001F079BC022001F076BC20
:10FA7000032001F073BC032001F0F2BB042001F06D
:10FA8000EFBB052001F0ECBB00F0E4BC0B2000F064
:10FA900071BE0C2000F06EBE0021072001F00ABEEE
:10FAA00000F09AB9002000F05FB9012000F05CB9C5
:10FAB000022000F059B9032000F010BF042000F02C
:10FAC0000DBF052000F00ABF062000F007BF072089
:10FAD00000F004BF082000F001BF092000F0FEBEC6
:10FAE0000A2000F0FBBE012000F0F2BA022000F074
:10FAF000EFBA032000F0ECBA0021082001F0DABDD3
:10FB0000062001F00BB8072001F008B8082001F02A
:10FB100005B8092001F002B8002000F043BB012025
:10FB200000F040BBF1B582B000240E4E0E4D02AF86
:10FB300007E034B128782E2106EB400040780EF023
:10FB400009F8385D694618F0A2F92878694606EB8D
:10FB5000400040780EF024F9641CE4B2042CE8D391
:10FB6000FEBD0000550100205401002009480A4A4A
:10FB7000007800EB800101EBC00102EB8111C97E2E
:10FB8000802918BF7047054901EB400004A1407867
:10FB90000EF006B954010020102400205501002069
:10FBA00064697361626C65643D2264697361626C4F
:10FBB000652200002DE9F0432A48ADF5017D90F85B
:10FBC000150300280CBF284C284C294DDFF8A480D1
:10FBD000294EA87928283CBFDFF8A090284F32D2C0
:10FBE000307807EB400040780DF078FE80280CD28A
:10FBF0003078012100EB800202EBC00008EB80109E
:10FC0000C1600DF5017DBDE8F083A87999F8001079
:10FC1000421C54F82030914204D11AA1684616F0D3
:10FC200091FC03E024A1684616F08CFC307869460C
:10FC300007EB400040780EF0B3F8A879401CC0B242
:10FC4000A8712828CCD30021A971307800EB80025C
:10FC500002EBC00008EB8010C1600DF5017DBDE82E
:10FC6000F0830000E415002038AA0208D8AA020890
:10FC7000D80100201024002054010020EE010020B3
:10FC8000550100203C6F7074696F6E2073656C6560
:10FC9000637465643D2273656C65637465642220DA
:10FCA00076616C75653D222564223E25733C2F6F7D
:10FCB0007074696F6E3E00003C6F7074696F6E20E7
:10FCC00076616C75653D222564223E25733C2F6F5D
:10FCD0007074696F6E3E000010B51A4C2378002BCB
:10FCE00008BF10BD184A1A49DFF860C0012809781A
:10FCF0000CEB410111D0022814D0032817D004289E
:10FD000018BF10BD985C10F0080F03D0487811A1FF
:10FD10000EF046F80020207010BD985C10F0010F26
:10FD20000AD110BD985C10F0020F05D110BD985C8F
:10FD300010F0040F08BF10BD4878BDE8104005A1C1
:10FD40000EF02EB8EE010020C6180020550100204C
:10FD500054010020636865636B65643D22636865D8
:10FD6000636B65642200000010B51449114C124BFE
:10FD70000978227803EB41017AB1114BD25C12F081
:10FD8000080F02D001280FD008E0022818BF10BDCC
:10FD900048780CA10EF004F803E028B1022818BF3F
:10FDA00010BD0020207010BD4878BDE8104005A1AE
:10FDB0000DF0F6BFEE010020550100205401002097
:10FDC000951C002073656C65637465643D227365E2
:10FDD0006C656374656422002DE9F041294CDFF8FD
:10FDE000A8802A4F607890B029283CBF284E294D22
:10FDF0003AD2387805EB400040780DF06FFD40288E
:10FE00000BD23878012100EB800202EBC00008EB36
:10FE10008010C16010B0BDE8F081627830783AB1EE
:10FE2000904213460FD11CA1684616F08BFB0EE0E2
:10FE300020B127A1684616F085FB08E02CA1684692
:10FE400016F080FB03E037A1684616F07BFB38789C
:10FE5000694605EB400040780DF0A2FF6078401C39
:10FE6000C0B260702928C4D300216170387800EBDB
:10FE7000800202EBC00008EB8010C16010B0BDE84A
:10FE8000F0810000D801002010240020540100203F
:10FE9000EE010020550100203C6F7074696F6E20E8
:10FEA00073656C65637465643D2273656C6563742A
:10FEB0006564222076616C75653D222530326422AE
:10FEC0003E253032643C2F6F7074696F6E3E0000C7
:10FED0003C6F7074696F6E2076616C75653D22258C
:10FEE000303264223E3C2F6F7074696F6E3E0000AA
:10FEF0003C6F7074696F6E2073656C6563746564C4
:10FF00003D2273656C6563746564222076616C754F
:10FF1000653D2225303264223E3C2F6F7074696F3C
:10FF20006E3E00003C6F7074696F6E2076616C7578
:10FF3000653D2225303264223E253032643C2F6FED
:10FF40007074696F6E3E000000B5174989B00128D2
:10FF500018D002281CD0032820D004281CBF09B0C8
:10FF600000BD91F8E52011A1684616F0EBFA1149A1
:10FF70000F48097800EB4100694640780DF010FF0A
:10FF800009B000BD1222BD31684607F09BFFEEE7C5
:10FF90001222CF31684607F095FFE8E7E131684665
:10FFA0000FF08EFCE3E70000E4150020256400005C
:10FFB0005501002054010020F0B5304D304E314F36
:10FFC0002978314C83B006EB4101012810D002287A
:10FFD00030D0032804BF487804F1A80134D00428A5
:10FFE00004BF487804F1B1012ED0052839D02DE0A6
:10FFF00094F8BB0001280FD048780DF06FFC402822
:020000040801F1
:100000000FD22878012100EB800202EBC00007EB41
:100010008010C16003B0F0BDD4F87100FFF782FD1D
:1000200014E0287804F1750106EB400040780DF0EB
:10003000B7FE0BE0B4F8A600694617F028FF287851
:10004000694606EB400040780DF0AAFE28780021B2
:1000500000EB800202EBC00007EB8010C16003B030
:10006000F0BD94F8BA2009A1684616F06BFA28781A
:10007000694606EB40004078E6E7000054010020A6
:100080005501002010240020E41500202564000004
:10009000074890F87000012818BF704705480649C6
:1000A000097800EB410005A140780DF079BE000011
:1000B000E4150020550100205401002063686563A9
:1000C0006B65643D22636865636B656422000000B4
:1000D000F0B5284D0446264F28788DB007EB400038
:1000E00040780DF0FBFB244E30280AD228780121FD
:1000F00000EB800202EBC00006EB8010C1600DB087
:10010000F0BD1E48012C04D0022C09D0032C0ED0C7
:1001100013E000F2C65130226846F2F7A7F80CE06F
:1001200000F2F65130226846F2F7A0F805E000F23E
:10013000266130226846F2F799F89DF80000002405
:1001400028B90FA00088ADF800008DF8024028788B
:10015000694607EB400040780DF022FE287800EB5E
:10016000800101EBC00006EB8010C4600DB0F0BD53
:10017000550100205401002010240020E415002027
:100180002222000005490448097800EB4100044997
:1001900040780DF005BE00005501002054010020FC
:1001A0002F1900202DE9F047434EDFF81091414D03
:1001B0003178434FADF5027D4FF000084FF0010A52
:1001C00009EB4101F8B101281CBF0DF5027DBDE826
:1001D000F08748780DF082FB0446B0F5007F88BFB9
:1001E0004FF400747B6A48F6FF701919814240D3BE
:1001F000C41A307800EB800101EBC00005EB8010E1
:10020000C0F80C803EE048780DF068FB802823D9C8
:1002100040F29C6421462B48F4F774FC009023467E
:1002200029A22BA102A816F08DF93078802209EBC3
:10023000400002A940780DF00BFD307800EB800102
:1002400001EBC00005EB8010C0F80C80C7F82480DB
:100250000DF5027DBDE8F087307800EB800101EB01
:10026000C00005EB8010C0F80CA00DF5027DBDE8C4
:10027000F087307800EB800101EBC00005EB8010C7
:10028000C0F80CA0002C04BF0DF5027DBDE8F0877E
:10029000A2B202A918460AF0ADFC3078A2B209EB6E
:1002A000400002A940780DF0D3FC786A20447862BF
:1002B000DBE700001024002054010020550100203D
:1002C000D8010020E415002056312E353100000001
:1002D00025730D0A25303858253034580D0A000092
:1002E0002DE9F043594FDFF8688100263978012560
:1002F000544CDFF8549183B008EB410101281CD025
:10030000022832D0032840D0042856D005286CD0CB
:1003100006281CBF03B0BDE8F08348780DF0DEFA74
:1003200080287BD2387800EB800101EBC00004EB21
:100330008010C56003B0BDE8F08348780DF0CEFAB8
:100340003028EFD3387809F29C4108EB4000407820
:100350000DF026FD387800EB800101EBC00004EBC6
:100360008010C66003B0BDE8F08337486946B0F836
:10037000CC0417F08CFD3878694608EB40004078D3
:100380000DF00EFD03B0BDE8F08348780DF0A6FA3D
:100390003028C7D3387809F2CE4108EB40004078C6
:1003A0000DF0FEFC387800EB800101EBC00004EB9F
:1003B0008010C66003B0BDE8F08348780DF08EFA77
:1003C0001828AFD3387809F2FE4108EB4000407896
:1003D0000DF0E6FC387800EB800101EBC00004EB87
:1003E0008010C66003B0BDE8F08348780DF076FA5F
:1003F000302897D3387809F2165108EB400040783E
:100400000DF0CEFC387800EB800101EBC00004EB6E
:100410008010C66003B0BDE8F083FFE7387809F2CA
:10042000465108EB400040780DF0BAFC387800EBFC
:10043000800101EBC00004EB8010C66003B0BDE892
:10044000F083000010240020E41500205401002057
:100450005501002000B5094883B009A1027868461B
:1004600016F070F808490748097800EB4100694622
:1004700040780DF095FC03B000BD0000EE010020B7
:100480002564000055010020540100202DE9F041B1
:100490003F4F404EDFF8008182B0012808BF0024A2
:1004A00028D0022845D003284ED0042853D0052850
:1004B00058D006285DD0072862D008281CBF02B09B
:1004C000BDE8F08134486946B0F8580617F0DFFC03
:1004D0003078694607EB400040780DF061FC02B0CF
:1004E000BDE8F08134B130783A2107EB4000407824
:1004F0000DF030FB08EB040595F86A0016F08AFF52
:100500000146307807EB400040780DF023FB95F86A
:100510006A0016F087FF0146307807EB400040780C
:100520000DF018FB601CC4B2062CDBD302B0BDE892
:10053000F081307808F15A0107EB4000407802B0B2
:10054000BDE8F0410DF02CBCD8F8460002B0BDE883
:10055000F041FFF7E7BAD8F84E0002B0BDE8F0412D
:10056000FFF7E0BAD8F84A0002B0BDE8F041FFF763
:10057000D9BAD8F8520002B0BDE8F041FFF7D2BABC
:10058000D8F8560002B0BDE8F041FFF7CBBA000042
:100590005501002054010020E415002000B583B06F
:1005A000132824BF03B000BDDFE800F0690A192852
:1005B000374655646B7279809299ABB3BBC3CB005D
:1005C000634864A190F83221684615F0BBFF634987
:1005D0006148097800EB41006946407874E05C4866
:1005E0005CA190F83321684615F0ACFF5B495A488E
:1005F000097800EB41006946407865E0544855A110
:1006000090F83421684615F09DFF54495248097806
:1006100000EB41006946407856E04D484DA190F806
:100620003521684615F08EFF4C494B48097800EBA0
:1006300041006946407847E0454846A190F83A2194
:10064000684615F07FFF45494348097800EB4100B3
:100650006946407838E03E483EA1B0F8E62068465A
:1006600015F070FF3D493C48097800EB41006946B0
:10067000407829E0364890F8360101281DD003B0B3
:1006800000BD334890F83601022816D003B000BDF3
:100690002F4890F8370101280FD003B000BD2C4837
:1006A00090F83701022808D003B000BD284890F820
:1006B000390101281CBF03B000BD2748274909782C
:1006C00000EB410026A140780DF06AFB03B000BDAD
:1006D0001F4890F839010228EFD003B000BD1C4834
:1006E00090F83B0101281CBF03B000BD1A481B490C
:1006F000097800EB41001AA140780DF051FB03B0DE
:1007000000BD134890F83B0102281CBF03B000BD98
:10071000ECE70F4890F83C0101281CBF03B000BD76
:10072000E4E70B4890F83C0102281CBF03B000BD71
:10073000DCE7074890F83D0101281CBF03B000BD6D
:10074000D4E7034890F83D010228CFD003B000BDA4
:10075000E41500202564000055010020540100200C
:1007600073656C65637465643D2273656C65637461
:100770006564220049490978002908BF704770B5AF
:10078000AAB00D287DD2DFE800F07C070707070735
:100790007C7C7C7C23405000414B4A1E03EBE203EF
:1007A00002F0070293F8F6314FF0010C0CFA02F256
:1007B000134266D03B4A895C814262D13B493A4848
:1007C000097800EB41003AA140780DF0E9FA58E0D1
:1007D000334A481E02EBE00300F0070093F8F631BD
:1007E0004FF0010C0CFA00F003424AD002EB8100FA
:1007F0006946D0F8F40117F071FB2C492A480978B2
:1008000000EB4100694640780CE02648085C03286C
:1008100018BF042835D025492348097800EB41004A
:1008200028A140780DF0BCFA2BE01E481B4D085C57
:10083000032818BF042822D11C4C1B4E207806EB3D
:10084000400040780DF04AF8A1280BD22078012111
:1008500000EB800202EBC0001F4A02EB8010C16077
:100860002AB070BD28786946401EC0B207F07DFEF0
:100870002078694606EB400040780DF091FA0020A0
:1008800028700A480021007800EB800202EBC000CB
:10089000114A02EB8010C1602AB070BDEE01002049
:1008A000E4150020B6180020550100205401002056
:1008B00073656C65637465643D2273656C65637410
:1008C0006564220064697361626C65643D226469D9
:1008D0007361626C65220000102400202DE9F04154
:1008E000404C414E3E4D217884B006EB4101012839
:1008F0002AD0022832D0032818BF052858D007284C
:1009000018BF092854D0042818BF062805D0082885
:100910001EBF0A2804B0BDE8F081001FC0F34F00DD
:1009200005EB800031A190F8833290F8822268466E
:1009300015F008FE2078694606EB400040780DF07F
:100940002FFA04B0BDE8F08195F89002012807BFA6
:10095000487829A104B0BDE8F0813BE048780CF06C
:10096000BDFF2A4F40280BD22078012100EB8002E6
:1009700002EBC00007EB8010C16004B0BDE8F0815D
:100980004FF0000885F8D082207805F2912106EB1F
:10099000400040780DF004FA207800EB800101EB74
:1009A000C00007EB8010C0F80C8004B0BDE8F081F7
:1009B000C01EC0F34F0005EB80000CA190F88132FF
:1009C00090F88022684615F0BDFD2078694606EB58
:1009D000400040780DF0E4F904B0BDE8F08100007B
:1009E000E415002054010020550100202530326418
:1009F0003A25303264000000636865636B65643DCE
:100A000022636865636B6564220000001024002087
:100A10002DE9F043244CDFF89480254DE07991B026
:100A20001F2834D2DFF88C90234F244E287806EB11
:100A3000400040780CF052FF40280BD2287801216A
:100A400000EB800202EBC00008EB8010C16011B027
:100A5000BDE8F083E27999F9D10257F8223090424B
:100A600004D117A1684615F06DFD03E022A1684688
:100A700015F068FD2878694606EB400040780DF0D7
:100A80008FF9E079401CC0B2E0711F28CED300215D
:100A9000E171287800EB800202EBC00008EB8010C7
:100AA000C16011B0BDE8F083D801002010240020FF
:100AB00054010020E415002078AB02085501002005
:100AC0003C6F7074696F6E2073656C6563746564E8
:100AD0003D2273656C6563746564222076616C7574
:100AE000653D222564223E474D5425733C2F6F708F
:100AF00074696F6E3E0000003C6F7074696F6E2009
:100B000076616C75653D222564223E474D54257300
:100B10003C2F6F7074696F6E3E00000000B58DB0A1
:100B20000A2824BF0DB000BDDFE800F01905050557
:100B3000051B2A31425000EBC0002849122201EB6C
:100B4000400000F1D601684607F0BCF92549244869
:100B5000097800EB4100694640780DF021F90DB0AD
:100B600000BD1E4820A190F83021684615F0EAFC2F
:100B70001C491B48097800EB41006946407813E0A6
:100B80001648D0F85A06FEF7CDFF0DB000BD134849
:100B900008A9B0F85E0617F07AF9124910480978EA
:100BA00000EB410008A940780DF0FAF80DB000BD47
:100BB000112208A94FF4D8300AF01CF80949084856
:100BC000097800EB410008A94078EDE705490448A1
:100BD000097800EB410005494078E5E7E41500207D
:100BE000550100205401002025640000441C002011
:100BF00010B5104C8AB02078002804BF0AB010BD90
:100C00000D4901EB800042790179CDE90012C378EA
:100C100082780AA102A815F095FC0C490A480978C7
:100C200000EB410002A940780DF0BAF800202070D6
:100C30000AB010BDEE010020E415002025642564F3
:100C400025642564000000005501002054010020A7
:100C500005490448097800EB4100044940780DF04B
:100C60009FB8000055010020540100201F190020EA
:100C700005490448097800EB4100044940780DF02B
:100C80008FB8000055010020540100202F190020CA
:100C900005490448097800EB4100044940780DF00B
:100CA0007FB800005501002054010020FF180020EB
:100CB00005490448097800EB4100044940780DF0EB
:100CC0006FB8000055010020540100200F190020CA
:100CD00010B52A4C00218AB0627882421CBF0AB04B
:100CE00010BD2278002A04BF0AB010BD012804BF3D
:100CF000501EC1B209D0022808BFD01D04D003285D
:100D000008BF02F1270000D1C1B21D4801F007035E
:100D100000EBD1024FF0010C92F840210CFA03F3E2
:100D20001A4225D0A1F1280201EB41010844102A02
:100D300090F84A1100910AD290F8491190F8482190
:100D40007031CBB20FA102A815F0FCFB07E090F8C0
:100D5000493190F848210BA102A815F0F3FB0E4988
:100D60000C48097800EB410002A940780DF018F812
:100D70000020207060700AB010BD0000EE0100205D
:100D8000E415002025303364253033642530336486
:100D900000000000550100205401002005490448CE
:100DA000097800EB4100044940780CF0F9BF0000DD
:100DB0005501002054010020CF8602082DE9F041A2
:100DC000244C254F254D607990B010283CBFDFF8AA
:100DD0009080244E30D2287806EB400040780CF00A
:100DE0007DFD40280BD22878012100EB800202EB28
:100DF000C00007EB8010C16010B0BDE8F0816079E1
:100E000098F80010421C9142134604D116A168467E
:100E100015F098FB03E021A1684615F093FB2878B4
:100E2000694606EB400040780CF0BAFF6079401C40
:100E3000C0B260711028CED300216171287800EB18
:100E4000800202EBC00007EB8010C16010B0BDE86B
:100E5000F0810000D801002010240020540100205F
:100E6000EE010020550100203C6F7074696F6E2008
:100E700073656C65637465643D2273656C6563744A
:100E80006564222076616C75653D222564223E25CD
:100E9000643C2F6F7074696F6E3E00003C6F70741D
:100EA000696F6E2076616C75653D222564223E2552
:100EB000643C2F6F7074696F6E3E00002DE9F04145
:100EC000224E0446204F307807EB400040780CF06B
:100ED00005FD1F4D20280AD23078012100EB800249
:100EE00002EBC00005EB8010C160BDE8F08119483D
:100EF000016801F00300012802D011F0800F01D039
:100F0000012C0ED001F08302022A08BF022C08D067
:100F1000032C0DD1012818BF022809D011F0800F31
:100F200006D130780CA107EB400040780CF038FF78
:100F30003078002100EB800202EBC00005EB80104E
:100F4000C160BDE8F081000055010020540100207F
:100F500010240020801C002073656C656374656438
:100F60003D2273656C656374656422002DE9F04170
:100F7000354C344DA6B0207805EB400040780CF09D
:100F8000ADFC012178282078304A00EB800303EB88
:100F9000C00002EB801050D32D4EC160327A102A6F
:100FA00024BF0021317248D22A4B02F1280003EB02
:100FB000D00C00F007009CF840C101FA00F01CEAD8
:100FC000000F08BF24A10AD02948104480790328C3
:100FD00008BF28A103D001280CBF2CA130A102EB2F
:100FE000820003EB800090F85B33002B0CBF31A331
:100FF00000F25B3390F86EC390F86D7390F86C83D9
:10100000CDF81CC0CDF81080CDE9052790F86B0312
:10101000CDE90021CDE90220284908A815F092FA6F
:10102000207808A905EB400040780CF0B9FE307A32
:10103000401C307226B0BDE8F081C16026B0BDE82A
:10104000F0810000550100205401002010240020F0
:10105000D8010020E4150020706963747572652F53
:101060004C45445F554E5553452E706E6700000049
:10107000801C0020706963747572652F4C45445F55
:10108000554E4B4E4F572E706E670000706963745B
:101090007572652F4C45445F4F4E2E706E67000091
:1010A000706963747572652F4C45445F4F46462ED8
:1010B000706E6700266E6273703B000054AC0208CD
:1010C00005490448097800EB4100044940780CF0D8
:1010D00067BE00005501002054010020E28602088E
:1010E0002DE9F0415248BCB0028843889A4204BFBF
:1010F0003CB0BDE8F0814F4890F8150300280CBFC4
:101100004D4D4E4D4E4C208AD8B1608ADFF8348167
:101110004D4F002818BF4D4E7CD0387806EB40006C
:1011200040780CF0DBFBC8283CD23878012100EB7A
:10113000800202EBC00008EB8010C1603CB0BDE84B
:10114000F0814348007800EB4000C000A082411CC1
:10115000218237499A42B1F802C00988A1EB0C01FB
:1011600098BF01F58061618289B2B1F5007F84BFCB
:101170004FF40071618289B2091A89B2618218291B
:1011800084BF182161823249294B824209781B8829
:1011900001EB4101A3EBC1018CBF481C01F20140EE
:1011A000A082B2E72B493AA807F070FC9DF8EF0047
:1011B00028289ABF05EB800050F8040C26A09DF863
:1011C000EE109DF8ED309DF8EC20CDE90510CDE94D
:1011D00003239DF8EA109DF8E900CDE900019DF890
:1011E000EB2002929DF8E830228A1C4908A815F0ED
:1011F000A9F9387808A906EB400040780CF0D0FD3A
:10120000608A401E0004000C6082218A01F1010105
:10121000218282D100212182387800EB800202EB0A
:10122000C00008EB8010C1603CB0BDE8F081000058
:101230009E000020E415002038AA0208D8AA02085F
:10124000D801002010240020540100205501002066
:10125000EE010020EC01002000000000F4AB0208C9
:1012600070B52C492A4A0128097802EB41012A4A23
:10127000138852880FD0022810D0032817D0274C8B
:10128000042894F800C01BD0052818BF70BDBCF11D
:10129000000F39D134E0934203D170BD934218BF9F
:1012A00070BD4878BDE870401DA10CF079BD934237
:1012B00018BF70BD4878BDE870401FA10CF070BD2C
:1012C000154C002065882488641B93423CBF04F5BC
:1012D000806080B288BFA0B204D0B0F5007F88BF24
:1012E0004FF400700CF1010202EB4202B0EBC20FAE
:1012F00088BF70BD4878BDE8704013A10CF050BDA8
:10130000487811A10CF04CFD0020207070BD000049
:1013100055010020540100209E000020EE01002015
:101320007374796C653D22646973706C61793A6E8F
:101330006F6E652200000000646973706C61793A19
:101340006E6F6E650000000064697361626C6564B5
:101350003D2264697361626C65220000F0B52C4F18
:101360002C4D2D4E396883B0012807D0022814D0A7
:10137000032808BF002439D003B0F0BD274801423C
:101380001CBF03B0F0BD307825A105EB40004078CC
:1013900003B0BDE8F0400CF003BD002211F4806FF3
:1013A00018BF012211F4006F18BF42F0020211F0C1
:1013B000100F18BF42F0040211F4800F18BF42F062
:1013C00008021DA1684615F0BDF83078694605EBA6
:1013D000400040780CF0E4FC03B0F0BD34B130784C
:1013E0002C2105EB400040780CF0B4FB381969461D
:1013F000807D16F04CFD3078694605EB4000407862
:101400000CF0CEFC601CC4B2282CE7D303B0F0BDB6
:10141000801C00205501002054010020040F4000D2
:101420007374796C653D22646973706C61793A6E8E
:101430006F6E6522000000002564000010B5F3F710
:1014400045FE04480168044A01F4E061114301606B
:1014500010BD00000CED00E00400FA0509480A4A3E
:10146000007800EB800101EBC00102EB8111C97E25
:10147000802908BF7047054901EB400004A140786E
:101480000CF08EBC540100201024002055010020D7
:1014900064697361626C65643D2264697361626C46
:1014A000652200002DE9F047274D80460C46A878BC
:1014B000DFF89890264E90B0A0423CBFDFF894A091
:1014C000254F34D2307807EB400040780CF006FA14
:1014D00040280BD23078012100EB800202EBC000E3
:1014E00009EB8010C16010B0BDE8F087A8789AF8C9
:1014F0000010421C914204BF9AF801104145134666
:1015000004D116A1684615F01DF803E020A1684635
:1015100015F018F83078694607EB400040780CF079
:101520003FFCA878401CC0B2A870A042CAD30021DA
:10153000A970307800EB800202EBC00009EB80104C
:10154000C16010B0BDE8F087D80100201024002051
:1015500054010020EE010020550100203C6F707402
:10156000696F6E2073656C65637465643D22736595
:101570006C6563746564222076616C75653D222517
:1015800064223E25643C2F6F7074696F6E3E0000CC
:101590003C6F7074696F6E2076616C75653D2225B5
:1015A00064223E25643C2F6F7074696F6E3E0000AC
:1015B0002DE9F041254CDFF89880264DE07890B079
:1015C00028283CBF244F254E2DD2287806EB40001A
:1015D00040780CF083F940280BD22878012100EBE9
:1015E000800202EBC00008EB8010C16010B0BDE8C3
:1015F000F081E0783978421C914204BF79785A2909
:1016000013461DD016A1684614F09CFF2878694641
:1016100006EB400040780CF0C3FBE078401CC0B201
:10162000E0702828D1D30021E170287800EB8002F7
:1016300002EBC00008EB8010C16010B0BDE8F08183
:101640000FA1684614F07EFFE0E70000D8010020FB
:101650001024002054010020EE010020550100203C
:101660003C6F7074696F6E2076616C75653D2225E4
:1016700064223E25643C2F6F7074696F6E3E0000DB
:101680003C6F7074696F6E2073656C65637465641C
:101690003D2273656C6563746564222076616C75A8
:1016A000653D222564223E25643C2F6F7074696F6E
:1016B0006E3E00002DE9F04FDFF8308291B098F8CF
:1016C0000030002B04BF11B0BDE8F08F98F801C0C6
:1016D000874F884D4FF0000A3A78BCF15A0F05EB5E
:1016E00042022DD0BCF1560F1CBF11B0BDE8F08FE7
:1016F000032800F0C8807D4A7F490428127801EB56
:10170000820100F0C880052800F0DC80062807BFB1
:1017100091F85F02012811B0BDE8F08F91F85E22C8
:1017200076A1684614F00EFF3878694605EB400054
:1017300040780CF035FB88F800A011B0BDE8F08FC0
:10174000DFF8BCC1012828D0022830D0DFF8B491DE
:101750004FF0010B07283AD0082855D009281CBFA4
:1017600011B0BDE8F08F684E3079112838BF674C52
:101770007BD2387805EB400040780CF0AFF8402879
:101780004AD2387800EB800101EBC00009EB8010F1
:10179000C0F80CB011B0BDE8F08F13F80C0000F0E9
:1017A0001F0088421CBF11B0BDE8F08F08E013F89D
:1017B0000C00C0F3411088421CBF11B0BDE8F08F8F
:1017C000507853A10CF0ECFA11B0BDE8F08F5078CE
:1017D0000CF084F81128D4D398F800006946401E14
:1017E000C0B214F00EFE3878694605EB4000407830
:1017F0000CF0D6FA387800EB800101EBC00009EB61
:101800008010C0F80CA096E7212B3CBF507845A172
:1018100053D311B0BDE8F08F98F800003279005D25
:101820003AB1904213460FD143A1684614F08AFEA4
:101830000EE020B14DA1684614F084FE08E052A1EC
:10184000684614F07FFE03E05BA1684614F07AFE60
:101850003878694605EB400040780CF0A1FA307901
:10186000401CC0B23071112883D386F804A03878A8
:1018700000EB800101EBC00009EB8010C0F80CA068
:1018800011B0BDE8F08F8B4207BF507820A111B096
:10189000BDE8F08F11E091F85F0201281CBF11B084
:1018A000BDE8F08F91F85C2214A1684614F04AFE5E
:1018B0003878694605EB400040780CF071FA11B0B9
:1018C000BDE8F08F91F85F0201281CBF11B0BDE8A0
:1018D000F08F91F85D2209A1684614F033FE387844
:1018E000694605EB40004078E7E70000EE01002084
:1018F0005401002055010020E4150020256400005B
:101900001B18002010240020D8010020551C0020A6
:1019100073656C65637465643D2273656C6563749F
:101920006564220064697361626C65643D22646968
:101930007361626C656422003C6F7074696F6E2025
:1019400073656C65637465643D2273656C6563746F
:101950006564222076616C75653D222564223E25F2
:10196000643C2F6F7074696F6E3E00003C6F707442
:10197000696F6E2076616C75653D2230223E3C2F8A
:101980006F7074696F6E3E003C6F7074696F6E208B
:1019900073656C65637465643D2273656C6563741F
:1019A0006564222076616C75653D2230223E3C2FB5
:1019B0006F7074696F6E3E003C6F7074696F6E205B
:1019C00076616C75653D222564223E25643C2F6F4F
:1019D0007074696F6E3E0000074890F8BC000128E3
:1019E00018BF704705480649097800EB410005A17A
:1019F00040780CF0D5B90000E41500205501002016
:101A000054010020636865636B65643D226368650B
:101A1000636B65642200000003480168034A01F417
:101A2000E0611143016070470CED00E00400FA052D
:101A300006490978814218BF704705480549097869
:101A400000EB410004A140780CF0AAB9EE0100209F
:101A5000550100205401002073656C656374656452
:101A60003D2273656C6563746564220010B512488D
:101A70000F4C104A0078A17B02EB4000012940780E
:101A800011D0022908BF0DA107D0032908BF0DA15D
:101A900003D004290CBF0EA111A10CF081F9002084
:101AA0002070A07310BD10A10CF07AF9F7E70000C8
:101AB000D801002055010020540100207375636394
:101AC000657373007765625570646174650000002A
:101AD000736F667477617265557064617465000038
:101AE0006E6F6E65000000006572726F720000001C
:101AF0002DE9F04F87B0FE4FA7F10108012498F8B7
:101B0000000017F810000C2880F00E86DFE810F0B7
:101B10000C004800890246037D038703CC03E503DC
:101B200022052F05AD05D10598F8000007EB400010
:101B300040780BF0B3FE002800F0F68598F800001E
:101B4000EC4E00EB800101EBC00106EB811101F1CD
:101B50001E020A61012207F81020FF20C876002526
:101B60008D760DF063F94AF6C871421898F80000B6
:101B700000EB800101EBC00106EB81118A604FF0A0
:101B8000FF32CA600D6081F83E5307EB40004FF012
:101B9000050340784FF000024FF001010AF0EEFC1F
:101BA0004FF0000ACDF800A098F80000534607EB6C
:101BB0004000524640780A210BF09AFAA0F57F4186
:101BC000FF3933D198F8000007EB400040780BF064
:101BD000ABFB70B998F80000C64B00EB800202EB3B
:101BE000C00203EB821205211177072107F81010BC
:101BF00000240DF01BF998F80010BE4B01EB810298
:101C000002EBC10203EB82129268801A002840F3B3
:101C10008B8507EB410040780BF000F998F8001035
:101C20000B2007F81100002400F07EBD0DF0FEF837
:101C30004AF6C871411898F80000AE4E00EB8002D9
:101C400002EBC00206EB8212C146916007EB400036
:101C5000CDF800A04FF0000340781A464FF0200165
:101C60000BF046FA052800D90520401C82B299F8ED
:101C7000000000EB800101EBC00107EB400006EB28
:101C800081111E3140780BF0B3FA99F8000003225D
:101C900000EB800101EBC00006EB80101E3096A126
:101CA000F0F751FBE0B199F80000042200EB80014D
:101CB00001EBC00006EB80101E3090A1F0F743FB53
:101CC000C8B199F80000072100EB800202EBC002C6
:101CD00006EB8212117707F81010002400F024BDE3
:101CE00099F8000000EB800101EBC00006EB8010CA
:101CF00080F81CA009E099F80000012100EB8002A7
:101D000002EBC00006EB80100177CDF800A099F837
:101D10000000002307EB40001A46407820210BF01A
:101D2000E7F90546CDF800A099F800002B4607EB2F
:101D30004000002240783F210BF0DAF9854200D2C2
:101D40002846024640F2153082420FD999F8000029
:101D5000052100EB800202EBC00206EB8212117734
:101D6000072107F81010002400F0DEBC99F80000ED
:101D700000EB800101EBC00107EB400006EB811195
:101D80001E3140780BF034FA99F8001001EB810213
:101D900002EBC10106EB8111084480F81EA001F19D
:101DA0001E0000F0C7FE99F8000000EB800101EB77
:101DB000C00006EB80101E30F0F7B0FA85B299F83B
:101DC000000000EB800101EBC00006EB8010411920
:101DD000497F2F290BD01F3004F00AFB99F800101F
:101DE00001EB810202EBC10106EB8111087699F843
:101DF000000000EB800101EBC00006EB8010017ECB
:101E0000FF2922D14119497F2F2905D02F212A46A8
:101E100002446B1C9DB291773AA241191368C1F834
:101E20001E305368C1F822301289CA8405F10901B5
:101E30008DB21F3004F0DCFA99F8001001EB81023A
:101E400002EBC10106EB8111087699F8000000EB66
:101E5000800101EBC00006EB801148191D3001F133
:101E60001E02824205D003782E2B02D0401E8242F1
:101E7000F9D100F1010B81F81DA0254D99F8000062
:101E800000EB800101EBC00006EB8010407F55F8AD
:101E90002010584615F022FF68B199F8000000EBB9
:101EA000800101EBC00006EB8010417F491CC9B2E4
:101EB00041770C29E2D399F8000000EB800101EB97
:101EC000C00006EB80101F30F9F702FD99F80010F2
:101ED00001EB810202EBC10106EB8111C876087E9D
:101EE000FF2831D0354604F03DFA10F0020F11E022
:101EF000550100201024002047455400504F5354F2
:101F000000000000696E6465782E68746D00000042
:101F100080A8020818D099F80000CB4600EB800199
:101F200001EBC00005EB8010007E04F035FA401C88
:101F300080B204F0EFFA9BF8001001EB810202EB93
:101F4000C10105EB81114876CDF800A099F8000099
:101F5000002307EB40001A46407820210BF0C8F818
:101F60000546EDB399F80000012100EB800202EB79
:101F7000C00206EB8212917607EB400006A940787A
:101F80000BF0E2F8681E82B240F21E3082420FD39C
:101F900099F80000052100EB800202EBC00206EB7D
:101FA00082121177072107F81010002400F0BCBB43
:101FB00099F800004D4600EB800101EBC00107EBF2
:101FC000400006EB81111E3140780BF011F92978A1
:101FD00001EB810202EBC10106EB81110A6900E00D
:101FE00004E010442622431C0B610270CDF800A0CF
:101FF00099F80000002307EB40001A4640780A21B8
:102000000BF076F8401C82B299F80000002107EB33
:10201000400040780BF0ECF899F80010022007F827
:102020001100DFF878A54FF00009DFF874B59EE0E5
:1020300098F8000007EB400040780BF075F968B99C
:1020400098F80000052100EB800202EBC0020BEBC8
:1020500082121177072107F8101000240CF0E6FE19
:1020600098F8001001EB810202EBC1020BEB821227
:102070009268801A002840F3578307EB41004078AC
:102080000AF0CCFE98F800100B2007F8110000248D
:1020900000F04ABB0CF0CAFE4AF6C871411898F825
:1020A000000000EB800202EBC0020BEB8212916099
:1020B000012D19D007EB4000CDF8009040782B4659
:1020C00000223A210BF014F8801C86B20024102E56
:1020D0001BD9681C82B298F80000002107EB400071
:1020E00040780BF085F842E098F80000022207EBF8
:1020F0004000002140780BF07BF898F80010032096
:1021000007F81100002400F00FBB98F800003246D9
:1021100007EB400002A940780BF06AF802A83044AF
:1021200000F8019CA81B86B2002502A85AF82510C9
:10213000F0F7FBF868B3681CC5B2032DF5D364B1A2
:10214000CDF8009098F80000002307EB40001A46F5
:1021500040780A210AF0CCFF0646701C82B298F83B
:102160000000002107EB400040780BF041F8CDF86B
:10217000009098F80000002307EB40001A464078D2
:102180000A210AF0B5FF0546A5F57F40FF3881D149
:102190004EE72846F9F764FB0124D0E798F80000E1
:1021A000FF4C00EB800101EBC00104EB8111CA7E02
:1021B000802A07D203220A77072107F8101000248B
:1021C00000F0B2BA08690025057098F8000000EB2D
:1021D000800101EBC00004EB80101E3000F0AAFC6F
:1021E00098F8001001EB810202EBC10204EB8212AD
:1021F0001061042007F81100907E10B9052007F83F
:1022000011000024957600F08FBAF0F7F7FC022851
:1022100000F08A8298F80010052007F8110098F85D
:10222000000007EB400040780BF038FB98F80010F6
:10223000DB4D01EB810202EBC10105EB8111C968A5
:1022400088421AD10CF0F2FD98F8001001EB8102DF
:1022500002EBC10205EB82129268801A00280CDDA5
:1022600007EB410040780AF0D9FD98F800100B20E8
:1022700007F81100002400F057BA98F8000000EBAE
:10228000800101EBC00005EB8010007F012806D122
:10229000F9F760F80690022847D0012858D098F83E
:1022A0000010062007F8110098F8000000EB8001EC
:1022B00001EBC002BA4901EB82110A7EFF2A7DD0F0
:1022C00000200860487EFF2879D0091D04F06EF8D0
:1022D00098F80010072007F8110098F80000022372
:1022E00007EB40000022407801210AF047F998F8F6
:1022F0000000AB4D00EB800101EBC00105EB81114B
:10230000A84A097F07EB400052F8211040780BF0F3
:1023100047FD98F8000000EB800101EBC00105EBE0
:1023200081110A7F082A5CD07FE098F8000007EB53
:10233000400040780BF0B2FA411E98F8000000EB24
:10234000800202EBC00005EB8010C16000F0ECB928
:1023500098F8000007EB400040780BF09FFA98F8DF
:10236000001001EB810202EBC10105EB8111C86095
:102370000CF05CFD4AF6C871421898F8000000EBBA
:10238000800101EBC00105EB81118A600A68C96810
:102390008A4207D907EB400040780AF0C5FF0028C1
:1023A00040F0C28198F80000062100EB800202EBA9
:1023B000C00205EB82121177072101E005E00CE075
:1023C00007F81010002400F0AFB904220A770721A3
:1023D00007F81010002400F0A7B94FF0FF30486054
:1023E00076E707EB40001E3140780BF0D9FC98F8F7
:1023F00000006DA107EB400040780BF0D1FC98F88D
:10240000000000EB800101EBC00107EB400005EB91
:1024100081111E3140780BF0C3FC98F80000674929
:1024200007EB400040780BF0BBFC98F8000000EB95
:10243000800101EBC00105EB81110A7F32B1012A55
:1024400004D00B2107F8101000F06EB9497F0C2959
:102450001ED007EB40005AA140780BF0A1FC98F881
:1024600000005B4A00EB800101EBC00105EB81112C
:1024700007EB4000497F407852F821100BF090FCA8
:1024800098F800004D4907EB400040780BF088FCBD
:1024900098F8000000EB800101EBC00105EB811111
:1024A000497F0B290DD107EB40004AA140780BF082
:1024B00077FC98F80000414907EB400040780BF0AA
:1024C0006FFC98F8000000EB800101EBC00005EB09
:1024D0008010007E03F046FF10F0010F07D098F83F
:1024E00000004AA107EB400040780BF059FC98F837
:1024F00000004DA107EB400040780BF051FC98F82C
:1025000000004DA107EB400040780BF049FC98F823
:1025100000002A4907EB400040780BF041FC98F896
:10252000000000EB800101EBC00105EB8111897E09
:1025300019B1082107F810100AE007EB40001F4905
:1025400040780BF02DFC98F80010092007F81100D6
:102550000024E9E098F80000184907EB40004078B3
:102560000BF01EFC98F80010092007F81100002459
:1025700000F0DAF988B198F80000094C00EB80010E
:1025800001EBC00004EB8010007E03F03FFE98F8E2
:102590000000FF2100EB800254E05CE010A902087B
:1025A00010240020E8A802080D0A0D0A3330342058
:1025B00052656469726563743A2000007CA8020861
:1025C000436F6E74656E742D547970653A20000007
:1025D000B4A80208436F6E74656E742D44697370FD
:1025E0006F736974696F6E3A206174746163686DAA
:1025F000656E743B2066696C656E616D653D436F09
:102600006E6669672E62696E00000000436F6E742B
:10261000656E742D456E636F64696E673A20677AE4
:1026200069700D0A0000000043616368652D436F07
:102630006E74726F6C3A20006E6F2D636163686513
:102640000000000002EBC00204EB821211760B21A5
:1026500007F81010012498F8000007EB40004078BC
:102660000BF03CF920BB01245EE098F8000007EB7A
:10267000400040780BF032F9102855D398F800004C
:102680002C4D00EB800101EBC00005EB8010806851
:10269000FCF708FF98F8000000EB800101EBC00197
:1026A00005EB8111C96819B90024092107F8101038
:1026B0003AE098F800001F4D00EB800101EBC000EC
:1026C00005EB8010007EFF280BD003F09FFD98F8EB
:1026D0000000FF2100EB800202EBC00005EB801040
:1026E000017698F8000000EB800101EBC00005EBDB
:1026F0008010407EFF280BD003F088FD98F8000082
:10270000FF2100EB800202EBC00005EB8010417658
:1027100098F8000007EB400040780AF07FFB98F83B
:102720000010002007F81100002C3FF4E7A907B0C3
:10273000BDE8F08F1024002070B504460A462146FB
:102740003D2000F03BF8054624B1207810B120462A
:1027500000F0F0F9284670BD2DE9F04104460E4620
:1027600032462146262000F029F80746022F18D1CC
:102770001048451E297800EB410040780BF08EF898
:10278000297801EB810202EBC1010B4A02EB8111B6
:102790000968884205D132462146002000F00EF833
:1027A000074624B1207810B1204600F0C3F938461E
:1027B000BDE8F08155010020102400202DE9F84FDC
:1027C00082460D461646564F4FF0000B07F10108A2
:1027D0003878BAF1000F08EB4000407808D00023A9
:1027E0001A465146CDF800B00AF082FC044602E0D9
:1027F0000BF054F80446A4F57F40FF3802D10220C4
:10280000BDE8F88FDFF81C91022E15D2A5B13878FB
:10281000224608EB4000002140780AF0E9FC01461E
:10282000387800EB800202EBC00009EB80100268F0
:10283000511A016001245AE075B3B01E844240DD94
:1028400082B23878294608EB400040780AF0D0FC84
:102850000246387800EB800101EBC00109EB8111E1
:102860000B689A1A0A60A11B891C08EB40008AB207
:10287000407800210AF0BCFC0146387800EB800269
:1028800002EBC00009EB80100268511A0160A81920
:1028900000F802BC01242AE03878224608EB400008
:1028A000002140780AF0A4FC0146387800EB800251
:1028B00002EBC00009EB80100268511A016000248D
:1028C00015E03878224608EB4000294640780AF0A7
:1028D0008FFC0146387800EB800202EBC00009EB68
:1028E00080100268511A016005F804B00024BAF1A2
:1028F000000F11D03878002108EB400040780AF032
:1029000023FC0146387800EB800202EBC00009EBA3
:1029100080100268511A01602046BDE8F88F00005F
:1029200054010020102400202DE9F04192B0514FB5
:102930007E1E307807EB400040780AF0CFFF3178F8
:10294000DFF8348101EB810202EBC10108EB811158
:102950000B684A68D21A824200D8104684B218190D
:102960000860F4B1402C01D2224600E040223078C9
:1029700000EB800101EBC00008EB80106946007E8F
:1029800003F098FC0546002D55D030782A4607EB19
:102990004000694640780BF05BF9601B84B2002C64
:1029A000E0D1307800EB800101EBC00108EB811130
:1029B0004B680A689A4258D10A2207F81020002072
:1029C000C860087E002103F049FC307800EB8001EC
:1029D00001EBC00008EB801010A9007E03F03EFC64
:1029E00068B1307800EB800101EBC00008EB80108B
:1029F0000168491C01609DF840007E28E5D13078CF
:102A000000EB800101EBC00008EB80100168491C5D
:102A1000016000F10801407E03F0C8FC307800EB53
:102A2000800101EBC00008EB8010011D407E03F027
:102A3000BDFC20B119E012B00120BDE8F081307872
:102A40004FF0FF3100EB800202EBC00008EB80107A
:102A50004160407E03F0DAFB3078FF2100EB80021A
:102A600002EBC00008EB8010417612B00020BDE8F8
:102A7000F081000055010020102400202DE9F047CE
:102A80000024DFF8AC80294EA2464FF0FF09A8F1E0
:102A9000010708EB44056878FE2841D00BF0A4FD3F
:102AA000A0B33C7008F814A004EB840000EBC40051
:102AB00006EB8010007EFF280AD003F0A7FB3878D1
:102AC00000EB800101EBC00006EB801080F818904D
:102AD000387800EB800101EBC00006EB8010407EEF
:102AE000FF280AD003F092FB387800EB800101EB5D
:102AF000C00006EB801080F819903878042308EBAA
:102B0000400000224078012109F038FD18F8140037
:102B100018B968780AF0C2FE10B13C70FEF7E8FF01
:102B2000601CC4B2022CB4D3BDE8F087102400208E
:102B3000550100202DE9F84304462046EFF7EEFB4F
:102B400085B2264600278DB14FF0200816F8010BFC
:102B5000691E8DB23D280ED026280CD02B280DD012
:102B600025280ED004F8010B002DEFD12770601C32
:102B70000770BDE8F88304F8017BF5E704F8018BE2
:102B8000F2E7022D01D20025EEE730788DF8010042
:102B9000701C461C01788DF80010681E401E85B21E
:102BA000009814F037FD04F8010BDDE770B5184DFF
:102BB00000EB400005EBC004207907280DD0607DB4
:102BC0000BF012FD217DC9B1002101EB410205EBA3
:102BD000C2021379032B0DD101E0012070BDD28810
:102BE000E3889A4206D118B104202071012070BDFB
:102BF000002070BD491CC9B20829E6D330B1607D00
:102C00000AF0F4F807202071012070BD002070BD8B
:102C1000042300202DE9F04F89B082460F469AF830
:102C20000D50DAF80840DAF804B0FE4EDFF8F88309
:102C3000307800EB400101EBC00008EB800090F819
:102C4000251021F0070180F8251011F0100F0CD18C
:102C50000CF0ECF842F210710144307800EB4002C5
:102C600002EBC00008EB8000C1613078EF4B00EB55
:102C7000400101EBC00108EB81004FF0060990F81C
:102C80002420042A22D0052A54D0B94615F0010F79
:102C900003D009F1010C1FFA8CF915F0020F03D0D3
:102CA00009F1010C1FFA8CF9D0F814C08669B445FB
:102CB0007ED3B0F80880B0F804E0ACEB060CA8EBCB
:102CC0000E08A8EB0C0C1FFA8CF892E015F0040F1C
:102CD00004D009B0BDE8F04FF2F740B815F0100F7E
:102CE00009D05C600021042008F052F909B0BDE869
:102CF000F04FF2F733B815F0020F16D00BF10100C8
:102D00001C469860F5F7B2FD20850121122008F0DD
:102D10003FF9307800EB400101EBC00008EB800088
:102D200080F8249009B0BDE8F08F09B0BDE8F04FFD
:102D3000F2F714B815F0040FF4D115F0100F0CD001
:102D40005F68A74209D01D466C600121042008F08D
:102D50001FF96F6009B0BDE8F08F15F0020FF9D0D0
:102D60000BF101001C469860BAF80E00A082F5F73E
:102D70007DFD208515F0100F25D00121102008F0D1
:102D800007F93078072100EB400202EBC00008EBA6
:102D9000800080F824100CF049F842F210710144D0
:102DA000307800EB400202EBC00008EB800000E04E
:102DB00019E0C16190F8251021F0100180F825106C
:102DC00009B0BDE8F08F0121122008F0E1F8307859
:102DD00000EB400101EBC00008EB800080F824907C
:102DE00009B0BDE8F08FA6EB0C0CACF1010C1FFA9A
:102DF0008CF88E4B9B68ABEB03039EB24FF0000C3C
:102E0000B9F1000F21D0B8F1000F25D0002B04DB61
:102E1000984502D94FF0010C0CE003EB090EBEF10E
:102E2000000F07DDA8EB090E0FFA8EFE9E4501DBB1
:102E30004FF0010C43450FDA33B20FFA89FE7344A9
:102E4000002B09DD4FF0010C06E0002B0FD003DB57
:102E5000984501D94FF0010CBCF1000F0AD015F0D4
:102E6000060F11D009B0BDE8F04FF1F777BF4FF072
:102E7000010CF1E715F0040FB2D109B00121BDE852
:102E8000F04F102008F084B815F0100FA8D0921F52
:102E9000072A80F06781DFE802F00416161616167E
:102EA000FC00624B5A68A2420AD01E461546746066
:102EB0000121042008F06CF8756009B0BDE8F08FBE
:102EC000072280F82420594BC2680892DB68D21A86
:102ED0000FFA82FCBCF1000F08DADFF84CC1D0F821
:102EE00004E05CF821C0AEEB0C0C6244DFF83CC19E
:102EF000DCF804E0CDF81CE07244A21A002A0EDDD2
:102F00009CF826E01EF0010F01D0012A06D009B07E
:102F10000021BDE8F04F102008F03AB8641ED0F848
:102F200010C0A3EB0C020FFA82FE079AA2EB0E026E
:102F30000692029263450AD23B4AD0F804E052F866
:102F40002120AEEB020E029AA2EB0E020292029A2E
:102F5000A21A0292029A002A44DDDFF8CCE042680D
:102F600005925EF821E0A2EB0E02DDF808E0724562
:102F700038D3DFF8B8E09EF8261021F0080121F0E0
:102F800010018EF8261090F8261021F0010180F82B
:102F9000261002996144016163450AD38B4213D222
:102FA000A1EB030C079B6344CEF80430CEF80C1061
:102FB0000AE01344994207D9DDF81CC0CB1A6344D8
:102FC000CEF80430CEF80C10059B994201D3891A33
:102FD0000161DEF80C10059B99423FD3891ACEF8A7
:102FE0000C103BE09C4539D0104A92F82620049200
:102FF00012F0080F2BD0049A12F0100F21D0DFF836
:103000002CE0069ACEF8042063450AD2AEF5257E60
:1030100083883EF82110591A0BB20EF52571D21A89
:103020004A6005E0A2010020E4510020785400200D
:10303000FE49C1F80CC090F8261041F0040180F858
:103040002610FA49049A42F0100281F82620F74926
:1030500091F8262042F0080281F82620026908999A
:103060008A4219D190F8261011F0080F1ED0EF4AAD
:103070005368A34210D192F8262012F0010F0BD012
:1030800090F8252022F0100280F8252021F0080178
:1030900000E0E3E080F82610E44BBAF80E0059682F
:1030A0000A1B801A82B2988AB0B125E00BF0BEFEEE
:1030B00042F210710144DE48007800EB400202EB5E
:1030C000C002DC4800EB8200C16190F8251021F0BD
:1030D000100180F82510DFE772B1D548007800EBC9
:1030E000400C0CEBC00CD34800EB8C0090F826C0D1
:1030F0004CF0020C80F826C09A82CD48007800EB94
:10310000400202EBC002CB4800EB820090F82400A2
:10311000082804D0092822D00A287DD022E0A14224
:1031200020D193F8260010F0010F1BD00BF07EFE8B
:1031300041F288310144BE48007800EB400202EBC6
:10314000C002BC4800EB8200C16190F8251041F03C
:10315000100180F82510092180F8241002E015F0F4
:10316000010F69D015F0200F7FF4A7AEB0490878A1
:1031700000EB400202EBC000AE4A02EB800090F888
:1031800024000B283FF499AE0A283FF496AE0C2891
:103190003FF493AE002F7DD030B2039000287ADC4C
:1031A0009AF80C000009C6EB800080B200F056FBD4
:1031B000B81986B2464500D946469C4881683144D4
:1031C0008160DFF86C82DFF86CA298F8000000EBF9
:1031D000400101EBC0000AEB800148698A6883194D
:1031E000934246D9121A571CBAB20092002391F8A2
:1031F00029105A1E0AF0E1FDF71BB8B2009098F8AA
:103200000000002300EB400101EBC0000AEB80004E
:1032100090F82910406800E018E05A1E0AF0CDFD31
:1032200098F8000000EB400101EBC0000AEB8000C1
:1032300041683944416131E05C600021142007F0AD
:10324000A7FE09B0BDE8F04FF1F788BDA1427FF4B9
:1032500034AE09B0BDE8F04FF1F780BD7348406867
:10326000401CA0427FF429AE09B0BDE8F04FF1F751
:1032700075BD0096002391F829105A1E0AF09DFD95
:1032800098F8000000EB400101EBC0000AEB800061
:10329000416901E07BE032E031444161634AB2F9C7
:1032A0002400411C73D0801B01B29184D08A084451
:1032B0000FFA80FC4FF0FF33BCF1000F01DA93846A
:1032C0009DE0002963DC91680144916098F800104A
:1032D00001EB410C0CEBC1010AEB8101D1F814C0E8
:1032E00060444861D1F808C0604506D94E68ACEB2F
:1032F000060CA0EB0C00401E486193847FE0B819D7
:10330000404502D9A8EB060087B29AF80C000009E4
:10331000800000F0A3FA464BDFF818C106EB07085F
:10332000187800EB400101EBC0000CEB800148690C
:103330008A6800EB080A924537D9A2EB000AAAEB8B
:10334000060A0AF1010A0FFA8AFEBEF1000F1FDB1E
:103350001FFA8AF20092002391F8291030445A1E75
:103360000AF02BFDA7EB0A0080B200903048002342
:103370005A1E007800EB400101EBC0012D4800EB24
:10338000810090F8291040680AF017FD15E036E03A
:1033900000974B683044D21A801A0023401E91F8DF
:1033A00029105A1E0AF009FD07E00097002391F842
:1033B000291030445A1E0AF000FD1C4AB2F92400BC
:1033C000401C0AD0908CB04210D9D18A01444145AA
:1033D00001D3804505D2D78205E003989084D78237
:1033E0000DE0881BD0820398908408E0D18A0144C4
:1033F000414504D2B14202D3A8EB0000D082B9F11A
:10340000000F36D00A4F0B4E387800EB400101EB2D
:10341000C00006EB800090F82410072901D0416914
:10342000816190F8251011F0800F05E0785400209C
:10343000A2010020E451002006D00121102007F055
:10344000A7FD08F00DFC14E041F0800180F8251084
:1034500011F0400F0DD141F0400180F825100BF024
:10346000EDFC397801EB410202EBC10106EB810171
:10347000488415F0010F3FF420AD2B4A0BEB0901F6
:103480009068411A491C7FF418AD401C9060274D8C
:10349000A2F52576287800EB400101EBC00006EB91
:1034A000800191F82400062806D007280ED00828AD
:1034B0001AD0092827D12DE00C2081F8240009B06A
:1034C0000121BDE8F04F112007F062BD0B2081F80B
:1034D00024000BF0B3FC297801EB410202EBC1019F
:1034E00006EB810148840EE05068A04208D100211B
:1034F000102007F04DFD09B0BDE8F04FF1F72EBCEC
:103500000A2081F8240009B00121BDE8F04F102005
:1035100007F03EBD0021102007F03AFD09B0BDE8DC
:10352000F04FF1F71BBC000078540020A2010020EE
:103530002548017A090646D5C18801F10101C180FB
:10354000017A027A01F1010161F3050202721F4959
:103550008A68120424D5027A520621D4027A002302
:1035600002F03F02052A08D9027A02F03F020A2A35
:1035700003D24288521C42800CE0027A02F03F02E1
:10358000022A08D9027A02F03F02062A03D20288F0
:10359000521C0280C380027A22F03F0202720BE0CA
:1035A00042883C2A08D90288142A05D2C288B2F57A
:1035B000FA7F01D9C28882808968C1F3C032017A5A
:1035C00062F386110172704754050020001001401B
:1035D0000F490020CA88B2F5966F18D94A88502A38
:1035E0000BD90A88B42A08D94A88C82A05D20A8879
:1035F000B2F58C7F01D2012004E04A88B2F5487F01
:1036000000D902200022CA804A800A808A8070473E
:10361000540500200E49012804D0087A20F08000CB
:10362000087270470020088048808880C880087A27
:1036300020F03F00087207488068C0F3C032087A63
:1036400062F386100872087A40F08000E8E7000014
:10365000540500200010014070B50C4D4FF4004699
:103660002E606A142A60002154102B1F002801DAF2
:103670001C6000E02C6040001A602A60491CC9B23E
:103680002029F3D31E602E6070BD0000140C014091
:1036900030B50446002002460EE00301A05CA0F114
:1036A0003005092D01D8303B04E0A0F14105052D7E
:1036B00005D8373B1844521C8A42EEDB30BD00204F
:1036C00030BD704738B505460C460421684602F007
:1036D000F7F9BDF80000082837D12146142002F080
:1036E000C7F8002831D18DF800009DF8020008309D
:1036F000C0B28DF80200082809D29DF80310491CB9
:10370000CBB28DF8033013B9401C8DF8020002F0E3
:10371000ADFB0028FBD040F6DD2002F055FD22462F
:103720000121284600F05CF80421684602F0B2FC52
:10373000201F82B24FF0FF31084602F0A2FB02F0D8
:103740008AFB0028FBD002F0EFF838BD2DE9F043EA
:1037500087B004460E4617469846142101A802F089
:10376000AFF99DF8040000F0F001402903D007B044
:103770000020BDE8F083BDF80A1031F0E00103D06D
:1037800007B00020BDE8F083DFF850900007810EFD
:1037900089F80010002002F06BF80546069099F8B1
:1037A000000002F0F5FC1DB107B00020BDE8F08379
:1037B00001A808F0E6F80CB1059820600498306084
:1037C0009DF80D003870BDF8060099F80010401AF9
:1037D000A8F8000007B00120BDE8F0835A010020DE
:1037E00030B585B005461B481423037045238DF87A
:1037F00000304FF0000C8DF801C0143294B2ADF8D7
:1038000002404288531C4380ADF80430ADF806C036
:103810007F208DF808008DF80910ADF80AC00E4819
:103820000068039028680490684608F0AAF81421FC
:103830006846F1F7E5F9ADF80A0022460021281D97
:1038400002F056FC1421684602F024FC05B000206A
:1038500030BD00005A010020555C00200249097863
:10386000084480B202F094BC5A01002073B50646A9
:1038700082B000203070044603AD04E01CB10AA100
:103880003046EEF717FD285D694614F000FB6946E7
:103890003046EEF70FFD641CE4B2042CEED3304644
:1038A000EEF73CFD04B070BD2E00000030B5CCB288
:1038B0006422B4FBF2F302FB134503700A23B5FB49
:1038C000F3F54570B4FBF3F503FB15448470C1F3C5
:1038D0000724B4FBF2F5C57002FB1545B5FBF3F503
:1038E0000571B4FBF3F503FB15444471C1F30744C0
:1038F000B4FBF2F5857102FB1545B5FBF3F5C57117
:10390000B4FBF3F503FB15440472090EB1FBF2F4AA
:1039100002FB1412B2FBF3F244728272B1FBF3F2B7
:1039200003FB1211C17230BD10B545F2555000F0C5
:1039300029F8022000F01AF840F6FE7000F01CF89A
:1039400000F00CF8BDE81040AFF3008002494CF6DF
:10395000CC400860704700000030004002494AF641
:10396000AA2008607047000000300040014948600C
:103970007047000000300040014988607047000037
:1039800000300040014908607047000000300040EE
:1039900070B51F4C607E282801D3002060761D4A38
:1039A0000121C0B202EBD00300F0070593F84430C8
:1039B00001FA05F52B4224D008F002FC607EE721D5
:1039C000401C60764C200CF0B7FF402154200CF0D6
:1039D000B3FF607E0A25B0FBF5F00F4E315C5C2032
:1039E0000CF0AAFF607EB0FBF5F105FB1100305C26
:1039F00040F0100164200CF09FFF4FF448706060AD
:103A000070BD401CC0B260762828CAD370BD0000CB
:103A1000E41D0020801C0020148702082DE9F041DD
:103A2000334F16463B4684463A7F481E5B7F0A2A40
:103A300007D2FA54797F814201DA491C7977BDE8CF
:103A4000F0812C4C2C4D0E2A0ED00D2A13D00C2AAE
:103A500015D00A2A18D00F2A01D00B2AEFD1002244
:103A600012234FF0500C2BE0A07800EB800005EB08
:103A70008000008936E08342E1DA5B1C02E0002B23
:103A8000DDD05B1E7B77DAE7634501D287F81DC086
:103A9000787F0A2202E03A54401CC0B28842FAD32E
:103AA000787F6045CBD9401E7877C8E7012804D0DD
:103AB000B85C0E2818D0092800D9BB54521CD2B2C9
:103AC00000208A42F2D30A4609493046EEF7CEFB7F
:103AD00000210A480BF046FFA07800EB800005EBC0
:103AE0008000C0882080AAE707F802C0E6E700004F
:103AF000C015002070000020888C0208EA870208A8
:103B00002DE9F041164D2C7F0F2C05D00B2C03D046
:103B1000BDE8F04100F0DEB9002420464FF6FF7604
:103B200008E02F5C04EB840406EA44043C44401C97
:103B3000A4B2C0B29042F4D3FF2901D91C8000E0A6
:103B40001C70002107480BF00DFF0749074A8878D1
:103B500000EB800002EB8000C0880880BDE8F081A7
:103B6000C0150020EA87020870000020888C020837
:103B700070B50E462549024608460B7F407F0A2B4A
:103B80000FD2904202D20B54487F31E02048008887
:103B900010F4C04F31D11F48017841F0020101708B
:103BA0002BE01D4C1D4D0F2B08D00B2B06D00E2BE0
:103BB00013D00D2B19D00C2B1CD01EE0134930460E
:103BC000EEF754FB002116480BF0CCFEA07800EB7A
:103BD000800005EB8000C08805E0A07800EB800045
:103BE00005EB80000089208007E0521E904204DA35
:103BF000401C01E008B1401E48770A48012141609D
